MPLINK 4.43, Linker
Linker Map File - Created Tue Aug 24 08:29:43 2021

                                 Section Info
                  Section       Type    Address   Location Size(Bytes)
                ---------  ---------  ---------  ---------  ---------
               _entry_scn       code   0x000000    program   0x000006
           .code___init.o       code   0x000006    program   0x000002
               highVector       code   0x000008    program   0x000006
             .stringtable    romdata   0x00000e    program   0x00000a
                lowVector       code   0x000018    program   0x000006
                   .cinit    romdata   0x00001e    program   0x000086
       .code_MainDemoV1.o       code   0x0000a4    program   0x013242
              .code_TCP.o       code   0x0132e6    program   0x00452c
              .code_UDP.o       code   0x017812    program   0x000f3a
 .code_GenericTCPClient.o       code   0x01874c    program   0x000bda
          .code_Helpers.o       code   0x019326    program   0x000abc
              .code_DNS.o       code   0x019de2    program   0x000a28
         .code_ETH97J60.o       code   0x01a80a    program   0x0009b0
 .code_GenericTCPServer.o       code   0x01b1ba    program   0x00055e
              .code_ARP.o       code   0x01b718    program   0x00048c
               .code_IP.o       code   0x01bba4    program   0x00029e
         .code_StackTsk.o       code   0x01be42    program   0x0001c4
                   STRING       code   0x01c006    program   0x0001bc
                     PROG       code   0x01c1c2    program   0x000128
             .code_Tick.o       code   0x01c2ea    program   0x0000ea
             .code_ICMP.o       code   0x01c3d4    program   0x0000d4
               _cinit_scn       code   0x01c4a8    program   0x00009e
         .code_fxd3232u.o       code   0x01c546    program   0x000048
           .romdata_TCP.o    romdata   0x01c58e    program   0x000036
.romdata_GenericTCPClient.o    romdata   0x01c5c4    program   0x000033
         .idata_c018i.o_i    romdata   0x01c5f7    program   0x000000
         .romdata_c018i.o    romdata   0x01c5f7    program   0x000000
        .romdata___init.o    romdata   0x01c5f7    program   0x000000
        .idata___init.o_i    romdata   0x01c5f7    program   0x000000
      .romdata_i2c1read.o    romdata   0x01c5f7    program   0x000000
      .idata_i2c1read.o_i    romdata   0x01c5f7    program   0x000000
      .romdata_fxd3232u.o    romdata   0x01c5f7    program   0x000000
      .idata_fxd3232u.o_i    romdata   0x01c5f7    program   0x000000
      .romdata_fxd1616u.o    romdata   0x01c5f7    program   0x000000
      .idata_fxd1616u.o_i    romdata   0x01c5f7    program   0x000000
      .romdata_fxd0808u.o    romdata   0x01c5f7    program   0x000000
      .idata_fxd0808u.o_i    romdata   0x01c5f7    program   0x000000
.romdata_GenericTCPServer.o    romdata   0x01c5f7    program   0x000000
           .romdata_UDP.o    romdata   0x01c5f7    program   0x000000
       .romdata_Helpers.o    romdata   0x01c5f7    program   0x000000
          .romdata_ICMP.o    romdata   0x01c5f7    program   0x000000
            .romdata_IP.o    romdata   0x01c5f7    program   0x000000
      .romdata_ETH97J60.o    romdata   0x01c5f7    program   0x000000
      .idata_StackTsk.o_i    romdata   0x01c5f7    program   0x000001
      .romdata_StackTsk.o    romdata   0x01c5f7    program   0x000000
           .romdata_DNS.o    romdata   0x01c5f7    program   0x000000
           .romdata_ARP.o    romdata   0x01c5f7    program   0x000000
          .romdata_Tick.o    romdata   0x01c5f7    program   0x000000
         .code_fxd1616u.o       code   0x01c5f8    program   0x00002c
                    .code       code   0x01c624    program   0x00002c
             _startup_scn       code   0x01c650    program   0x00001c
         .code_fxd0808u.o       code   0x01c66c    program   0x00001c
         .code_i2c1read.o       code   0x01c688    program   0x00001a
    .romdata_MainDemoV1.o    romdata   0x01c6a2    program   0x000006
           .idata_UDP.o_i    romdata   0x01c6a8    program   0x000002
          .idata_Tick.o_i    romdata   0x01c6aa    program   0x000004
           .idata_TCP.o_i    romdata   0x01c6ae    program   0x000002
    .idata_MainDemoV1.o_i    romdata   0x01c6b0    program   0x000015
            .idata_IP.o_i    romdata   0x01c6c5    program   0x000002
       .idata_Helpers.o_i    romdata   0x01c6c7    program   0x000004
          .idata_ICMP.o_i    romdata   0x01c6c7    program   0x000000
.idata_GenericTCPServer.o_i    romdata   0x01c6cb    program   0x000002
.idata_GenericTCPClient.o_i    romdata   0x01c6cd    program   0x000008
      .idata_ETH97J60.o_i    romdata   0x01c6d5    program   0x000000
           .idata_DNS.o_i    romdata   0x01c6d5    program   0x000003
           .idata_ARP.o_i    romdata   0x01c6d8    program   0x000001
            .code_c018i.o       code   0x01c6da    program   0x000000
.config_1fff8_MainDemoV1.o    romdata   0x01fff8    program   0x000001
.config_1fffa_MainDemoV1.o    romdata   0x01fffa    program   0x000001
.config_1fffd_MainDemoV1.o    romdata   0x01fffd    program   0x000001
                MATH_DATA      udata   0x000000       data   0x000014
                 .tmpdata      udata   0x000014       data   0x00000c
                   udata6      udata   0x000060       data   0x000087
.udata_GenericTCPServer.o      udata   0x0000e7       data   0x00000d
            .udata_Tick.o      udata   0x0000f4       data   0x00000a
             .idata_UDP.o      idata   0x0000fe       data   0x000002
                 TCB_uRAM      udata   0x000100       data   0x0000fc
            .udata_ICMP.o      udata   0x0001fc       data   0x000004
                   udata2      udata   0x000200       data   0x000200
             .udata_UDP.o      udata   0x000400       data   0x0000f6
           .udata_c018i.o      udata   0x0004f6       data   0x00000a
                   udata5      udata   0x000500       data   0x0000ea
              .udata_IP.o      udata   0x0005ea       data   0x000012
            .idata_Tick.o      idata   0x0005fc       data   0x000004
                  udata11      udata   0x000600       data   0x0000d5
             .udata_ARP.o      udata   0x0006d5       data   0x000027
         .idata_Helpers.o      idata   0x0006fc       data   0x000004
             .udata_TCP.o      udata   0x000700       data   0x0000cf
             .udata_DNS.o      udata   0x0007cf       data   0x000026
        .udata_StackTsk.o      udata   0x0007f5       data   0x00000b
                   udata8      udata   0x000800       data   0x0000b0
      .udata_MainDemoV1.o      udata   0x0008b0       data   0x000041
.udata_GenericTCPClient.o      udata   0x0008f1       data   0x00000e
        .idata_StackTsk.o      idata   0x0008ff       data   0x000001
                   udata1      udata   0x000900       data   0x000083
                  udata10      udata   0x000983       data   0x000068
      .idata_MainDemoV1.o      idata   0x0009eb       data   0x000015
         .udata_Helpers.o      udata   0x000a00       data   0x00003a
                   udata4      udata   0x000a3a       data   0x000038
        .udata_ETH97J60.o      udata   0x000a72       data   0x000036
  TCP.o:TCPAdjustFIFOSize     actrec   0x000b00       data   0x000006
      TCP.o:TCPRAMCopyROM     actrec   0x000b00       data   0x000012
MainDemoV1.o:choix_memoirePRECEDENT     actrec   0x000b00       data   0x000005
         TCP.o:TCPProcess     actrec   0x000b00       data   0x000025
       TCP.o:TCPPeekArray     actrec   0x000b00       data   0x000006
MainDemoV1.o:TRAMEENVOIRS485DONNEES     actrec   0x000b00       data   0x000002
     Tick.o:TickGetDiv64K     actrec   0x000b00       data   0x000004
   TCP.o:TCPGetRxFIFOFree     actrec   0x000b00       data   0x000004
MainDemoV1.o:calcul_addmemoirePRECEDENT     actrec   0x000b00       data   0x000006
        TCP.o:TCPGetArray     actrec   0x000b00       data   0x000004
             TCP.o:TCPGet     actrec   0x000b00       data   0x000002
      MainDemoV1.o:client     actrec   0x000b00       data   0x000003
   TCP.o:TCPGetTxFIFOFull     actrec   0x000b00       data   0x000004
        TCP.o:TCPPutArray     actrec   0x000b00       data   0x000006
             TCP.o:TCPPut     actrec   0x000b00       data   0x000002
  MainDemoV1.o:IntToChar5     actrec   0x000b00       data   0x00000c
MainDemoV1.o:CHERCHER_DONNNEES_CABLES     actrec   0x000b00       data   0x000009
MainDemoV1.o:enregistrer_donnees     actrec   0x000b00       data   0x000001
MainDemoV1.o:Recuperer_param_cms     actrec   0x000b00       data   0x000001
       MainDemoV1.o:TEMPO     actrec   0x000b00       data   0x000001
MainDemoV1.o:TRANSFORMER_TRAME_MEMOIRE_EN_TELGAT     actrec   0x000b00       data   0x000003
  MainDemoV1.o:Init_RS485     actrec   0x000b00       data   0x000002
       MainDemoV1.o:CRC16     actrec   0x000b00       data   0x000007
   MainDemoV1.o:IntToChar     actrec   0x000b00       data   0x00000c
 MainDemoV1.o:gestion_rob     actrec   0x000b00       data   0x000001
MainDemoV1.o:analyser_les_alarmes_en_cours     actrec   0x000b00       data   0x000005
MainDemoV1.o:creer_trame_horloge     actrec   0x000b00       data   0x000007
MainDemoV1.o:ECRIRE_EEPROMBYTE     actrec   0x000b00       data   0x000007
         UDP.o:UDPProcess     actrec   0x000b00       data   0x000019
        UDP.o:UDPGetArray     actrec   0x000b00       data   0x000002
MainDemoV1.o:RECEVOIR_RS485     actrec   0x000b00       data   0x000005
           UDP.o:UDPFlush     actrec   0x000b00       data   0x00001c
          UDP.o:UDPOpenEx     actrec   0x000b00       data   0x000003
            UDP.o:UDPInit     actrec   0x000b00       data   0x000001
MainDemoV1.o:TRANSFORMER_TRAME_MEM_EN_COM     actrec   0x000b00       data   0x000004
MainDemoV1.o:entrer_trame_horloge     actrec   0x000b00       data   0x000007
         ARP.o:ARPSendPkt     actrec   0x000b00       data   0x00001c
         ARP.o:ARPProcess     actrec   0x000b00       data   0x00001c
Helpers.o:leftRotateDWORD     actrec   0x000b00       data   0x000002
Helpers.o:FormatNetBIOSName     actrec   0x000b00       data   0x000001
 Helpers.o:stricmppgm2ram     actrec   0x000b00       data   0x000002
         ARP.o:ARPResolve     actrec   0x000b00       data   0x00001c
          Helpers.o:uitoa     actrec   0x000b00       data   0x000006
Helpers.o:ROMStringToIPAddress     actrec   0x000b00       data   0x000007
        Helpers.o:strnchr     actrec   0x000b00       data   0x000001
      Helpers.o:strncpy_m     actrec   0x000b00       data   0x000008
Helpers.o:StringToIPAddress     actrec   0x000b00       data   0x000007
       ICMP.o:ICMPProcess     actrec   0x000b00       data   0x000004
Helpers.o:GenerateRandomDWORD     actrec   0x000b00       data   0x000014
   ETH97J60.o:WritePHYReg     actrec   0x000b00       data   0x000001
         IP.o:IPGetHeader     actrec   0x000b00       data   0x000016
GenericTCPClient.o:delay_qms1     actrec   0x000b00       data   0x000003
       DNS.o:DNSPutString     actrec   0x000b00       data   0x000004
    DNS.o:DNSPutROMString     actrec   0x000b00       data   0x000005
GenericTCPClient.o:IntToChar1     actrec   0x000b00       data   0x00000c
  ETH97J60.o:MACGetHeader     actrec   0x000b00       data   0x000014
GenericTCPClient.o:CRC116     actrec   0x000b00       data   0x000006
       ETH97J60.o:MACInit     actrec   0x000b01       data   0x000001
MainDemoV1.o:INITGESTIONCARTEIO     actrec   0x000b02       data   0x000001
     DNS.o:DNSDiscardName     actrec   0x000b02       data   0x000001
            TCP.o:TCPOpen     actrec   0x000b03       data   0x000001
        UDP.o:UDPPutArray     actrec   0x000b04       data   0x000002
MainDemoV1.o:CHERCHER_DONNEES_GROUPE     actrec   0x000b05       data   0x000001
MainDemoV1.o:TRAMERECEPTIONRS485DONNEES     actrec   0x000b05       data   0x000002
     UDP.o:UDPPutROMArray     actrec   0x000b05       data   0x000002
   MainDemoV1.o:ProcessIO     actrec   0x000b06       data   0x000001
MainDemoV1.o:DisplayIPValue     actrec   0x000b06       data   0x000005
            TCP.o:TCPPeek     actrec   0x000b06       data   0x000001
      TCP.o:TCPIsPutReady     actrec   0x000b06       data   0x000001
MainDemoV1.o:GROUPE_EN_MEMOIRE     actrec   0x000b07       data   0x000002
MainDemoV1.o:ECRIRE_HORLOGE     actrec   0x000b07       data   0x000001
MainDemoV1.o:MODIFICATION_TABLE_DEXISTENCE     actrec   0x000b07       data   0x000005
MainDemoV1.o:SAV_EXISTENCE     actrec   0x000b07       data   0x000003
MainDemoV1.o:litHORLOGE_i2c     actrec   0x000b07       data   0x000001
MainDemoV1.o:LIRE_HORLOGE     actrec   0x000b08       data   0x000001
MainDemoV1.o:calcul_addmemoire     actrec   0x000b09       data   0x000006
MainDemoV1.o:choix_memoire     actrec   0x000b09       data   0x000005
 MainDemoV1.o:TYPEDECARTE     actrec   0x000b09       data   0x000001
MainDemoV1.o:putstringI2C     actrec   0x000b0c       data   0x000003
MainDemoV1.o:controle_CRC2021     actrec   0x000b0c       data   0x000007
MainDemoV1.o:ENVOYER_GROUPE     actrec   0x000b0c       data   0x000001
MainDemoV1.o:resume_voies     actrec   0x000b0c       data   0x000006
     TCP.o:TCPPutROMArray     actrec   0x000b12       data   0x000006
 MainDemoV1.o:LIRE_EEPROM     actrec   0x000b12       data   0x000006
 MainDemoV1.o:delay_qmsip     actrec   0x000b12       data   0x000003
    ETH97J60.o:ReadPHYReg     actrec   0x000b14       data   0x000002
            TCP.o:TCPInit     actrec   0x000b14       data   0x00000b
ETH97J60.o:MACCalcRxChecksum     actrec   0x000b16       data   0x000004
MainDemoV1.o:recuperer_trame_memoire     actrec   0x000b18       data   0x000004
 UDP.o:FindMatchingSocket     actrec   0x000b19       data   0x000004
            UDP.o:UDPTask     actrec   0x000b1c       data   0x000005
   Helpers.o:LFSRSeedRand     actrec   0x000b1f       data   0x000005
       Helpers.o:LFSRRand     actrec   0x000b25       data   0x000001
           Tick.o:TickGet     actrec   0x000b25       data   0x000004
TCP.o:GetMaxSegSizeOption     actrec   0x000b25       data   0x000004
 TCP.o:FindMatchingSocket     actrec   0x000b25       data   0x000006
ETH97J60.o:CalcIPBufferChecksum     actrec   0x000b25       data   0x00001e
ETH97J60.o:MACGetFreeRxSize     actrec   0x000b25       data   0x000004
         IP.o:IPPutHeader     actrec   0x000b25       data   0x000014
  ETH97J60.o:MACDiscardRx     actrec   0x000b25       data   0x000002
ETH97J60.o:MACSetReadPtrInRx     actrec   0x000b29       data   0x000002
      ETH97J60.o:MACFlush     actrec   0x000b29       data   0x000001
ETH97J60.o:MACSetWritePtr     actrec   0x000b2b       data   0x000002
 ETH97J60.o:MACSetReadPtr     actrec   0x000b2b       data   0x000002
ETH97J60.o:MACMemCopyAsync     actrec   0x000b2b       data   0x000006
     Tick.o:TickGetDiv256     actrec   0x000b2b       data   0x000004
 Helpers.o:CalcIPChecksum     actrec   0x000b39       data   0x000008
          Helpers.o:swaps     actrec   0x000b39       data   0x000003
       TCP.o:HandleTCPSeg     actrec   0x000b43       data   0x00001c
      DNS.o:DNSIsResolved     actrec   0x000b43       data   0x000019
     MainDemoV1.o:verifMP     actrec   0x000b5f       data   0x000004
    MainDemoV1.o:nom_site     actrec   0x000b5f       data   0x000003
MainDemoV1.o:ENVOIE_DES_TRAMES     actrec   0x000b5f       data   0x00000b
GenericTCPClient.o:GenericTCPClient     actrec   0x000b5f       data   0x00000e
        MainDemoV1.o:page     actrec   0x000b5f       data   0x000004
   MainDemoV1.o:MOUCHARD2     actrec   0x000b5f       data   0x000008
    MainDemoV1.o:MOUCHARD     actrec   0x000b5f       data   0x00000a
MainDemoV1.o:TRAMERECEPTIONminitel     actrec   0x000b5f       data   0x000002
MainDemoV1.o:gestion_menu3     actrec   0x000b61       data   0x000001
MainDemoV1.o:TRAMERECEPTIONTCPDONNEES     actrec   0x000b63       data   0x000002
GenericTCPServer.o:GenericTCPServer     actrec   0x000b6a       data   0x000003
MainDemoV1.o:voir_qui_existe     actrec   0x000b6d       data   0x00000d
MainDemoV1.o:MOUCHARDREGLAHEURE     actrec   0x000b6d       data   0x000001
MainDemoV1.o:gestion_menu1     actrec   0x000b6d       data   0x000001
MainDemoV1.o:gestion_menu8     actrec   0x000b6d       data   0x000001
MainDemoV1.o:gestion_menu6b     actrec   0x000b6d       data   0x000001
MainDemoV1.o:gestion_menu6a     actrec   0x000b6d       data   0x000002
MainDemoV1.o:VALIDER_CAPTEUR     actrec   0x000b6f       data   0x000002
MainDemoV1.o:EFFACER_CAPTEUR     actrec   0x000b6f       data   0x000002
 MainDemoV1.o:ecouteTCPIP     actrec   0x000b71       data   0x000001
            TCP.o:TCPTick     actrec   0x000b7a       data   0x00000a
     StackTsk.o:StackTask     actrec   0x000b84       data   0x000008
   ETH97J60.o:MACGetArray     actrec   0x000b8c       data   0x000003
      MainDemoV1.o:mainio     actrec   0x000b8f       data   0x000001
  TCP.o:TCPFindROMArrayEx     actrec   0x000c00       data   0x000031
     TCP.o:TCPFindArrayEx     actrec   0x000c00       data   0x000030
MainDemoV1.o:ANALYSE_SE_ALARME     actrec   0x000c00       data   0x0000d4
            TCP.o:SendTCP     actrec   0x000cd4       data   0x000028
                   .stack      udata   0x000d00       data   0x000100
                   udata9      udata   0x000e00       data   0x000063
.idata_GenericTCPClient.o      idata   0x000e63       data   0x000008
             .idata_DNS.o      idata   0x000e6b       data   0x000003
             .idata_TCP.o      idata   0x000e6e       data   0x000002
              .idata_IP.o      idata   0x000e70       data   0x000002
.idata_GenericTCPServer.o      idata   0x000e72       data   0x000002
             .idata_ARP.o      idata   0x000e74       data   0x000001
          .idata___init.o      idata   0x000e75       data   0x000000
          .udata___init.o      udata   0x000e75       data   0x000000
        .idata_i2c1read.o      idata   0x000e75       data   0x000000
        .udata_i2c1read.o      udata   0x000e75       data   0x000000
        .idata_fxd3232u.o      idata   0x000e75       data   0x000000
        .udata_fxd3232u.o      udata   0x000e75       data   0x000000
        .idata_fxd1616u.o      idata   0x000e75       data   0x000000
        .udata_fxd1616u.o      udata   0x000e75       data   0x000000
        .idata_fxd0808u.o      idata   0x000e75       data   0x000000
        .udata_fxd0808u.o      udata   0x000e75       data   0x000000
            .idata_ICMP.o      idata   0x000e75       data   0x000000
        .idata_ETH97J60.o      idata   0x000e75       data   0x000000
           .idata_c018i.o      idata   0x000e75       data   0x000000
              SFR_BANKED0      udata   0x000e80       data   0x000006
              SFR_BANKED1      udata   0x000e8a       data   0x000001
              SFR_BANKED2      udata   0x000e97       data   0x000003
              SFR_BANKED3      udata   0x000ea0       data   0x000001
              SFR_BANKED4      udata   0x000ea2       data   0x000003
              SFR_BANKED5      udata   0x000ea6       data   0x000002
              SFR_BANKED6      udata   0x000eaa       data   0x000002
              SFR_BANKED7      udata   0x000eb2       data   0x000001
              SFR_BANKED8      udata   0x000eb4       data   0x000001
              SFR_BANKED9      udata   0x000eb6       data   0x000004
             SFR_BANKED10      udata   0x000ec0       data   0x000012
             SFR_BANKED11      udata   0x000ed4       data   0x000002
             SFR_BANKED12      udata   0x000ed8       data   0x000002
             SFR_BANKED13      udata   0x000ee2       data   0x000016
             SFR_BANKED14      udata   0x000efb       data   0x000001
             SFR_BANKED15      udata   0x000efd       data   0x000002
       SYN_QUEUE_RAM_SECT      udata   0x000f00       data   0x00003c
            SFR_UNBANKED0      udata   0x000f60       data   0x0000a0



                              Program Memory Usage 
                               Start         End      
                           ---------   ---------      
                            0x000000    0x01c6d8      
                            0x01fff8    0x01fff8      
                            0x01fffa    0x01fffa      
                            0x01fffd    0x01fffd      
            116444 out of 131072 program addresses used, program memory utilization is 88%



                              Symbols - Sorted by Name
                     Name    Address   Location    Storage File                     
                ---------  ---------  ---------  --------- ---------                
        ANALYSE_SE_ALARME   0x01289a    program     extern C:\Users\LFRAD\Documents\CMS2Luc\ProjetsNettoyesCMSGit\ProjetCarteIO\project\MainDemoV1.c
                  ARPInit   0x01b86e    program     extern C:\Users\LFRAD\Documents\CMS2Luc\ProjetsNettoyesCMSGit\ProjetCarteIO\project\ARP.c
            ARPIsResolved   0x01ba5a    program     extern C:\Users\LFRAD\Documents\CMS2Luc\ProjetsNettoyesCMSGit\ProjetCarteIO\project\ARP.c
               ARPProcess   0x01b886    program     extern C:\Users\LFRAD\Documents\CMS2Luc\ProjetsNettoyesCMSGit\ProjetCarteIO\project\ARP.c
                   ARPPut   0x01b75e    program     static C:\Users\LFRAD\Documents\CMS2Luc\ProjetsNettoyesCMSGit\ProjetCarteIO\project\ARP.c
               ARPResolve   0x01b9d2    program     extern C:\Users\LFRAD\Documents\CMS2Luc\ProjetsNettoyesCMSGit\ProjetCarteIO\project\ARP.c
               ARPSendPkt   0x01b718    program     extern C:\Users\LFRAD\Documents\CMS2Luc\ProjetsNettoyesCMSGit\ProjetCarteIO\project\ARP.c
  CHERCHER_DONNEES_GROUPE   0x00c7ea    program     extern C:\Users\LFRAD\Documents\CMS2Luc\ProjetsNettoyesCMSGit\ProjetCarteIO\project\MainDemoV1.c
 CHERCHER_DONNNEES_CABLES   0x00b868    program     extern C:\Users\LFRAD\Documents\CMS2Luc\ProjetsNettoyesCMSGit\ProjetCarteIO\project\MainDemoV1.c
                   CRC116   0x019274    program     extern C:\Users\LFRAD\Documents\CMS2Luc\ProjetsNettoyesCMSGit\ProjetCarteIO\project\GenericTCPClient.c
                    CRC16   0x0019dc    program     extern C:\Users\LFRAD\Documents\CMS2Luc\ProjetsNettoyesCMSGit\ProjetCarteIO\project\MainDemoV1.c
CREER_TRAMEIN_CAPTEUR_DU_MINITEL   0x00f7a2    program     extern C:\Users\LFRAD\Documents\CMS2Luc\ProjetsNettoyesCMSGit\ProjetCarteIO\project\MainDemoV1.c
     CalcIPBufferChecksum   0x01ad88    program     extern C:\Users\LFRAD\Documents\CMS2Luc\ProjetsNettoyesCMSGit\ProjetCarteIO\project\ETH97J60.c
           CalcIPChecksum   0x019af0    program     extern C:\Users\LFRAD\Documents\CMS2Luc\ProjetsNettoyesCMSGit\ProjetCarteIO\project\Helpers.c
              CloseSocket   0x016298    program     static C:\Users\LFRAD\Documents\CMS2Luc\ProjetsNettoyesCMSGit\ProjetCarteIO\project\TCP.c
            DNSBeginUsage   0x019de2    program     extern C:\Users\LFRAD\Documents\CMS2Luc\ProjetsNettoyesCMSGit\ProjetCarteIO\project\DNS.c
           DNSDiscardName   0x01a7c0    program     static C:\Users\LFRAD\Documents\CMS2Luc\ProjetsNettoyesCMSGit\ProjetCarteIO\project\DNS.c
              DNSEndUsage   0x019df4    program     extern C:\Users\LFRAD\Documents\CMS2Luc\ProjetsNettoyesCMSGit\ProjetCarteIO\project\DNS.c
            DNSIsResolved   0x019ea0    program     extern C:\Users\LFRAD\Documents\CMS2Luc\ProjetsNettoyesCMSGit\ProjetCarteIO\project\DNS.c
          DNSPutROMString   0x01a6f0    program     static C:\Users\LFRAD\Documents\CMS2Luc\ProjetsNettoyesCMSGit\ProjetCarteIO\project\DNS.c
             DNSPutString   0x01a640    program     static C:\Users\LFRAD\Documents\CMS2Luc\ProjetsNettoyesCMSGit\ProjetCarteIO\project\DNS.c
               DNSResolve   0x019e1a    program     extern C:\Users\LFRAD\Documents\CMS2Luc\ProjetsNettoyesCMSGit\ProjetCarteIO\project\DNS.c
            DNSResolveROM   0x019e5a    program     extern C:\Users\LFRAD\Documents\CMS2Luc\ProjetsNettoyesCMSGit\ProjetCarteIO\project\DNS.c
           DisplayIPValue   0x000242    program     extern C:\Users\LFRAD\Documents\CMS2Luc\ProjetsNettoyesCMSGit\ProjetCarteIO\project\MainDemoV1.c
        ECRIRE_EEPROMBYTE   0x00dd96    program     extern C:\Users\LFRAD\Documents\CMS2Luc\ProjetsNettoyesCMSGit\ProjetCarteIO\project\MainDemoV1.c
           ECRIRE_HORLOGE   0x012410    program     extern C:\Users\LFRAD\Documents\CMS2Luc\ProjetsNettoyesCMSGit\ProjetCarteIO\project\MainDemoV1.c
          EFFACER_CAPTEUR   0x00f8fa    program     extern C:\Users\LFRAD\Documents\CMS2Luc\ProjetsNettoyesCMSGit\ProjetCarteIO\project\MainDemoV1.c
        ENVOIE_DES_TRAMES   0x00e22a    program     extern C:\Users\LFRAD\Documents\CMS2Luc\ProjetsNettoyesCMSGit\ProjetCarteIO\project\MainDemoV1.c
           ENVOYER_GROUPE   0x001ab0    program     extern C:\Users\LFRAD\Documents\CMS2Luc\ProjetsNettoyesCMSGit\ProjetCarteIO\project\MainDemoV1.c
                 FXD0808U   0x01c66c    program     extern E:\MPASM_MPLINK_PIC18_LT_Branch_3_42\pic18-lt\cxx-framework\src\traditional\math\fxd0808u.c
                 FXD1616U   0x01c5f8    program     extern E:\MPASM_MPLINK_PIC18_LT_Branch_3_42\pic18-lt\cxx-framework\src\traditional\math\fxd1616u.c
                 FXD3232U   0x01c546    program     extern E:\MPASM_MPLINK_PIC18_LT_Branch_3_42\pic18-lt\cxx-framework\src\traditional\math\fxd3232u.c
                 FXM1616S   0x01c1c2    program     extern E:\MPASM_MPLINK_PIC18_LT_Branch_3_42\pic18-lt\cxx-framework\src\traditional\math\fxm1616s.asm
                 FXM1616U   0x01c21c    program     extern E:\MPASM_MPLINK_PIC18_LT_Branch_3_42\pic18-lt\cxx-framework\src\traditional\math\fxm1616u.asm
                 FXM2424U   0x01c258    program     extern E:\MPASM_MPLINK_PIC18_LT_Branch_3_42\pic18-lt\cxx-framework\src\traditional\math\fxm2424u.asm
       FindMatchingSocket   0x015b8e    program     static C:\Users\LFRAD\Documents\CMS2Luc\ProjetsNettoyesCMSGit\ProjetCarteIO\project\TCP.c
       FindMatchingSocket   0x0185d4    program     static C:\Users\LFRAD\Documents\CMS2Luc\ProjetsNettoyesCMSGit\ProjetCarteIO\project\UDP.c
        FormatNetBIOSName   0x019c32    program     extern C:\Users\LFRAD\Documents\CMS2Luc\ProjetsNettoyesCMSGit\ProjetCarteIO\project\Helpers.c
        GROUPE_EN_MEMOIRE   0x0121e2    program     extern C:\Users\LFRAD\Documents\CMS2Luc\ProjetsNettoyesCMSGit\ProjetCarteIO\project\MainDemoV1.c
      GenerateRandomDWORD   0x019408    program     extern C:\Users\LFRAD\Documents\CMS2Luc\ProjetsNettoyesCMSGit\ProjetCarteIO\project\Helpers.c
         GenericTCPClient   0x01874c    program     extern C:\Users\LFRAD\Documents\CMS2Luc\ProjetsNettoyesCMSGit\ProjetCarteIO\project\GenericTCPClient.c
         GenericTCPServer   0x01b1ba    program     extern C:\Users\LFRAD\Documents\CMS2Luc\ProjetsNettoyesCMSGit\ProjetCarteIO\project\GenericTCPServer.c
      GetMaxSegSizeOption   0x016322    program     static C:\Users\LFRAD\Documents\CMS2Luc\ProjetsNettoyesCMSGit\ProjetCarteIO\project\TCP.c
              GetTickCopy   0x01c2fa    program     static C:\Users\LFRAD\Documents\CMS2Luc\ProjetsNettoyesCMSGit\ProjetCarteIO\project\Tick.c
             HandleTCPSeg   0x01642a    program     static C:\Users\LFRAD\Documents\CMS2Luc\ProjetsNettoyesCMSGit\ProjetCarteIO\project\TCP.c
                  HighISR   0x00015e    program     extern C:\Users\LFRAD\Documents\CMS2Luc\ProjetsNettoyesCMSGit\ProjetCarteIO\project\MainDemoV1.c
               HighVector   0x000008    program     extern C:\Users\LFRAD\Documents\CMS2Luc\ProjetsNettoyesCMSGit\ProjetCarteIO\project\MainDemoV1.c
           ICMPBeginUsage   0x012c52    program     extern C:\Users\LFRAD\Documents\CMS2Luc\ProjetsNettoyesCMSGit\ProjetCarteIO\project\MainDemoV1.c
              ICMPProcess   0x01c3d4    program     extern C:\Users\LFRAD\Documents\CMS2Luc\ProjetsNettoyesCMSGit\ProjetCarteIO\project\ICMP.c
       INITGESTIONCARTEIO   0x001fdc    program     extern C:\Users\LFRAD\Documents\CMS2Luc\ProjetsNettoyesCMSGit\ProjetCarteIO\project\MainDemoV1.c
              IPGetHeader   0x01bba4    program     extern C:\Users\LFRAD\Documents\CMS2Luc\ProjetsNettoyesCMSGit\ProjetCarteIO\project\IP.c
              IPPutHeader   0x01bc98    program     extern C:\Users\LFRAD\Documents\CMS2Luc\ProjetsNettoyesCMSGit\ProjetCarteIO\project\IP.c
            IPSetRxBuffer   0x01bd80    program     extern C:\Users\LFRAD\Documents\CMS2Luc\ProjetsNettoyesCMSGit\ProjetCarteIO\project\IP.c
            InitAppConfig   0x000300    program     static C:\Users\LFRAD\Documents\CMS2Luc\ProjetsNettoyesCMSGit\ProjetCarteIO\project\MainDemoV1.c
                 Init_I2C   0x00200c    program     extern C:\Users\LFRAD\Documents\CMS2Luc\ProjetsNettoyesCMSGit\ProjetCarteIO\project\MainDemoV1.c
               Init_RS485   0x00201e    program     extern C:\Users\LFRAD\Documents\CMS2Luc\ProjetsNettoyesCMSGit\ProjetCarteIO\project\MainDemoV1.c
          InitializeBoard   0x0002bc    program     static C:\Users\LFRAD\Documents\CMS2Luc\ProjetsNettoyesCMSGit\ProjetCarteIO\project\MainDemoV1.c
                IntToChar   0x00144c    program     extern C:\Users\LFRAD\Documents\CMS2Luc\ProjetsNettoyesCMSGit\ProjetCarteIO\project\MainDemoV1.c
               IntToChar1   0x018ce4    program     extern C:\Users\LFRAD\Documents\CMS2Luc\ProjetsNettoyesCMSGit\ProjetCarteIO\project\GenericTCPClient.c
               IntToChar5   0x012d56    program     extern C:\Users\LFRAD\Documents\CMS2Luc\ProjetsNettoyesCMSGit\ProjetCarteIO\project\MainDemoV1.c
                 LFSRRand   0x019382    program     extern C:\Users\LFRAD\Documents\CMS2Luc\ProjetsNettoyesCMSGit\ProjetCarteIO\project\Helpers.c
             LFSRSeedRand   0x019326    program     extern C:\Users\LFRAD\Documents\CMS2Luc\ProjetsNettoyesCMSGit\ProjetCarteIO\project\Helpers.c
              LIRE_EEPROM   0x001d4c    program     extern C:\Users\LFRAD\Documents\CMS2Luc\ProjetsNettoyesCMSGit\ProjetCarteIO\project\MainDemoV1.c
       LIRE_HEURE_MINITEL   0x00b190    program     extern C:\Users\LFRAD\Documents\CMS2Luc\ProjetsNettoyesCMSGit\ProjetCarteIO\project\MainDemoV1.c
             LIRE_HORLOGE   0x00faac    program     extern C:\Users\LFRAD\Documents\CMS2Luc\ProjetsNettoyesCMSGit\ProjetCarteIO\project\MainDemoV1.c
                   LowISR   0x0000a4    program     extern C:\Users\LFRAD\Documents\CMS2Luc\ProjetsNettoyesCMSGit\ProjetCarteIO\project\MainDemoV1.c
                LowVector   0x000018    program     extern C:\Users\LFRAD\Documents\CMS2Luc\ProjetsNettoyesCMSGit\ProjetCarteIO\project\MainDemoV1.c
        MACCalcRxChecksum   0x01ad0a    program     extern C:\Users\LFRAD\Documents\CMS2Luc\ProjetsNettoyesCMSGit\ProjetCarteIO\project\ETH97J60.c
             MACDiscardRx   0x01a95a    program     extern C:\Users\LFRAD\Documents\CMS2Luc\ProjetsNettoyesCMSGit\ProjetCarteIO\project\ETH97J60.c
                 MACFlush   0x01ac34    program     extern C:\Users\LFRAD\Documents\CMS2Luc\ProjetsNettoyesCMSGit\ProjetCarteIO\project\ETH97J60.c
                   MACGet   0x01b056    program     extern C:\Users\LFRAD\Documents\CMS2Luc\ProjetsNettoyesCMSGit\ProjetCarteIO\project\ETH97J60.c
              MACGetArray   0x01b05c    program     extern C:\Users\LFRAD\Documents\CMS2Luc\ProjetsNettoyesCMSGit\ProjetCarteIO\project\ETH97J60.c
         MACGetFreeRxSize   0x01a9c6    program     extern C:\Users\LFRAD\Documents\CMS2Luc\ProjetsNettoyesCMSGit\ProjetCarteIO\project\ETH97J60.c
             MACGetHeader   0x01aa66    program     extern C:\Users\LFRAD\Documents\CMS2Luc\ProjetsNettoyesCMSGit\ProjetCarteIO\project\ETH97J60.c
                  MACInit   0x01a80a    program     extern C:\Users\LFRAD\Documents\CMS2Luc\ProjetsNettoyesCMSGit\ProjetCarteIO\project\ETH97J60.c
              MACIsLinked   0x01a900    program     extern C:\Users\LFRAD\Documents\CMS2Luc\ProjetsNettoyesCMSGit\ProjetCarteIO\project\ETH97J60.c
         MACIsMemCopyDone   0x01b048    program     extern C:\Users\LFRAD\Documents\CMS2Luc\ProjetsNettoyesCMSGit\ProjetCarteIO\project\ETH97J60.c
             MACIsTxReady   0x01a920    program     extern C:\Users\LFRAD\Documents\CMS2Luc\ProjetsNettoyesCMSGit\ProjetCarteIO\project\ETH97J60.c
          MACMemCopyAsync   0x01aea0    program     extern C:\Users\LFRAD\Documents\CMS2Luc\ProjetsNettoyesCMSGit\ProjetCarteIO\project\ETH97J60.c
             MACPowerDown   0x01b19a    program     extern C:\Users\LFRAD\Documents\CMS2Luc\ProjetsNettoyesCMSGit\ProjetCarteIO\project\ETH97J60.c
               MACPowerUp   0x01b1ac    program     extern C:\Users\LFRAD\Documents\CMS2Luc\ProjetsNettoyesCMSGit\ProjetCarteIO\project\ETH97J60.c
                   MACPut   0x01b0c2    program     extern C:\Users\LFRAD\Documents\CMS2Luc\ProjetsNettoyesCMSGit\ProjetCarteIO\project\ETH97J60.c
              MACPutArray   0x01b0cc    program     extern C:\Users\LFRAD\Documents\CMS2Luc\ProjetsNettoyesCMSGit\ProjetCarteIO\project\ETH97J60.c
             MACPutHeader   0x01abd6    program     extern C:\Users\LFRAD\Documents\CMS2Luc\ProjetsNettoyesCMSGit\ProjetCarteIO\project\ETH97J60.c
           MACPutROMArray   0x01b0fe    program     extern C:\Users\LFRAD\Documents\CMS2Luc\ProjetsNettoyesCMSGit\ProjetCarteIO\project\ETH97J60.c
            MACSetReadPtr   0x01acee    program     extern C:\Users\LFRAD\Documents\CMS2Luc\ProjetsNettoyesCMSGit\ProjetCarteIO\project\ETH97J60.c
        MACSetReadPtrInRx   0x01ac80    program     extern C:\Users\LFRAD\Documents\CMS2Luc\ProjetsNettoyesCMSGit\ProjetCarteIO\project\ETH97J60.c
           MACSetWritePtr   0x01acd2    program     extern C:\Users\LFRAD\Documents\CMS2Luc\ProjetsNettoyesCMSGit\ProjetCarteIO\project\ETH97J60.c
MODIFICATION_TABLE_DEXISTENCE   0x00df2a    program     extern C:\Users\LFRAD\Documents\CMS2Luc\ProjetsNettoyesCMSGit\ProjetCarteIO\project\MainDemoV1.c
                 MOUCHARD   0x0088ee    program     extern C:\Users\LFRAD\Documents\CMS2Luc\ProjetsNettoyesCMSGit\ProjetCarteIO\project\MainDemoV1.c
                MOUCHARD2   0x0087b2    program     extern C:\Users\LFRAD\Documents\CMS2Luc\ProjetsNettoyesCMSGit\ProjetCarteIO\project\MainDemoV1.c
       MOUCHARDREGLAHEURE   0x008590    program     extern C:\Users\LFRAD\Documents\CMS2Luc\ProjetsNettoyesCMSGit\ProjetCarteIO\project\MainDemoV1.c
                ProcessIO   0x000294    program     static C:\Users\LFRAD\Documents\CMS2Luc\ProjetsNettoyesCMSGit\ProjetCarteIO\project\MainDemoV1.c
             RECEPTTCPACK   0x002cf2    program     extern C:\Users\LFRAD\Documents\CMS2Luc\ProjetsNettoyesCMSGit\ProjetCarteIO\project\MainDemoV1.c
           RECEVOIR_RS485   0x00fb2e    program     extern C:\Users\LFRAD\Documents\CMS2Luc\ProjetsNettoyesCMSGit\ProjetCarteIO\project\MainDemoV1.c
             RECEVOIR_TCP   0x00c1c6    program     extern C:\Users\LFRAD\Documents\CMS2Luc\ProjetsNettoyesCMSGit\ProjetCarteIO\project\MainDemoV1.c
     ROMStringToIPAddress   0x019702    program     extern C:\Users\LFRAD\Documents\CMS2Luc\ProjetsNettoyesCMSGit\ProjetCarteIO\project\Helpers.c
                    RS485   0x012484    program     extern C:\Users\LFRAD\Documents\CMS2Luc\ProjetsNettoyesCMSGit\ProjetCarteIO\project\MainDemoV1.c
                 ReadI2C1   0x01c688    program     extern E:\MPASM_MPLINK_PIC18_LT_Branch_3_42\pic18-lt\cxx-framework\src\pmc_common\i2c\i2c1read.c
               ReadPHYReg   0x01b13a    program     extern C:\Users\LFRAD\Documents\CMS2Luc\ProjetsNettoyesCMSGit\ProjetCarteIO\project\ETH97J60.c
      Recuperer_param_cms   0x00b204    program     extern C:\Users\LFRAD\Documents\CMS2Luc\ProjetsNettoyesCMSGit\ProjetCarteIO\project\MainDemoV1.c
                RemoteURL   0x01c5c4    program     static C:\Users\LFRAD\Documents\CMS2Luc\ProjetsNettoyesCMSGit\ProjetCarteIO\project\GenericTCPClient.c
           SAV_CHG_ALARME   0x012606    program     extern C:\Users\LFRAD\Documents\CMS2Luc\ProjetsNettoyesCMSGit\ProjetCarteIO\project\MainDemoV1.c
            SAV_EXISTENCE   0x012002    program     extern C:\Users\LFRAD\Documents\CMS2Luc\ProjetsNettoyesCMSGit\ProjetCarteIO\project\MainDemoV1.c
                  SendTCP   0x015602    program     static C:\Users\LFRAD\Documents\CMS2Luc\ProjetsNettoyesCMSGit\ProjetCarteIO\project\TCP.c
     SerializedMACAddress   0x01c6a2    program     static C:\Users\LFRAD\Documents\CMS2Luc\ProjetsNettoyesCMSGit\ProjetCarteIO\project\MainDemoV1.c
        StackApplications   0x01c004    program     extern C:\Users\LFRAD\Documents\CMS2Luc\ProjetsNettoyesCMSGit\ProjetCarteIO\project\StackTsk.c
                StackInit   0x01be42    program     extern C:\Users\LFRAD\Documents\CMS2Luc\ProjetsNettoyesCMSGit\ProjetCarteIO\project\StackTsk.c
                StackTask   0x01be7a    program     extern C:\Users\LFRAD\Documents\CMS2Luc\ProjetsNettoyesCMSGit\ProjetCarteIO\project\StackTsk.c
        StringToIPAddress   0x01954c    program     extern C:\Users\LFRAD\Documents\CMS2Luc\ProjetsNettoyesCMSGit\ProjetCarteIO\project\Helpers.c
            SwapARPPacket   0x01bb06    program     extern C:\Users\LFRAD\Documents\CMS2Luc\ProjetsNettoyesCMSGit\ProjetCarteIO\project\ARP.c
             SwapIPHeader   0x01bd98    program     static C:\Users\LFRAD\Documents\CMS2Luc\ProjetsNettoyesCMSGit\ProjetCarteIO\project\IP.c
            SwapTCPHeader   0x0160e2    program     static C:\Users\LFRAD\Documents\CMS2Luc\ProjetsNettoyesCMSGit\ProjetCarteIO\project\TCP.c
                  SyncTCB   0x013374    program     static C:\Users\LFRAD\Documents\CMS2Luc\ProjetsNettoyesCMSGit\ProjetCarteIO\project\TCP.c
              SyncTCBStub   0x0132e6    program     static C:\Users\LFRAD\Documents\CMS2Luc\ProjetsNettoyesCMSGit\ProjetCarteIO\project\TCP.c
        TCPAdjustFIFOSize   0x0173fc    program     extern C:\Users\LFRAD\Documents\CMS2Luc\ProjetsNettoyesCMSGit\ProjetCarteIO\project\TCP.c
                 TCPClose   0x0139b8    program     extern C:\Users\LFRAD\Documents\CMS2Luc\ProjetsNettoyesCMSGit\ProjetCarteIO\project\TCP.c
               TCPDiscard   0x01405e    program     extern C:\Users\LFRAD\Documents\CMS2Luc\ProjetsNettoyesCMSGit\ProjetCarteIO\project\TCP.c
            TCPDisconnect   0x0138dc    program     extern C:\Users\LFRAD\Documents\CMS2Luc\ProjetsNettoyesCMSGit\ProjetCarteIO\project\TCP.c
           TCPFindArrayEx   0x01451c    program     extern C:\Users\LFRAD\Documents\CMS2Luc\ProjetsNettoyesCMSGit\ProjetCarteIO\project\TCP.c
                TCPFindEx   0x014c5a    program     extern C:\Users\LFRAD\Documents\CMS2Luc\ProjetsNettoyesCMSGit\ProjetCarteIO\project\TCP.c
        TCPFindROMArrayEx   0x0148a0    program     extern C:\Users\LFRAD\Documents\CMS2Luc\ProjetsNettoyesCMSGit\ProjetCarteIO\project\TCP.c
                 TCPFlush   0x013a3c    program     extern C:\Users\LFRAD\Documents\CMS2Luc\ProjetsNettoyesCMSGit\ProjetCarteIO\project\TCP.c
                   TCPGet   0x014110    program     extern C:\Users\LFRAD\Documents\CMS2Luc\ProjetsNettoyesCMSGit\ProjetCarteIO\project\TCP.c
              TCPGetArray   0x0141bc    program     extern C:\Users\LFRAD\Documents\CMS2Luc\ProjetsNettoyesCMSGit\ProjetCarteIO\project\TCP.c
         TCPGetRemoteInfo   0x0139de    program     extern C:\Users\LFRAD\Documents\CMS2Luc\ProjetsNettoyesCMSGit\ProjetCarteIO\project\TCP.c
         TCPGetRxFIFOFree   0x014322    program     extern C:\Users\LFRAD\Documents\CMS2Luc\ProjetsNettoyesCMSGit\ProjetCarteIO\project\TCP.c
         TCPGetTxFIFOFull   0x013ffa    program     extern C:\Users\LFRAD\Documents\CMS2Luc\ProjetsNettoyesCMSGit\ProjetCarteIO\project\TCP.c
                  TCPInit   0x01341e    program     extern C:\Users\LFRAD\Documents\CMS2Luc\ProjetsNettoyesCMSGit\ProjetCarteIO\project\TCP.c
           TCPIsConnected   0x0138ae    program     extern C:\Users\LFRAD\Documents\CMS2Luc\ProjetsNettoyesCMSGit\ProjetCarteIO\project\TCP.c
            TCPIsGetReady   0x014094    program     extern C:\Users\LFRAD\Documents\CMS2Luc\ProjetsNettoyesCMSGit\ProjetCarteIO\project\TCP.c
            TCPIsPutReady   0x013a78    program     extern C:\Users\LFRAD\Documents\CMS2Luc\ProjetsNettoyesCMSGit\ProjetCarteIO\project\TCP.c
                  TCPOpen   0x0136d0    program     extern C:\Users\LFRAD\Documents\CMS2Luc\ProjetsNettoyesCMSGit\ProjetCarteIO\project\TCP.c
                  TCPPeek   0x0144f4    program     extern C:\Users\LFRAD\Documents\CMS2Luc\ProjetsNettoyesCMSGit\ProjetCarteIO\project\TCP.c
             TCPPeekArray   0x01437e    program     extern C:\Users\LFRAD\Documents\CMS2Luc\ProjetsNettoyesCMSGit\ProjetCarteIO\project\TCP.c
               TCPProcess   0x0154bc    program     extern C:\Users\LFRAD\Documents\CMS2Luc\ProjetsNettoyesCMSGit\ProjetCarteIO\project\TCP.c
                   TCPPut   0x013b0e    program     extern C:\Users\LFRAD\Documents\CMS2Luc\ProjetsNettoyesCMSGit\ProjetCarteIO\project\TCP.c
              TCPPutArray   0x013c0e    program     extern C:\Users\LFRAD\Documents\CMS2Luc\ProjetsNettoyesCMSGit\ProjetCarteIO\project\TCP.c
           TCPPutROMArray   0x013db2    program     extern C:\Users\LFRAD\Documents\CMS2Luc\ProjetsNettoyesCMSGit\ProjetCarteIO\project\TCP.c
          TCPPutROMString   0x013f9c    program     extern C:\Users\LFRAD\Documents\CMS2Luc\ProjetsNettoyesCMSGit\ProjetCarteIO\project\TCP.c
             TCPPutString   0x013f5c    program     extern C:\Users\LFRAD\Documents\CMS2Luc\ProjetsNettoyesCMSGit\ProjetCarteIO\project\TCP.c
               TCPRAMCopy   0x01766a    program     static C:\Users\LFRAD\Documents\CMS2Luc\ProjetsNettoyesCMSGit\ProjetCarteIO\project\TCP.c
            TCPRAMCopyROM   0x017732    program     static C:\Users\LFRAD\Documents\CMS2Luc\ProjetsNettoyesCMSGit\ProjetCarteIO\project\TCP.c
     TCPSocketInitializer   0x01c58e    program     extern C:\Users\LFRAD\Documents\CMS2Luc\ProjetsNettoyesCMSGit\ProjetCarteIO\project\h\Configs\TCPIPETH97.h
                  TCPTick   0x014c8a    program     extern C:\Users\LFRAD\Documents\CMS2Luc\ProjetsNettoyesCMSGit\ProjetCarteIO\project\TCP.c
              TCPWasReset   0x013880    program     extern C:\Users\LFRAD\Documents\CMS2Luc\ProjetsNettoyesCMSGit\ProjetCarteIO\project\TCP.c
                    TEMPO   0x008a8a    program     extern C:\Users\LFRAD\Documents\CMS2Luc\ProjetsNettoyesCMSGit\ProjetCarteIO\project\MainDemoV1.c
        TRAMECAPTEURBIDON   0x002b80    program     extern C:\Users\LFRAD\Documents\CMS2Luc\ProjetsNettoyesCMSGit\ProjetCarteIO\project\MainDemoV1.c
   TRAMEENVOIRS485DONNEES   0x0122f6    program     extern C:\Users\LFRAD\Documents\CMS2Luc\ProjetsNettoyesCMSGit\ProjetCarteIO\project\MainDemoV1.c
     TRAMEENVOITCPDONNEES   0x00b150    program     extern C:\Users\LFRAD\Documents\CMS2Luc\ProjetsNettoyesCMSGit\ProjetCarteIO\project\MainDemoV1.c
TRAMERECEPTIONRS485DONNEES   0x00e1b0    program     extern C:\Users\LFRAD\Documents\CMS2Luc\ProjetsNettoyesCMSGit\ProjetCarteIO\project\MainDemoV1.c
 TRAMERECEPTIONTCPDONNEES   0x00a996    program     extern C:\Users\LFRAD\Documents\CMS2Luc\ProjetsNettoyesCMSGit\ProjetCarteIO\project\MainDemoV1.c
    TRAMERECEPTIONminitel   0x009cae    program     extern C:\Users\LFRAD\Documents\CMS2Luc\ProjetsNettoyesCMSGit\ProjetCarteIO\project\MainDemoV1.c
TRANSFORMER_TRAME_MEMOIRE_EN_TELGAT   0x002d92    program     extern C:\Users\LFRAD\Documents\CMS2Luc\ProjetsNettoyesCMSGit\ProjetCarteIO\project\MainDemoV1.c
TRANSFORMER_TRAME_MEM_EN_COM   0x00fbc4    program     extern C:\Users\LFRAD\Documents\CMS2Luc\ProjetsNettoyesCMSGit\ProjetCarteIO\project\MainDemoV1.c
               TSIGN1616A   0x01c20e    program     static E:\MPASM_MPLINK_PIC18_LT_Branch_3_42\pic18-lt\cxx-framework\src\traditional\math\fxm1616s.asm
              TYPEDECARTE   0x00b7d4    program     extern C:\Users\LFRAD\Documents\CMS2Luc\ProjetsNettoyesCMSGit\ProjetCarteIO\project\MainDemoV1.c
TickConvertToMilliseconds   0x01c392    program     extern C:\Users\LFRAD\Documents\CMS2Luc\ProjetsNettoyesCMSGit\ProjetCarteIO\project\Tick.c
                  TickGet   0x01c320    program     extern C:\Users\LFRAD\Documents\CMS2Luc\ProjetsNettoyesCMSGit\ProjetCarteIO\project\Tick.c
            TickGetDiv256   0x01c346    program     extern C:\Users\LFRAD\Documents\CMS2Luc\ProjetsNettoyesCMSGit\ProjetCarteIO\project\Tick.c
            TickGetDiv64K   0x01c36c    program     extern C:\Users\LFRAD\Documents\CMS2Luc\ProjetsNettoyesCMSGit\ProjetCarteIO\project\Tick.c
                 TickInit   0x01c2ea    program     extern C:\Users\LFRAD\Documents\CMS2Luc\ProjetsNettoyesCMSGit\ProjetCarteIO\project\Tick.c
               TickUpdate   0x01c3c0    program     extern C:\Users\LFRAD\Documents\CMS2Luc\ProjetsNettoyesCMSGit\ProjetCarteIO\project\Tick.c
                 UDPClose   0x017e7a    program     extern C:\Users\LFRAD\Documents\CMS2Luc\ProjetsNettoyesCMSGit\ProjetCarteIO\project\UDP.c
               UDPDiscard   0x018460    program     extern C:\Users\LFRAD\Documents\CMS2Luc\ProjetsNettoyesCMSGit\ProjetCarteIO\project\UDP.c
                 UDPFlush   0x0181bc    program     extern C:\Users\LFRAD\Documents\CMS2Luc\ProjetsNettoyesCMSGit\ProjetCarteIO\project\UDP.c
                   UDPGet   0x0183b2    program     extern C:\Users\LFRAD\Documents\CMS2Luc\ProjetsNettoyesCMSGit\ProjetCarteIO\project\UDP.c
              UDPGetArray   0x0183e6    program     extern C:\Users\LFRAD\Documents\CMS2Luc\ProjetsNettoyesCMSGit\ProjetCarteIO\project\UDP.c
                  UDPInit   0x017812    program     extern C:\Users\LFRAD\Documents\CMS2Luc\ProjetsNettoyesCMSGit\ProjetCarteIO\project\UDP.c
            UDPIsGetReady   0x018374    program     extern C:\Users\LFRAD\Documents\CMS2Luc\ProjetsNettoyesCMSGit\ProjetCarteIO\project\UDP.c
              UDPIsOpened   0x017e4c    program     extern C:\Users\LFRAD\Documents\CMS2Luc\ProjetsNettoyesCMSGit\ProjetCarteIO\project\UDP.c
            UDPIsPutReady   0x017f52    program     extern C:\Users\LFRAD\Documents\CMS2Luc\ProjetsNettoyesCMSGit\ProjetCarteIO\project\UDP.c
                UDPOpenEx   0x01782e    program     extern C:\Users\LFRAD\Documents\CMS2Luc\ProjetsNettoyesCMSGit\ProjetCarteIO\project\UDP.c
               UDPProcess   0x01847a    program     extern C:\Users\LFRAD\Documents\CMS2Luc\ProjetsNettoyesCMSGit\ProjetCarteIO\project\UDP.c
                   UDPPut   0x017fbc    program     extern C:\Users\LFRAD\Documents\CMS2Luc\ProjetsNettoyesCMSGit\ProjetCarteIO\project\UDP.c
              UDPPutArray   0x018006    program     extern C:\Users\LFRAD\Documents\CMS2Luc\ProjetsNettoyesCMSGit\ProjetCarteIO\project\UDP.c
           UDPPutROMArray   0x018094    program     extern C:\Users\LFRAD\Documents\CMS2Luc\ProjetsNettoyesCMSGit\ProjetCarteIO\project\UDP.c
          UDPPutROMString   0x018162    program     extern C:\Users\LFRAD\Documents\CMS2Luc\ProjetsNettoyesCMSGit\ProjetCarteIO\project\UDP.c
             UDPPutString   0x018126    program     extern C:\Users\LFRAD\Documents\CMS2Luc\ProjetsNettoyesCMSGit\ProjetCarteIO\project\UDP.c
           UDPSetRxBuffer   0x017f30    program     extern C:\Users\LFRAD\Documents\CMS2Luc\ProjetsNettoyesCMSGit\ProjetCarteIO\project\UDP.c
           UDPSetTxBuffer   0x017ee2    program     extern C:\Users\LFRAD\Documents\CMS2Luc\ProjetsNettoyesCMSGit\ProjetCarteIO\project\UDP.c
                  UDPTask   0x017a54    program     extern C:\Users\LFRAD\Documents\CMS2Luc\ProjetsNettoyesCMSGit\ProjetCarteIO\project\UDP.c
          VALIDER_CAPTEUR   0x00d43e    program     extern C:\Users\LFRAD\Documents\CMS2Luc\ProjetsNettoyesCMSGit\ProjetCarteIO\project\MainDemoV1.c
                WriteI2CC   0x001f6a    program     extern C:\Users\LFRAD\Documents\CMS2Luc\ProjetsNettoyesCMSGit\ProjetCarteIO\project\MainDemoV1.c
              WritePHYReg   0x01b16a    program     extern C:\Users\LFRAD\Documents\CMS2Luc\ProjetsNettoyesCMSGit\ProjetCarteIO\project\ETH97J60.c
              _2jContinue   0x01c0c2    program     static E:\MPASM_MPLINK_PIC18_LT_Branch_3_42\pic18-lt\cxx-framework\src\traditional\stdclib\memset.asm
                   _2jEnd   0x01c126    program     static E:\MPASM_MPLINK_PIC18_LT_Branch_3_42\pic18-lt\cxx-framework\src\traditional\stdclib\slenpgm.asm
              _3jContinue   0x01c08e    program     static E:\MPASM_MPLINK_PIC18_LT_Branch_3_42\pic18-lt\cxx-framework\src\traditional\stdclib\mcpyp2r.asm
                   _3jEnd   0x01c0cc    program     static E:\MPASM_MPLINK_PIC18_LT_Branch_3_42\pic18-lt\cxx-framework\src\traditional\stdclib\memset.asm
              _4jContinue   0x01c03a    program     static E:\MPASM_MPLINK_PIC18_LT_Branch_3_42\pic18-lt\cxx-framework\src\traditional\stdclib\memcpy.asm
              _4jContinue   0x01c170    program     static E:\MPASM_MPLINK_PIC18_LT_Branch_3_42\pic18-lt\cxx-framework\src\traditional\stdclib\strncpy.asm
                   _4jEnd   0x01c098    program     static E:\MPASM_MPLINK_PIC18_LT_Branch_3_42\pic18-lt\cxx-framework\src\traditional\stdclib\mcpyp2r.asm
                   _5jEnd   0x01c17a    program     static E:\MPASM_MPLINK_PIC18_LT_Branch_3_42\pic18-lt\cxx-framework\src\traditional\stdclib\strncpy.asm
                   _5jEnd   0x01c044    program     static E:\MPASM_MPLINK_PIC18_LT_Branch_3_42\pic18-lt\cxx-framework\src\traditional\stdclib\memcpy.asm
           ___do_lbl00002   0x01c318    program     static                          
           ___do_lbl00003   0x01c31c    program     static                          
           ___do_lbl00004   0x01c2fa    program     static                          
         ___else_lbl00022   0x01aaa8    program     static                          
          ___for_lbl00101   0x019bfa    program     static                          
          ___for_lbl00102   0x019c02    program     static                          
          ___for_lbl00103   0x019bde    program     static                          
          ___for_lbl00104   0x019c18    program     static                          
          ___for_lbl00105   0x019c1e    program     static                          
          ___for_lbl00106   0x019c02    program     static                          
           ___if_lbl00014   0x0194b2    program     static                          
           ___if_lbl00015   0x0194c8    program     static                          
           ___if_lbl00016   0x01951a    program     static                          
           ___if_lbl00017   0x019522    program     static                          
           ___if_lbl00020   0x01aaa6    program     static                          
           ___if_lbl00021   0x01aab2    program     static                          
           ___if_lbl00023   0x01aac2    program     static                          
           ___if_lbl00024   0x01aac6    program     static                          
           ___if_lbl00025   0x01aad6    program     static                          
           ___if_lbl00031   0x01ab66    program     static                          
           ___if_lbl00034   0x01abcc    program     static                          
       ___return_lbl00000   0x01c58c    program     static                          
       ___return_lbl00000   0x01a8fe    program     static                          
       ___return_lbl00000   0x01c622    program     static                          
       ___return_lbl00000   0x01c686    program     static                          
       ___return_lbl00000   0x000004    program     static                          
       ___return_lbl00001   0x01c66a    program     static                          
       ___return_lbl00001   0x01c31e    program     static                          
       ___return_lbl00002   0x01c544    program     static                          
       ___return_lbl00002   0x00001c    program     static                          
       ___return_lbl00003   0x00000c    program     static                          
       ___return_lbl00009   0x01954a    program     static                          
       ___return_lbl00019   0x01abd4    program     static                          
       ___return_lbl00087   0x01b0ca    program     static                          
       ___return_lbl00088   0x01b0fc    program     static                          
       ___return_lbl00091   0x01b138    program     static                          
       ___return_lbl00094   0x01b168    program     static                          
       ___return_lbl00097   0x01b198    program     static                          
       ___return_lbl00100   0x019c30    program     static                          
        ___while_lbl00001   0x01a816    program     static                          
        ___while_lbl00002   0x01a81c    program     static                          
        ___while_lbl00010   0x01944c    program     static                          
        ___while_lbl00011   0x019524    program     static                          
        ___while_lbl00012   0x019454    program     static                          
        ___while_lbl00013   0x019458    program     static                          
        ___while_lbl00089   0x01b0cc    program     static                          
        ___while_lbl00090   0x01b0fc    program     static                          
        ___while_lbl00092   0x01b0fe    program     static                          
        ___while_lbl00093   0x01b138    program     static                          
        ___while_lbl00095   0x01b148    program     static                          
        ___while_lbl00096   0x01b14e    program     static                          
        ___while_lbl00098   0x01b192    program     static                          
        ___while_lbl00099   0x01b198    program     static                          
               __config_0   0x01fff8    program     static C:\Users\LFRAD\Documents\CMS2Luc\ProjetsNettoyesCMSGit\ProjetCarteIO\project\MainDemoV1.c
               __config_1   0x01fffa    program     static C:\Users\LFRAD\Documents\CMS2Luc\ProjetsNettoyesCMSGit\ProjetCarteIO\project\MainDemoV1.c
               __config_2   0x01fffd    program     static C:\Users\LFRAD\Documents\CMS2Luc\ProjetsNettoyesCMSGit\ProjetCarteIO\project\MainDemoV1.c
                   __init   0x000006    program     extern E:\MPASM_MPLINK_PIC18_LT_Branch_3_42\pic18-lt\cxx-framework\src\traditional\stdclib\__init.c
               __string_0   0x00000e    program     static C:\Users\LFRAD\Documents\CMS2Luc\ProjetsNettoyesCMSGit\ProjetCarteIO\project\MainDemoV1.c
               __tmplbl_0   0x019492    program     static                          
              __tmplbl_10   0x01ab2e    program     static                          
              __tmplbl_11   0x01ab2c    program     static                          
              __tmplbl_12   0x01abc0    program     static                          
              __tmplbl_13   0x01abb2    program     static                          
             __tmplbl_138   0x0173fa    program     static                          
              __tmplbl_14   0x01abb8    program     static                          
             __tmplbl_140   0x0173fa    program     static                          
             __tmplbl_142   0x0173fa    program     static                          
             __tmplbl_144   0x0173fa    program     static                          
             __tmplbl_146   0x0173fa    program     static                          
             __tmplbl_149   0x0173fa    program     static                          
             __tmplbl_157   0x0173fa    program     static                          
             __tmplbl_158   0x0173fa    program     static                          
             __tmplbl_160   0x0173fa    program     static                          
             __tmplbl_162   0x0173fa    program     static                          
             __tmplbl_163   0x0173fa    program     static                          
               __tmplbl_5   0x01ab64    program     static                          
               __tmplbl_6   0x01ab5a    program     static                          
               __tmplbl_7   0x01ab4c    program     static                          
             __tmplbl_728   0x0013ec    program     static                          
             __tmplbl_743   0x000af6    program     static                          
             __tmplbl_751   0x002b76    program     static                          
             __tmplbl_752   0x002b5a    program     static                          
             __tmplbl_758   0x002062    program     static                          
             __tmplbl_764   0x00800c    program     static                          
             __tmplbl_766   0x00800c    program     static                          
             __tmplbl_767   0x004542    program     static                          
             __tmplbl_776   0x00800c    program     static                          
             __tmplbl_782   0x00800c    program     static                          
             __tmplbl_783   0x005522    program     static                          
             __tmplbl_788   0x00800c    program     static                          
             __tmplbl_789   0x005d84    program     static                          
             __tmplbl_794   0x00800c    program     static                          
             __tmplbl_799   0x00800c    program     static                          
               __tmplbl_8   0x01ab42    program     static                          
             __tmplbl_800   0x006f44    program     static                          
             __tmplbl_808   0x00800c    program     static                          
             __tmplbl_814   0x00800c    program     static                          
             __tmplbl_815   0x00800c    program     static                          
             __tmplbl_876   0x00f692    program     static                          
             __tmplbl_877   0x00f588    program     static                          
             __tmplbl_878   0x00f1f2    program     static                          
             __tmplbl_879   0x00f034    program     static                          
             __tmplbl_880   0x00ee46    program     static                          
             __tmplbl_881   0x00ec94    program     static                          
             __tmplbl_884   0x00f7a0    program     static                          
             __tmplbl_885   0x00f7a0    program     static                          
             __tmplbl_887   0x00f7a0    program     static                          
             __tmplbl_892   0x00f7a0    program     static                          
             __tmplbl_896   0x00f7a0    program     static                          
             __tmplbl_899   0x00f7a0    program     static                          
               __tmplbl_9   0x01ab38    program     static                          
             __tmplbl_900   0x00f7a0    program     static                          
             __tmplbl_901   0x00f7a0    program     static                          
            __zero_memory   0x01c624    program     extern E:\MPASM_MPLINK_PIC18_LT_Branch_3_42\pic18-lt\cxx-framework\src\traditional\proc\p18f97j60.asm
                _do_cinit   0x01c4a8    program     extern E:\MPASM_MPLINK_PIC18_LT_Branch_3_42\pic18-lt\cxx-framework\src\traditional\startup\c018i.c
                   _entry   0x000000    program     extern E:\MPASM_MPLINK_PIC18_LT_Branch_3_42\pic18-lt\cxx-framework\src\traditional\startup\c018i.c
                   _false   0x01c588    program     static                          
                 _startup   0x01c650    program     extern E:\MPASM_MPLINK_PIC18_LT_Branch_3_42\pic18-lt\cxx-framework\src\traditional\startup\c018i.c
analyser_les_alarmes_en_cours   0x00cfb2    program     extern C:\Users\LFRAD\Documents\CMS2Luc\ProjetsNettoyesCMSGit\ProjetCarteIO\project\MainDemoV1.c
             btohexa_high   0x0199c0    program     extern C:\Users\LFRAD\Documents\CMS2Luc\ProjetsNettoyesCMSGit\ProjetCarteIO\project\Helpers.c
              btohexa_low   0x0199de    program     extern C:\Users\LFRAD\Documents\CMS2Luc\ProjetsNettoyesCMSGit\ProjetCarteIO\project\Helpers.c
               calcul_CRC   0x012338    program     extern C:\Users\LFRAD\Documents\CMS2Luc\ProjetsNettoyesCMSGit\ProjetCarteIO\project\MainDemoV1.c
        calcul_addmemoire   0x002fd8    program     extern C:\Users\LFRAD\Documents\CMS2Luc\ProjetsNettoyesCMSGit\ProjetCarteIO\project\MainDemoV1.c
calcul_addmemoirePRECEDENT   0x0126fc    program     extern C:\Users\LFRAD\Documents\CMS2Luc\ProjetsNettoyesCMSGit\ProjetCarteIO\project\MainDemoV1.c
               calcul_c_l   0x00be5c    program     extern C:\Users\LFRAD\Documents\CMS2Luc\ProjetsNettoyesCMSGit\ProjetCarteIO\project\MainDemoV1.c
            choix_memoire   0x0031ea    program     extern C:\Users\LFRAD\Documents\CMS2Luc\ProjetsNettoyesCMSGit\ProjetCarteIO\project\MainDemoV1.c
   choix_memoirePRECEDENT   0x01263e    program     extern C:\Users\LFRAD\Documents\CMS2Luc\ProjetsNettoyesCMSGit\ProjetCarteIO\project\MainDemoV1.c
                   client   0x012b66    program     extern C:\Users\LFRAD\Documents\CMS2Luc\ProjetsNettoyesCMSGit\ProjetCarteIO\project\MainDemoV1.c
                compare_l   0x01c646    program     static E:\MPASM_MPLINK_PIC18_LT_Branch_3_42\pic18-lt\cxx-framework\src\traditional\proc\p18f97j60.asm
             controle_CRC   0x012282    program     extern C:\Users\LFRAD\Documents\CMS2Luc\ProjetsNettoyesCMSGit\ProjetCarteIO\project\MainDemoV1.c
         controle_CRC2021   0x012c64    program     extern C:\Users\LFRAD\Documents\CMS2Luc\ProjetsNettoyesCMSGit\ProjetCarteIO\project\MainDemoV1.c
                copy_loop   0x01c51a    program     static                          
            copy_one_byte   0x01c520    program     static                          
      creer_trame_horloge   0x00d9d6    program     extern C:\Users\LFRAD\Documents\CMS2Luc\ProjetsNettoyesCMSGit\ProjetCarteIO\project\MainDemoV1.c
                delay_qms   0x001a74    program     extern C:\Users\LFRAD\Documents\CMS2Luc\ProjetsNettoyesCMSGit\ProjetCarteIO\project\MainDemoV1.c
               delay_qms1   0x0192f8    program     extern C:\Users\LFRAD\Documents\CMS2Luc\ProjetsNettoyesCMSGit\ProjetCarteIO\project\GenericTCPClient.c
              delay_qmsip   0x001a82    program     extern C:\Users\LFRAD\Documents\CMS2Luc\ProjetsNettoyesCMSGit\ProjetCarteIO\project\MainDemoV1.c
                     done   0x01c544    program     static                          
             done_copying   0x01c52e    program     static                          
                   droite   0x00c058    program     extern C:\Users\LFRAD\Documents\CMS2Luc\ProjetsNettoyesCMSGit\ProjetCarteIO\project\MainDemoV1.c
                  echange   0x0013ee    program     extern C:\Users\LFRAD\Documents\CMS2Luc\ProjetsNettoyesCMSGit\ProjetCarteIO\project\MainDemoV1.c
              ecouteTCPIP   0x012570    program     extern C:\Users\LFRAD\Documents\CMS2Luc\ProjetsNettoyesCMSGit\ProjetCarteIO\project\MainDemoV1.c
                  endloop   0x01c682    program     static                          
                  endloop   0x01c61e    program     static                          
      enregistrer_donnees   0x00b3d2    program     extern C:\Users\LFRAD\Documents\CMS2Luc\ProjetsNettoyesCMSGit\ProjetCarteIO\project\MainDemoV1.c
     entrer_trame_horloge   0x012116    program     extern C:\Users\LFRAD\Documents\CMS2Luc\ProjetsNettoyesCMSGit\ProjetCarteIO\project\MainDemoV1.c
             envoi_cursur   0x0096a4    program     extern C:\Users\LFRAD\Documents\CMS2Luc\ProjetsNettoyesCMSGit\ProjetCarteIO\project\MainDemoV1.c
       envoyerHORLOGE_i2c   0x01249c    program     extern C:\Users\LFRAD\Documents\CMS2Luc\ProjetsNettoyesCMSGit\ProjetCarteIO\project\MainDemoV1.c
                   gauche   0x00bfb0    program     extern C:\Users\LFRAD\Documents\CMS2Luc\ProjetsNettoyesCMSGit\ProjetCarteIO\project\MainDemoV1.c
            gestion_menu1   0x00a8f0    program     extern C:\Users\LFRAD\Documents\CMS2Luc\ProjetsNettoyesCMSGit\ProjetCarteIO\project\MainDemoV1.c
            gestion_menu2   0x00a564    program     extern C:\Users\LFRAD\Documents\CMS2Luc\ProjetsNettoyesCMSGit\ProjetCarteIO\project\MainDemoV1.c
            gestion_menu3   0x00a12e    program     extern C:\Users\LFRAD\Documents\CMS2Luc\ProjetsNettoyesCMSGit\ProjetCarteIO\project\MainDemoV1.c
            gestion_menu5   0x009f0a    program     extern C:\Users\LFRAD\Documents\CMS2Luc\ProjetsNettoyesCMSGit\ProjetCarteIO\project\MainDemoV1.c
            gestion_menu6   0x009d7a    program     extern C:\Users\LFRAD\Documents\CMS2Luc\ProjetsNettoyesCMSGit\ProjetCarteIO\project\MainDemoV1.c
           gestion_menu6a   0x009230    program     extern C:\Users\LFRAD\Documents\CMS2Luc\ProjetsNettoyesCMSGit\ProjetCarteIO\project\MainDemoV1.c
           gestion_menu6b   0x008d7a    program     extern C:\Users\LFRAD\Documents\CMS2Luc\ProjetsNettoyesCMSGit\ProjetCarteIO\project\MainDemoV1.c
            gestion_menu8   0x008b04    program     extern C:\Users\LFRAD\Documents\CMS2Luc\ProjetsNettoyesCMSGit\ProjetCarteIO\project\MainDemoV1.c
             gestion_page   0x00acbc    program     extern C:\Users\LFRAD\Documents\CMS2Luc\ProjetsNettoyesCMSGit\ProjetCarteIO\project\MainDemoV1.c
              gestion_rob   0x00bf7c    program     extern C:\Users\LFRAD\Documents\CMS2Luc\ProjetsNettoyesCMSGit\ProjetCarteIO\project\MainDemoV1.c
                 getsI2CC   0x001f12    program     extern C:\Users\LFRAD\Documents\CMS2Luc\ProjetsNettoyesCMSGit\ProjetCarteIO\project\MainDemoV1.c
                     haut   0x00d422    program     extern C:\Users\LFRAD\Documents\CMS2Luc\ProjetsNettoyesCMSGit\ProjetCarteIO\project\MainDemoV1.c
                  hexatob   0x019980    program     extern C:\Users\LFRAD\Documents\CMS2Luc\ProjetsNettoyesCMSGit\ProjetCarteIO\project\Helpers.c
              infos_etats   0x00db1a    program     extern C:\Users\LFRAD\Documents\CMS2Luc\ProjetsNettoyesCMSGit\ProjetCarteIO\project\MainDemoV1.c
                     jEnd   0x01c0d4    program     static E:\MPASM_MPLINK_PIC18_LT_Branch_3_42\pic18-lt\cxx-framework\src\traditional\stdclib\memset.asm
                     jEnd   0x01c0a0    program     static E:\MPASM_MPLINK_PIC18_LT_Branch_3_42\pic18-lt\cxx-framework\src\traditional\stdclib\mcpyp2r.asm
                     jEnd   0x01c0f0    program     static E:\MPASM_MPLINK_PIC18_LT_Branch_3_42\pic18-lt\cxx-framework\src\traditional\stdclib\strlen.asm
                     jEnd   0x01c04a    program     static E:\MPASM_MPLINK_PIC18_LT_Branch_3_42\pic18-lt\cxx-framework\src\traditional\stdclib\memcpy.asm
                     jEnd   0x01c128    program     static E:\MPASM_MPLINK_PIC18_LT_Branch_3_42\pic18-lt\cxx-framework\src\traditional\stdclib\slenpgm.asm
                     jEnd   0x01c1c0    program     static E:\MPASM_MPLINK_PIC18_LT_Branch_3_42\pic18-lt\cxx-framework\src\traditional\stdclib\strupr.asm
                     jEnd   0x01c186    program     static E:\MPASM_MPLINK_PIC18_LT_Branch_3_42\pic18-lt\cxx-framework\src\traditional\stdclib\strncpy.asm
                    jLoop   0x01c1ac    program     static E:\MPASM_MPLINK_PIC18_LT_Branch_3_42\pic18-lt\cxx-framework\src\traditional\stdclib\strupr.asm
                    jLoop   0x01c164    program     static E:\MPASM_MPLINK_PIC18_LT_Branch_3_42\pic18-lt\cxx-framework\src\traditional\stdclib\strncpy.asm
                    jLoop   0x01c110    program     static E:\MPASM_MPLINK_PIC18_LT_Branch_3_42\pic18-lt\cxx-framework\src\traditional\stdclib\slenpgm.asm
                    jLoop   0x01c0e6    program     static E:\MPASM_MPLINK_PIC18_LT_Branch_3_42\pic18-lt\cxx-framework\src\traditional\stdclib\strlen.asm
                    jLoop   0x01c0b6    program     static E:\MPASM_MPLINK_PIC18_LT_Branch_3_42\pic18-lt\cxx-framework\src\traditional\stdclib\memset.asm
                    jLoop   0x01c082    program     static E:\MPASM_MPLINK_PIC18_LT_Branch_3_42\pic18-lt\cxx-framework\src\traditional\stdclib\mcpyp2r.asm
                    jLoop   0x01c02e    program     static E:\MPASM_MPLINK_PIC18_LT_Branch_3_42\pic18-lt\cxx-framework\src\traditional\stdclib\memcpy.asm
                    jSkip   0x01c1bc    program     static E:\MPASM_MPLINK_PIC18_LT_Branch_3_42\pic18-lt\cxx-framework\src\traditional\stdclib\strupr.asm
          leftRotateDWORD   0x019bca    program     extern C:\Users\LFRAD\Documents\CMS2Luc\ProjetsNettoyesCMSGit\ProjetCarteIO\project\Helpers.c
           litHORLOGE_i2c   0x0123d0    program     extern C:\Users\LFRAD\Documents\CMS2Luc\ProjetsNettoyesCMSGit\ProjetCarteIO\project\MainDemoV1.c
                     loop   0x01c660    program     static                          
                     loop   0x01c674    program     static                          
                     loop   0x01c602    program     static                          
                     loop   0x01c554    program     static                          
                   loop_h   0x01c63e    program     static E:\MPASM_MPLINK_PIC18_LT_Branch_3_42\pic18-lt\cxx-framework\src\traditional\proc\p18f97j60.asm
                   loop_l   0x01c648    program     static E:\MPASM_MPLINK_PIC18_LT_Branch_3_42\pic18-lt\cxx-framework\src\traditional\proc\p18f97j60.asm
                     main   0x000184    program     extern C:\Users\LFRAD\Documents\CMS2Luc\ProjetsNettoyesCMSGit\ProjetCarteIO\project\MainDemoV1.c
                   mainio   0x00083a    program     extern C:\Users\LFRAD\Documents\CMS2Luc\ProjetsNettoyesCMSGit\ProjetCarteIO\project\MainDemoV1.c
                   memcpy   0x01c006    program     extern E:\MPASM_MPLINK_PIC18_LT_Branch_3_42\pic18-lt\cxx-framework\src\traditional\stdclib\memcpy.asm
            memcpypgm2ram   0x01c05c    program     extern E:\MPASM_MPLINK_PIC18_LT_Branch_3_42\pic18-lt\cxx-framework\src\traditional\stdclib\mcpyp2r.asm
                   memset   0x01c0a2    program     extern E:\MPASM_MPLINK_PIC18_LT_Branch_3_42\pic18-lt\cxx-framework\src\traditional\stdclib\memset.asm
                  minitel   0x00800e    program     extern C:\Users\LFRAD\Documents\CMS2Luc\ProjetsNettoyesCMSGit\ProjetCarteIO\project\MainDemoV1.c
                 nom_site   0x00ab12    program     extern C:\Users\LFRAD\Documents\CMS2Luc\ProjetsNettoyesCMSGit\ProjetCarteIO\project\MainDemoV1.c
                     page   0x0032c8    program     extern C:\Users\LFRAD\Documents\CMS2Luc\ProjetsNettoyesCMSGit\ProjetCarteIO\project\MainDemoV1.c
            position_init   0x0096d2    program     extern C:\Users\LFRAD\Documents\CMS2Luc\ProjetsNettoyesCMSGit\ProjetCarteIO\project\MainDemoV1.c
             putstringI2C   0x0124ca    program     extern C:\Users\LFRAD\Documents\CMS2Luc\ProjetsNettoyesCMSGit\ProjetCarteIO\project\MainDemoV1.c
  recuperer_trame_memoire   0x010ee8    program     extern C:\Users\LFRAD\Documents\CMS2Luc\ProjetsNettoyesCMSGit\ProjetCarteIO\project\MainDemoV1.c
             resume_voies   0x00c23c    program     extern C:\Users\LFRAD\Documents\CMS2Luc\ProjetsNettoyesCMSGit\ProjetCarteIO\project\MainDemoV1.c
                   saisie   0x00c140    program     extern C:\Users\LFRAD\Documents\CMS2Luc\ProjetsNettoyesCMSGit\ProjetCarteIO\project\MainDemoV1.c
           stricmppgm2ram   0x0199fa    program     extern C:\Users\LFRAD\Documents\CMS2Luc\ProjetsNettoyesCMSGit\ProjetCarteIO\project\Helpers.c
                   strlen   0x01c0d6    program     extern E:\MPASM_MPLINK_PIC18_LT_Branch_3_42\pic18-lt\cxx-framework\src\traditional\stdclib\strlen.asm
                strlenpgm   0x01c0f2    program     extern E:\MPASM_MPLINK_PIC18_LT_Branch_3_42\pic18-lt\cxx-framework\src\traditional\stdclib\slenpgm.asm
                  strnchr   0x019c96    program     extern C:\Users\LFRAD\Documents\CMS2Luc\ProjetsNettoyesCMSGit\ProjetCarteIO\project\Helpers.c
                  strncpy   0x01c13c    program     extern E:\MPASM_MPLINK_PIC18_LT_Branch_3_42\pic18-lt\cxx-framework\src\traditional\stdclib\strncpy.asm
                strncpy_m   0x019cf0    program     extern C:\Users\LFRAD\Documents\CMS2Luc\ProjetsNettoyesCMSGit\ProjetCarteIO\project\Helpers.c
                   strupr   0x01c198    program     extern E:\MPASM_MPLINK_PIC18_LT_Branch_3_42\pic18-lt\cxx-framework\src\traditional\stdclib\strupr.asm
              sup_capteur   0x00d6c8    program     extern C:\Users\LFRAD\Documents\CMS2Luc\ProjetsNettoyesCMSGit\ProjetCarteIO\project\MainDemoV1.c
                    swapl   0x019ac2    program     extern C:\Users\LFRAD\Documents\CMS2Luc\ProjetsNettoyesCMSGit\ProjetCarteIO\project\Helpers.c
                    swaps   0x019aa2    program     extern C:\Users\LFRAD\Documents\CMS2Luc\ProjetsNettoyesCMSGit\ProjetCarteIO\project\Helpers.c
               tabulation   0x00bf92    program     extern C:\Users\LFRAD\Documents\CMS2Luc\ProjetsNettoyesCMSGit\ProjetCarteIO\project\MainDemoV1.c
                     test   0x01c4c2    program     static                          
                 testINT2   0x012550    program     extern C:\Users\LFRAD\Documents\CMS2Luc\ProjetsNettoyesCMSGit\ProjetCarteIO\project\MainDemoV1.c
                    uitoa   0x0198ba    program     extern C:\Users\LFRAD\Documents\CMS2Luc\ProjetsNettoyesCMSGit\ProjetCarteIO\project\Helpers.c
         variables_groupe   0x00c590    program     extern C:\Users\LFRAD\Documents\CMS2Luc\ProjetsNettoyesCMSGit\ProjetCarteIO\project\MainDemoV1.c
                  verifMP   0x00aa18    program     extern C:\Users\LFRAD\Documents\CMS2Luc\ProjetsNettoyesCMSGit\ProjetCarteIO\project\MainDemoV1.c
          voir_qui_existe   0x002056    program     extern C:\Users\LFRAD\Documents\CMS2Luc\ProjetsNettoyesCMSGit\ProjetCarteIO\project\MainDemoV1.c
               zero_block   0x01c63e    program     static E:\MPASM_MPLINK_PIC18_LT_Branch_3_42\pic18-lt\cxx-framework\src\traditional\proc\p18f97j60.asm
                       AA   0x000930       data     extern C:\Users\LFRAD\Documents\CMS2Luc\ProjetsNettoyesCMSGit\ProjetCarteIO\project\MainDemoV1.c
            ACTIONENCOURS   0x000900       data     extern C:\Users\LFRAD\Documents\CMS2Luc\ProjetsNettoyesCMSGit\ProjetCarteIO\project\MainDemoV1.c
                   ADCON0   0x000fc2       data     extern E:\MPASM_MPLINK_PIC18_LT_Branch_3_42\pic18-lt\cxx-framework\src\traditional\proc\p18f97j60.asm
               ADCON0Save   0x000b0f       data     static C:\Users\LFRAD\Documents\CMS2Luc\ProjetsNettoyesCMSGit\ProjetCarteIO\project\Helpers.c
               ADCON0bits   0x000fc2       data     extern E:\MPASM_MPLINK_PIC18_LT_Branch_3_42\pic18-lt\cxx-framework\src\traditional\proc\p18f97j60.asm
                   ADCON1   0x000fc1       data     extern E:\MPASM_MPLINK_PIC18_LT_Branch_3_42\pic18-lt\cxx-framework\src\traditional\proc\p18f97j60.asm
               ADCON1bits   0x000fc1       data     extern E:\MPASM_MPLINK_PIC18_LT_Branch_3_42\pic18-lt\cxx-framework\src\traditional\proc\p18f97j60.asm
                   ADCON2   0x000fc0       data     extern E:\MPASM_MPLINK_PIC18_LT_Branch_3_42\pic18-lt\cxx-framework\src\traditional\proc\p18f97j60.asm
               ADCON2Save   0x000b10       data     static C:\Users\LFRAD\Documents\CMS2Luc\ProjetsNettoyesCMSGit\ProjetCarteIO\project\Helpers.c
               ADCON2bits   0x000fc0       data     extern E:\MPASM_MPLINK_PIC18_LT_Branch_3_42\pic18-lt\cxx-framework\src\traditional\proc\p18f97j60.asm
                     ADDE   0x00067e       data     static C:\Users\LFRAD\Documents\CMS2Luc\ProjetsNettoyesCMSGit\ProjetCarteIO\project\MainDemoV1.c
                     ADDE   0x0006a3       data     static C:\Users\LFRAD\Documents\CMS2Luc\ProjetsNettoyesCMSGit\ProjetCarteIO\project\MainDemoV1.c
                     ADDH   0x0006c1       data     static C:\Users\LFRAD\Documents\CMS2Luc\ProjetsNettoyesCMSGit\ProjetCarteIO\project\MainDemoV1.c
                    ADDHL   0x0006a4       data     static C:\Users\LFRAD\Documents\CMS2Luc\ProjetsNettoyesCMSGit\ProjetCarteIO\project\MainDemoV1.c
                    ADDHL   0x00067f       data     static C:\Users\LFRAD\Documents\CMS2Luc\ProjetsNettoyesCMSGit\ProjetCarteIO\project\MainDemoV1.c
                    ADRES   0x000fc3       data     extern E:\MPASM_MPLINK_PIC18_LT_Branch_3_42\pic18-lt\cxx-framework\src\traditional\proc\p18f97j60.asm
                   ADRESH   0x000fc4       data     extern E:\MPASM_MPLINK_PIC18_LT_Branch_3_42\pic18-lt\cxx-framework\src\traditional\proc\p18f97j60.asm
                   ADRESL   0x000fc3       data     extern E:\MPASM_MPLINK_PIC18_LT_Branch_3_42\pic18-lt\cxx-framework\src\traditional\proc\p18f97j60.asm
                   ALARME   0x000600       data     extern C:\Users\LFRAD\Documents\CMS2Luc\ProjetsNettoyesCMSGit\ProjetCarteIO\project\MainDemoV1.c
             ALARMEATRANS   0x0009e6       data     extern C:\Users\LFRAD\Documents\CMS2Luc\ProjetsNettoyesCMSGit\ProjetCarteIO\project\MainDemoV1.c
                AN0String   0x0008e5       data     extern C:\Users\LFRAD\Documents\CMS2Luc\ProjetsNettoyesCMSGit\ProjetCarteIO\project\MainDemoV1.c
                    ANNEE   0x000b05       data     static C:\Users\LFRAD\Documents\CMS2Luc\ProjetsNettoyesCMSGit\ProjetCarteIO\project\MainDemoV1.c
                    ANNEE   0x000b05       data     static C:\Users\LFRAD\Documents\CMS2Luc\ProjetsNettoyesCMSGit\ProjetCarteIO\project\MainDemoV1.c
                     AddH   0x0006bc       data     static C:\Users\LFRAD\Documents\CMS2Luc\ProjetsNettoyesCMSGit\ProjetCarteIO\project\MainDemoV1.c
                     AddH   0x000b16       data     static C:\Users\LFRAD\Documents\CMS2Luc\ProjetsNettoyesCMSGit\ProjetCarteIO\project\MainDemoV1.c
                     AddH   0x000b05       data     static C:\Users\LFRAD\Documents\CMS2Luc\ProjetsNettoyesCMSGit\ProjetCarteIO\project\MainDemoV1.c
                     AddL   0x000b06       data     static C:\Users\LFRAD\Documents\CMS2Luc\ProjetsNettoyesCMSGit\ProjetCarteIO\project\MainDemoV1.c
                     AddL   0x000b17       data     static C:\Users\LFRAD\Documents\CMS2Luc\ProjetsNettoyesCMSGit\ProjetCarteIO\project\MainDemoV1.c
                AppConfig   0x0008b0       data     extern C:\Users\LFRAD\Documents\CMS2Luc\ProjetsNettoyesCMSGit\ProjetCarteIO\project\MainDemoV1.c
               AsciiChars   0x000a11       data     static C:\Users\LFRAD\Documents\CMS2Luc\ProjetsNettoyesCMSGit\ProjetCarteIO\project\Helpers.c
                  BAUDCON   0x000f7e       data     extern E:\MPASM_MPLINK_PIC18_LT_Branch_3_42\pic18-lt\cxx-framework\src\traditional\proc\p18f97j60.asm
                 BAUDCON1   0x000f7e       data     extern E:\MPASM_MPLINK_PIC18_LT_Branch_3_42\pic18-lt\cxx-framework\src\traditional\proc\p18f97j60.asm
             BAUDCON1bits   0x000f7e       data     extern E:\MPASM_MPLINK_PIC18_LT_Branch_3_42\pic18-lt\cxx-framework\src\traditional\proc\p18f97j60.asm
                 BAUDCON2   0x000f7c       data     extern E:\MPASM_MPLINK_PIC18_LT_Branch_3_42\pic18-lt\cxx-framework\src\traditional\proc\p18f97j60.asm
             BAUDCON2bits   0x000f7c       data     extern E:\MPASM_MPLINK_PIC18_LT_Branch_3_42\pic18-lt\cxx-framework\src\traditional\proc\p18f97j60.asm
              BAUDCONbits   0x000f7e       data     extern E:\MPASM_MPLINK_PIC18_LT_Branch_3_42\pic18-lt\cxx-framework\src\traditional\proc\p18f97j60.asm
                  BAUDCTL   0x000f7e       data     extern E:\MPASM_MPLINK_PIC18_LT_Branch_3_42\pic18-lt\cxx-framework\src\traditional\proc\p18f97j60.asm
                 BAUDCTL1   0x000f7e       data     extern E:\MPASM_MPLINK_PIC18_LT_Branch_3_42\pic18-lt\cxx-framework\src\traditional\proc\p18f97j60.asm
             BAUDCTL1bits   0x000f7e       data     extern E:\MPASM_MPLINK_PIC18_LT_Branch_3_42\pic18-lt\cxx-framework\src\traditional\proc\p18f97j60.asm
                 BAUDCTL2   0x000f7c       data     extern E:\MPASM_MPLINK_PIC18_LT_Branch_3_42\pic18-lt\cxx-framework\src\traditional\proc\p18f97j60.asm
             BAUDCTL2bits   0x000f7c       data     extern E:\MPASM_MPLINK_PIC18_LT_Branch_3_42\pic18-lt\cxx-framework\src\traditional\proc\p18f97j60.asm
              BAUDCTLbits   0x000f7e       data     extern E:\MPASM_MPLINK_PIC18_LT_Branch_3_42\pic18-lt\cxx-framework\src\traditional\proc\p18f97j60.asm
            BOUCLEATTENTE   0x00087f       data     extern C:\Users\LFRAD\Documents\CMS2Luc\ProjetsNettoyesCMSGit\ProjetCarteIO\project\MainDemoV1.c
                      BSR   0x000fe0       data     extern E:\MPASM_MPLINK_PIC18_LT_Branch_3_42\pic18-lt\cxx-framework\src\traditional\proc\p18f97j60.asm
                   Buffer   0x000a0f       data     static C:\Users\LFRAD\Documents\CMS2Luc\ProjetsNettoyesCMSGit\ProjetCarteIO\project\Helpers.c
                    CABLE   0x000908       data     extern C:\Users\LFRAD\Documents\CMS2Luc\ProjetsNettoyesCMSGit\ProjetCarteIO\project\MainDemoV1.c
                     CCON   0x00091e       data     extern C:\Users\LFRAD\Documents\CMS2Luc\ProjetsNettoyesCMSGit\ProjetCarteIO\project\MainDemoV1.c
                  CCP1CON   0x000fbd       data     extern E:\MPASM_MPLINK_PIC18_LT_Branch_3_42\pic18-lt\cxx-framework\src\traditional\proc\p18f97j60.asm
              CCP1CONbits   0x000fbd       data     extern E:\MPASM_MPLINK_PIC18_LT_Branch_3_42\pic18-lt\cxx-framework\src\traditional\proc\p18f97j60.asm
                  CCP2CON   0x000fba       data     extern E:\MPASM_MPLINK_PIC18_LT_Branch_3_42\pic18-lt\cxx-framework\src\traditional\proc\p18f97j60.asm
              CCP2CONbits   0x000fba       data     extern E:\MPASM_MPLINK_PIC18_LT_Branch_3_42\pic18-lt\cxx-framework\src\traditional\proc\p18f97j60.asm
                  CCP3CON   0x000fb7       data     extern E:\MPASM_MPLINK_PIC18_LT_Branch_3_42\pic18-lt\cxx-framework\src\traditional\proc\p18f97j60.asm
              CCP3CONbits   0x000fb7       data     extern E:\MPASM_MPLINK_PIC18_LT_Branch_3_42\pic18-lt\cxx-framework\src\traditional\proc\p18f97j60.asm
                  CCP4CON   0x000f73       data     extern E:\MPASM_MPLINK_PIC18_LT_Branch_3_42\pic18-lt\cxx-framework\src\traditional\proc\p18f97j60.asm
              CCP4CONbits   0x000f73       data     extern E:\MPASM_MPLINK_PIC18_LT_Branch_3_42\pic18-lt\cxx-framework\src\traditional\proc\p18f97j60.asm
                  CCP5CON   0x000f70       data     extern E:\MPASM_MPLINK_PIC18_LT_Branch_3_42\pic18-lt\cxx-framework\src\traditional\proc\p18f97j60.asm
              CCP5CONbits   0x000f70       data     extern E:\MPASM_MPLINK_PIC18_LT_Branch_3_42\pic18-lt\cxx-framework\src\traditional\proc\p18f97j60.asm
                    CCPR1   0x000fbe       data     extern E:\MPASM_MPLINK_PIC18_LT_Branch_3_42\pic18-lt\cxx-framework\src\traditional\proc\p18f97j60.asm
                   CCPR1H   0x000fbf       data     extern E:\MPASM_MPLINK_PIC18_LT_Branch_3_42\pic18-lt\cxx-framework\src\traditional\proc\p18f97j60.asm
                   CCPR1L   0x000fbe       data     extern E:\MPASM_MPLINK_PIC18_LT_Branch_3_42\pic18-lt\cxx-framework\src\traditional\proc\p18f97j60.asm
                    CCPR2   0x000fbb       data     extern E:\MPASM_MPLINK_PIC18_LT_Branch_3_42\pic18-lt\cxx-framework\src\traditional\proc\p18f97j60.asm
                   CCPR2H   0x000fbc       data     extern E:\MPASM_MPLINK_PIC18_LT_Branch_3_42\pic18-lt\cxx-framework\src\traditional\proc\p18f97j60.asm
                   CCPR2L   0x000fbb       data     extern E:\MPASM_MPLINK_PIC18_LT_Branch_3_42\pic18-lt\cxx-framework\src\traditional\proc\p18f97j60.asm
                    CCPR3   0x000fb8       data     extern E:\MPASM_MPLINK_PIC18_LT_Branch_3_42\pic18-lt\cxx-framework\src\traditional\proc\p18f97j60.asm
                   CCPR3H   0x000fb9       data     extern E:\MPASM_MPLINK_PIC18_LT_Branch_3_42\pic18-lt\cxx-framework\src\traditional\proc\p18f97j60.asm
                   CCPR3L   0x000fb8       data     extern E:\MPASM_MPLINK_PIC18_LT_Branch_3_42\pic18-lt\cxx-framework\src\traditional\proc\p18f97j60.asm
                    CCPR4   0x000f74       data     extern E:\MPASM_MPLINK_PIC18_LT_Branch_3_42\pic18-lt\cxx-framework\src\traditional\proc\p18f97j60.asm
                   CCPR4H   0x000f75       data     extern E:\MPASM_MPLINK_PIC18_LT_Branch_3_42\pic18-lt\cxx-framework\src\traditional\proc\p18f97j60.asm
                   CCPR4L   0x000f74       data     extern E:\MPASM_MPLINK_PIC18_LT_Branch_3_42\pic18-lt\cxx-framework\src\traditional\proc\p18f97j60.asm
                    CCPR5   0x000f71       data     extern E:\MPASM_MPLINK_PIC18_LT_Branch_3_42\pic18-lt\cxx-framework\src\traditional\proc\p18f97j60.asm
                   CCPR5H   0x000f72       data     extern E:\MPASM_MPLINK_PIC18_LT_Branch_3_42\pic18-lt\cxx-framework\src\traditional\proc\p18f97j60.asm
                   CCPR5L   0x000f71       data     extern E:\MPASM_MPLINK_PIC18_LT_Branch_3_42\pic18-lt\cxx-framework\src\traditional\proc\p18f97j60.asm
               CHG_CODAGE   0x000e3c       data     extern C:\Users\LFRAD\Documents\CMS2Luc\ProjetsNettoyesCMSGit\ProjetCarteIO\project\MainDemoV1.c
                    CMCON   0x000fb4       data     extern E:\MPASM_MPLINK_PIC18_LT_Branch_3_42\pic18-lt\cxx-framework\src\traditional\proc\p18f97j60.asm
                CMCONbits   0x000fb4       data     extern E:\MPASM_MPLINK_PIC18_LT_Branch_3_42\pic18-lt\cxx-framework\src\traditional\proc\p18f97j60.asm
                     CMOD   0x000926       data     extern C:\Users\LFRAD\Documents\CMS2Luc\ProjetsNettoyesCMSGit\ProjetCarteIO\project\MainDemoV1.c
                  CMouPAS   0x000902       data     extern C:\Users\LFRAD\Documents\CMS2Luc\ProjetsNettoyesCMSGit\ProjetCarteIO\project\MainDemoV1.c
                      COD   0x000918       data     extern C:\Users\LFRAD\Documents\CMS2Luc\ProjetsNettoyesCMSGit\ProjetCarteIO\project\MainDemoV1.c
              COMMENTAIRE   0x00095b       data     extern C:\Users\LFRAD\Documents\CMS2Luc\ProjetsNettoyesCMSGit\ProjetCarteIO\project\MainDemoV1.c
           COMMENTAIRESAV   0x000e4d       data     extern C:\Users\LFRAD\Documents\CMS2Luc\ProjetsNettoyesCMSGit\ProjetCarteIO\project\MainDemoV1.c
             CONSTITUTION   0x00093f       data     extern C:\Users\LFRAD\Documents\CMS2Luc\ProjetsNettoyesCMSGit\ProjetCarteIO\project\MainDemoV1.c
                      CRC   0x0000e7       data     extern C:\Users\LFRAD\Documents\CMS2Luc\ProjetsNettoyesCMSGit\ProjetCarteIO\project\GenericTCPServer.c
                  CRC2021   0x00066a       data     extern C:\Users\LFRAD\Documents\CMS2Luc\ProjetsNettoyesCMSGit\ProjetCarteIO\project\MainDemoV1.c
                   CRC485   0x000a43       data     extern C:\Users\LFRAD\Documents\CMS2Luc\ProjetsNettoyesCMSGit\ProjetCarteIO\project\MainDemoV1.c
                 CRC_ETAT   0x0009ea       data     extern C:\Users\LFRAD\Documents\CMS2Luc\ProjetsNettoyesCMSGit\ProjetCarteIO\project\MainDemoV1.c
                   CRCcal   0x000b0c       data     static C:\Users\LFRAD\Documents\CMS2Luc\ProjetsNettoyesCMSGit\ProjetCarteIO\project\MainDemoV1.c
                     CREP   0x000922       data     extern C:\Users\LFRAD\Documents\CMS2Luc\ProjetsNettoyesCMSGit\ProjetCarteIO\project\MainDemoV1.c
                   CVRCON   0x000fb5       data     extern E:\MPASM_MPLINK_PIC18_LT_Branch_3_42\pic18-lt\cxx-framework\src\traditional\proc\p18f97j60.asm
               CVRCONbits   0x000fb5       data     extern E:\MPASM_MPLINK_PIC18_LT_Branch_3_42\pic18-lt\cxx-framework\src\traditional\proc\p18f97j60.asm
                    Cache   0x0006d5       data     static C:\Users\LFRAD\Documents\CMS2Luc\ProjetsNettoyesCMSGit\ProjetCarteIO\project\ARP.c
             CalcChecksum   0x000b00       data     static C:\Users\LFRAD\Documents\CMS2Luc\ProjetsNettoyesCMSGit\ProjetCarteIO\project\IP.c
                    Carac   0x000b00       data     static C:\Users\LFRAD\Documents\CMS2Luc\ProjetsNettoyesCMSGit\ProjetCarteIO\project\MainDemoV1.c
                     Cent   0x000b02       data     static C:\Users\LFRAD\Documents\CMS2Luc\ProjetsNettoyesCMSGit\ProjetCarteIO\project\MainDemoV1.c
                     Cent   0x000b02       data     static C:\Users\LFRAD\Documents\CMS2Luc\ProjetsNettoyesCMSGit\ProjetCarteIO\project\MainDemoV1.c
                     Cent   0x000b02       data     static C:\Users\LFRAD\Documents\CMS2Luc\ProjetsNettoyesCMSGit\ProjetCarteIO\project\GenericTCPClient.c
                 Checksum   0x000b27       data     static C:\Users\LFRAD\Documents\CMS2Luc\ProjetsNettoyesCMSGit\ProjetCarteIO\project\ETH97J60.c
                 ChunkLen   0x000b2b       data     static C:\Users\LFRAD\Documents\CMS2Luc\ProjetsNettoyesCMSGit\ProjetCarteIO\project\ETH97J60.c
    CurrentPacketLocation   0x000a74       data     static C:\Users\LFRAD\Documents\CMS2Luc\ProjetsNettoyesCMSGit\ProjetCarteIO\project\ETH97J60.c
                     DATE   0x000b06       data     static C:\Users\LFRAD\Documents\CMS2Luc\ProjetsNettoyesCMSGit\ProjetCarteIO\project\MainDemoV1.c
                     DATE   0x000b06       data     static C:\Users\LFRAD\Documents\CMS2Luc\ProjetsNettoyesCMSGit\ProjetCarteIO\project\MainDemoV1.c
                     DDRA   0x000f92       data     extern E:\MPASM_MPLINK_PIC18_LT_Branch_3_42\pic18-lt\cxx-framework\src\traditional\proc\p18f97j60.asm
                 DDRAbits   0x000f92       data     extern E:\MPASM_MPLINK_PIC18_LT_Branch_3_42\pic18-lt\cxx-framework\src\traditional\proc\p18f97j60.asm
                     DDRB   0x000f93       data     extern E:\MPASM_MPLINK_PIC18_LT_Branch_3_42\pic18-lt\cxx-framework\src\traditional\proc\p18f97j60.asm
                 DDRBbits   0x000f93       data     extern E:\MPASM_MPLINK_PIC18_LT_Branch_3_42\pic18-lt\cxx-framework\src\traditional\proc\p18f97j60.asm
                     DDRC   0x000f94       data     extern E:\MPASM_MPLINK_PIC18_LT_Branch_3_42\pic18-lt\cxx-framework\src\traditional\proc\p18f97j60.asm
                 DDRCbits   0x000f94       data     extern E:\MPASM_MPLINK_PIC18_LT_Branch_3_42\pic18-lt\cxx-framework\src\traditional\proc\p18f97j60.asm
                     DDRD   0x000f95       data     extern E:\MPASM_MPLINK_PIC18_LT_Branch_3_42\pic18-lt\cxx-framework\src\traditional\proc\p18f97j60.asm
                 DDRDbits   0x000f95       data     extern E:\MPASM_MPLINK_PIC18_LT_Branch_3_42\pic18-lt\cxx-framework\src\traditional\proc\p18f97j60.asm
                     DDRE   0x000f96       data     extern E:\MPASM_MPLINK_PIC18_LT_Branch_3_42\pic18-lt\cxx-framework\src\traditional\proc\p18f97j60.asm
                 DDREbits   0x000f96       data     extern E:\MPASM_MPLINK_PIC18_LT_Branch_3_42\pic18-lt\cxx-framework\src\traditional\proc\p18f97j60.asm
                     DDRF   0x000f97       data     extern E:\MPASM_MPLINK_PIC18_LT_Branch_3_42\pic18-lt\cxx-framework\src\traditional\proc\p18f97j60.asm
                 DDRFbits   0x000f97       data     extern E:\MPASM_MPLINK_PIC18_LT_Branch_3_42\pic18-lt\cxx-framework\src\traditional\proc\p18f97j60.asm
                     DDRG   0x000f98       data     extern E:\MPASM_MPLINK_PIC18_LT_Branch_3_42\pic18-lt\cxx-framework\src\traditional\proc\p18f97j60.asm
                 DDRGbits   0x000f98       data     extern E:\MPASM_MPLINK_PIC18_LT_Branch_3_42\pic18-lt\cxx-framework\src\traditional\proc\p18f97j60.asm
                     DDRH   0x000f99       data     extern E:\MPASM_MPLINK_PIC18_LT_Branch_3_42\pic18-lt\cxx-framework\src\traditional\proc\p18f97j60.asm
                 DDRHbits   0x000f99       data     extern E:\MPASM_MPLINK_PIC18_LT_Branch_3_42\pic18-lt\cxx-framework\src\traditional\proc\p18f97j60.asm
                     DDRJ   0x000f9a       data     extern E:\MPASM_MPLINK_PIC18_LT_Branch_3_42\pic18-lt\cxx-framework\src\traditional\proc\p18f97j60.asm
                 DDRJbits   0x000f9a       data     extern E:\MPASM_MPLINK_PIC18_LT_Branch_3_42\pic18-lt\cxx-framework\src\traditional\proc\p18f97j60.asm
             DEBIT_GLOBAL   0x0005b5       data     extern C:\Users\LFRAD\Documents\CMS2Luc\ProjetsNettoyesCMSGit\ProjetCarteIO\project\MainDemoV1.c
         DEMANDE_DE_LAUTO   0x0000e1       data     extern C:\Users\LFRAD\Documents\CMS2Luc\ProjetsNettoyesCMSGit\ProjetCarteIO\project\MainDemoV1.c
   DEMANDE_INFOS_CAPTEURS   0x000a4b       data     extern C:\Users\LFRAD\Documents\CMS2Luc\ProjetsNettoyesCMSGit\ProjetCarteIO\project\MainDemoV1.c
                 DISTANCE   0x000950       data     extern C:\Users\LFRAD\Documents\CMS2Luc\ProjetsNettoyesCMSGit\ProjetCarteIO\project\MainDemoV1.c
                     DMil   0x000b08       data     static C:\Users\LFRAD\Documents\CMS2Luc\ProjetsNettoyesCMSGit\ProjetCarteIO\project\MainDemoV1.c
                     DMil   0x000b08       data     static C:\Users\LFRAD\Documents\CMS2Luc\ProjetsNettoyesCMSGit\ProjetCarteIO\project\MainDemoV1.c
                     DMil   0x000b08       data     static C:\Users\LFRAD\Documents\CMS2Luc\ProjetsNettoyesCMSGit\ProjetCarteIO\project\GenericTCPClient.c
                      DNS   0x0000a2       data     extern C:\Users\LFRAD\Documents\CMS2Luc\ProjetsNettoyesCMSGit\ProjetCarteIO\project\MainDemoV1.c
          DNSAnswerHeader   0x000b52       data     static C:\Users\LFRAD\Documents\CMS2Luc\ProjetsNettoyesCMSGit\ProjetCarteIO\project\DNS.c
                DNSHeader   0x000b46       data     static C:\Users\LFRAD\Documents\CMS2Luc\ProjetsNettoyesCMSGit\ProjetCarteIO\project\DNS.c
              DNSHostName   0x0007cf       data     static C:\Users\LFRAD\Documents\CMS2Luc\ProjetsNettoyesCMSGit\ProjetCarteIO\project\DNS.c
           DNSHostNameROM   0x0007d1       data     static C:\Users\LFRAD\Documents\CMS2Luc\ProjetsNettoyesCMSGit\ProjetCarteIO\project\DNS.c
                     Data   0x000b07       data     static C:\Users\LFRAD\Documents\CMS2Luc\ProjetsNettoyesCMSGit\ProjetCarteIO\project\MainDemoV1.c
                     Data   0x000aa6       data     static C:\Users\LFRAD\Documents\CMS2Luc\ProjetsNettoyesCMSGit\ProjetCarteIO\project\ETH97J60.c
               DataBuffer   0x000b2d       data     static C:\Users\LFRAD\Documents\CMS2Luc\ProjetsNettoyesCMSGit\ProjetCarteIO\project\ETH97J60.c
                  DataPtr   0x000b41       data     static C:\Users\LFRAD\Documents\CMS2Luc\ProjetsNettoyesCMSGit\ProjetCarteIO\project\ETH97J60.c
               DestIPAddr   0x0006e3       data     static C:\Users\LFRAD\Documents\CMS2Luc\ProjetsNettoyesCMSGit\ProjetCarteIO\project\ARP.c
                    Digit   0x000b01       data     static C:\Users\LFRAD\Documents\CMS2Luc\ProjetsNettoyesCMSGit\ProjetCarteIO\project\Helpers.c
                  Divisor   0x000b03       data     static C:\Users\LFRAD\Documents\CMS2Luc\ProjetsNettoyesCMSGit\ProjetCarteIO\project\Helpers.c
                      Diz   0x000b04       data     static C:\Users\LFRAD\Documents\CMS2Luc\ProjetsNettoyesCMSGit\ProjetCarteIO\project\MainDemoV1.c
                      Diz   0x000b04       data     static C:\Users\LFRAD\Documents\CMS2Luc\ProjetsNettoyesCMSGit\ProjetCarteIO\project\GenericTCPClient.c
                      Diz   0x000b04       data     static C:\Users\LFRAD\Documents\CMS2Luc\ProjetsNettoyesCMSGit\ProjetCarteIO\project\MainDemoV1.c
                  EALARME   0x000c6e       data     static C:\Users\LFRAD\Documents\CMS2Luc\ProjetsNettoyesCMSGit\ProjetCarteIO\project\MainDemoV1.c
                  ECCP1AS   0x000fb6       data     extern E:\MPASM_MPLINK_PIC18_LT_Branch_3_42\pic18-lt\cxx-framework\src\traditional\proc\p18f97j60.asm
              ECCP1ASbits   0x000fb6       data     extern E:\MPASM_MPLINK_PIC18_LT_Branch_3_42\pic18-lt\cxx-framework\src\traditional\proc\p18f97j60.asm
                 ECCP1CON   0x000fbd       data     extern E:\MPASM_MPLINK_PIC18_LT_Branch_3_42\pic18-lt\cxx-framework\src\traditional\proc\p18f97j60.asm
             ECCP1CONbits   0x000fbd       data     extern E:\MPASM_MPLINK_PIC18_LT_Branch_3_42\pic18-lt\cxx-framework\src\traditional\proc\p18f97j60.asm
                 ECCP1DEL   0x000f79       data     extern E:\MPASM_MPLINK_PIC18_LT_Branch_3_42\pic18-lt\cxx-framework\src\traditional\proc\p18f97j60.asm
             ECCP1DELbits   0x000f79       data     extern E:\MPASM_MPLINK_PIC18_LT_Branch_3_42\pic18-lt\cxx-framework\src\traditional\proc\p18f97j60.asm
                  ECCP2AS   0x000f68       data     extern E:\MPASM_MPLINK_PIC18_LT_Branch_3_42\pic18-lt\cxx-framework\src\traditional\proc\p18f97j60.asm
              ECCP2ASbits   0x000f68       data     extern E:\MPASM_MPLINK_PIC18_LT_Branch_3_42\pic18-lt\cxx-framework\src\traditional\proc\p18f97j60.asm
                 ECCP2CON   0x000fba       data     extern E:\MPASM_MPLINK_PIC18_LT_Branch_3_42\pic18-lt\cxx-framework\src\traditional\proc\p18f97j60.asm
             ECCP2CONbits   0x000fba       data     extern E:\MPASM_MPLINK_PIC18_LT_Branch_3_42\pic18-lt\cxx-framework\src\traditional\proc\p18f97j60.asm
                 ECCP2DEL   0x000f67       data     extern E:\MPASM_MPLINK_PIC18_LT_Branch_3_42\pic18-lt\cxx-framework\src\traditional\proc\p18f97j60.asm
             ECCP2DELbits   0x000f67       data     extern E:\MPASM_MPLINK_PIC18_LT_Branch_3_42\pic18-lt\cxx-framework\src\traditional\proc\p18f97j60.asm
                  ECCP3AS   0x000f6a       data     extern E:\MPASM_MPLINK_PIC18_LT_Branch_3_42\pic18-lt\cxx-framework\src\traditional\proc\p18f97j60.asm
              ECCP3ASbits   0x000f6a       data     extern E:\MPASM_MPLINK_PIC18_LT_Branch_3_42\pic18-lt\cxx-framework\src\traditional\proc\p18f97j60.asm
                 ECCP3CON   0x000fb7       data     extern E:\MPASM_MPLINK_PIC18_LT_Branch_3_42\pic18-lt\cxx-framework\src\traditional\proc\p18f97j60.asm
             ECCP3CONbits   0x000fb7       data     extern E:\MPASM_MPLINK_PIC18_LT_Branch_3_42\pic18-lt\cxx-framework\src\traditional\proc\p18f97j60.asm
                 ECCP3DEL   0x000f69       data     extern E:\MPASM_MPLINK_PIC18_LT_Branch_3_42\pic18-lt\cxx-framework\src\traditional\proc\p18f97j60.asm
             ECCP3DELbits   0x000f69       data     extern E:\MPASM_MPLINK_PIC18_LT_Branch_3_42\pic18-lt\cxx-framework\src\traditional\proc\p18f97j60.asm
                    ECON1   0x000fd2       data     extern E:\MPASM_MPLINK_PIC18_LT_Branch_3_42\pic18-lt\cxx-framework\src\traditional\proc\p18f97j60.asm
                ECON1bits   0x000fd2       data     extern E:\MPASM_MPLINK_PIC18_LT_Branch_3_42\pic18-lt\cxx-framework\src\traditional\proc\p18f97j60.asm
                    ECON2   0x000efe       data     extern E:\MPASM_MPLINK_PIC18_LT_Branch_3_42\pic18-lt\cxx-framework\src\traditional\proc\p18f97j60.asm
                ECON2bits   0x000efe       data     extern E:\MPASM_MPLINK_PIC18_LT_Branch_3_42\pic18-lt\cxx-framework\src\traditional\proc\p18f97j60.asm
                    EDATA   0x000f61       data     extern E:\MPASM_MPLINK_PIC18_LT_Branch_3_42\pic18-lt\cxx-framework\src\traditional\proc\p18f97j60.asm
                EDATAbits   0x000f61       data     extern E:\MPASM_MPLINK_PIC18_LT_Branch_3_42\pic18-lt\cxx-framework\src\traditional\proc\p18f97j60.asm
                   EDMACS   0x000ef6       data     extern E:\MPASM_MPLINK_PIC18_LT_Branch_3_42\pic18-lt\cxx-framework\src\traditional\proc\p18f97j60.asm
                  EDMACSH   0x000ef7       data     extern E:\MPASM_MPLINK_PIC18_LT_Branch_3_42\pic18-lt\cxx-framework\src\traditional\proc\p18f97j60.asm
                  EDMACSL   0x000ef6       data     extern E:\MPASM_MPLINK_PIC18_LT_Branch_3_42\pic18-lt\cxx-framework\src\traditional\proc\p18f97j60.asm
                  EDMADST   0x000ef4       data     extern E:\MPASM_MPLINK_PIC18_LT_Branch_3_42\pic18-lt\cxx-framework\src\traditional\proc\p18f97j60.asm
                 EDMADSTH   0x000ef5       data     extern E:\MPASM_MPLINK_PIC18_LT_Branch_3_42\pic18-lt\cxx-framework\src\traditional\proc\p18f97j60.asm
                 EDMADSTL   0x000ef4       data     extern E:\MPASM_MPLINK_PIC18_LT_Branch_3_42\pic18-lt\cxx-framework\src\traditional\proc\p18f97j60.asm
                   EDMAND   0x000ef2       data     extern E:\MPASM_MPLINK_PIC18_LT_Branch_3_42\pic18-lt\cxx-framework\src\traditional\proc\p18f97j60.asm
                  EDMANDH   0x000ef3       data     extern E:\MPASM_MPLINK_PIC18_LT_Branch_3_42\pic18-lt\cxx-framework\src\traditional\proc\p18f97j60.asm
                  EDMANDL   0x000ef2       data     extern E:\MPASM_MPLINK_PIC18_LT_Branch_3_42\pic18-lt\cxx-framework\src\traditional\proc\p18f97j60.asm
                   EDMAST   0x000ef0       data     extern E:\MPASM_MPLINK_PIC18_LT_Branch_3_42\pic18-lt\cxx-framework\src\traditional\proc\p18f97j60.asm
                  EDMASTH   0x000ef1       data     extern E:\MPASM_MPLINK_PIC18_LT_Branch_3_42\pic18-lt\cxx-framework\src\traditional\proc\p18f97j60.asm
                  EDMASTL   0x000ef0       data     extern E:\MPASM_MPLINK_PIC18_LT_Branch_3_42\pic18-lt\cxx-framework\src\traditional\proc\p18f97j60.asm
                   EECON1   0x000fa6       data     extern E:\MPASM_MPLINK_PIC18_LT_Branch_3_42\pic18-lt\cxx-framework\src\traditional\proc\p18f97j60.asm
               EECON1bits   0x000fa6       data     extern E:\MPASM_MPLINK_PIC18_LT_Branch_3_42\pic18-lt\cxx-framework\src\traditional\proc\p18f97j60.asm
                   EECON2   0x000fa7       data     extern E:\MPASM_MPLINK_PIC18_LT_Branch_3_42\pic18-lt\cxx-framework\src\traditional\proc\p18f97j60.asm
                  EFLOCON   0x000e97       data     extern E:\MPASM_MPLINK_PIC18_LT_Branch_3_42\pic18-lt\cxx-framework\src\traditional\proc\p18f97j60.asm
              EFLOCONbits   0x000e97       data     extern E:\MPASM_MPLINK_PIC18_LT_Branch_3_42\pic18-lt\cxx-framework\src\traditional\proc\p18f97j60.asm
                     EHT0   0x000ec0       data     extern E:\MPASM_MPLINK_PIC18_LT_Branch_3_42\pic18-lt\cxx-framework\src\traditional\proc\p18f97j60.asm
                     EHT1   0x000ec1       data     extern E:\MPASM_MPLINK_PIC18_LT_Branch_3_42\pic18-lt\cxx-framework\src\traditional\proc\p18f97j60.asm
                     EHT2   0x000ec2       data     extern E:\MPASM_MPLINK_PIC18_LT_Branch_3_42\pic18-lt\cxx-framework\src\traditional\proc\p18f97j60.asm
                     EHT3   0x000ec3       data     extern E:\MPASM_MPLINK_PIC18_LT_Branch_3_42\pic18-lt\cxx-framework\src\traditional\proc\p18f97j60.asm
                     EHT4   0x000ec4       data     extern E:\MPASM_MPLINK_PIC18_LT_Branch_3_42\pic18-lt\cxx-framework\src\traditional\proc\p18f97j60.asm
                     EHT5   0x000ec5       data     extern E:\MPASM_MPLINK_PIC18_LT_Branch_3_42\pic18-lt\cxx-framework\src\traditional\proc\p18f97j60.asm
                     EHT6   0x000ec6       data     extern E:\MPASM_MPLINK_PIC18_LT_Branch_3_42\pic18-lt\cxx-framework\src\traditional\proc\p18f97j60.asm
                     EHT7   0x000ec7       data     extern E:\MPASM_MPLINK_PIC18_LT_Branch_3_42\pic18-lt\cxx-framework\src\traditional\proc\p18f97j60.asm
                      EIE   0x000efb       data     extern E:\MPASM_MPLINK_PIC18_LT_Branch_3_42\pic18-lt\cxx-framework\src\traditional\proc\p18f97j60.asm
                  EIEbits   0x000efb       data     extern E:\MPASM_MPLINK_PIC18_LT_Branch_3_42\pic18-lt\cxx-framework\src\traditional\proc\p18f97j60.asm
                      EIR   0x000f60       data     extern E:\MPASM_MPLINK_PIC18_LT_Branch_3_42\pic18-lt\cxx-framework\src\traditional\proc\p18f97j60.asm
                  EIRbits   0x000f60       data     extern E:\MPASM_MPLINK_PIC18_LT_Branch_3_42\pic18-lt\cxx-framework\src\traditional\proc\p18f97j60.asm
             ENVOYEROUPAS   0x000b77       data     static C:\Users\LFRAD\Documents\CMS2Luc\ProjetsNettoyesCMSGit\ProjetCarteIO\project\MainDemoV1.c
                    EPAUS   0x000e98       data     extern E:\MPASM_MPLINK_PIC18_LT_Branch_3_42\pic18-lt\cxx-framework\src\traditional\proc\p18f97j60.asm
                   EPAUSH   0x000e99       data     extern E:\MPASM_MPLINK_PIC18_LT_Branch_3_42\pic18-lt\cxx-framework\src\traditional\proc\p18f97j60.asm
                   EPAUSL   0x000e98       data     extern E:\MPASM_MPLINK_PIC18_LT_Branch_3_42\pic18-lt\cxx-framework\src\traditional\proc\p18f97j60.asm
                  EPKTCNT   0x000ed9       data     extern E:\MPASM_MPLINK_PIC18_LT_Branch_3_42\pic18-lt\cxx-framework\src\traditional\proc\p18f97j60.asm
                    EPMCS   0x000ed0       data     extern E:\MPASM_MPLINK_PIC18_LT_Branch_3_42\pic18-lt\cxx-framework\src\traditional\proc\p18f97j60.asm
                   EPMCSH   0x000ed1       data     extern E:\MPASM_MPLINK_PIC18_LT_Branch_3_42\pic18-lt\cxx-framework\src\traditional\proc\p18f97j60.asm
                   EPMCSL   0x000ed0       data     extern E:\MPASM_MPLINK_PIC18_LT_Branch_3_42\pic18-lt\cxx-framework\src\traditional\proc\p18f97j60.asm
                    EPMM0   0x000ec8       data     extern E:\MPASM_MPLINK_PIC18_LT_Branch_3_42\pic18-lt\cxx-framework\src\traditional\proc\p18f97j60.asm
                    EPMM1   0x000ec9       data     extern E:\MPASM_MPLINK_PIC18_LT_Branch_3_42\pic18-lt\cxx-framework\src\traditional\proc\p18f97j60.asm
                    EPMM2   0x000eca       data     extern E:\MPASM_MPLINK_PIC18_LT_Branch_3_42\pic18-lt\cxx-framework\src\traditional\proc\p18f97j60.asm
                    EPMM3   0x000ecb       data     extern E:\MPASM_MPLINK_PIC18_LT_Branch_3_42\pic18-lt\cxx-framework\src\traditional\proc\p18f97j60.asm
                    EPMM4   0x000ecc       data     extern E:\MPASM_MPLINK_PIC18_LT_Branch_3_42\pic18-lt\cxx-framework\src\traditional\proc\p18f97j60.asm
                    EPMM5   0x000ecd       data     extern E:\MPASM_MPLINK_PIC18_LT_Branch_3_42\pic18-lt\cxx-framework\src\traditional\proc\p18f97j60.asm
                    EPMM6   0x000ece       data     extern E:\MPASM_MPLINK_PIC18_LT_Branch_3_42\pic18-lt\cxx-framework\src\traditional\proc\p18f97j60.asm
                    EPMM7   0x000ecf       data     extern E:\MPASM_MPLINK_PIC18_LT_Branch_3_42\pic18-lt\cxx-framework\src\traditional\proc\p18f97j60.asm
                     EPMO   0x000ed4       data     extern E:\MPASM_MPLINK_PIC18_LT_Branch_3_42\pic18-lt\cxx-framework\src\traditional\proc\p18f97j60.asm
                    EPMOH   0x000ed5       data     extern E:\MPASM_MPLINK_PIC18_LT_Branch_3_42\pic18-lt\cxx-framework\src\traditional\proc\p18f97j60.asm
                    EPMOL   0x000ed4       data     extern E:\MPASM_MPLINK_PIC18_LT_Branch_3_42\pic18-lt\cxx-framework\src\traditional\proc\p18f97j60.asm
                    ERDPT   0x000f7a       data     extern E:\MPASM_MPLINK_PIC18_LT_Branch_3_42\pic18-lt\cxx-framework\src\traditional\proc\p18f97j60.asm
                   ERDPTH   0x000f7b       data     extern E:\MPASM_MPLINK_PIC18_LT_Branch_3_42\pic18-lt\cxx-framework\src\traditional\proc\p18f97j60.asm
                   ERDPTL   0x000f7a       data     extern E:\MPASM_MPLINK_PIC18_LT_Branch_3_42\pic18-lt\cxx-framework\src\traditional\proc\p18f97j60.asm
                  ERXFCON   0x000ed8       data     extern E:\MPASM_MPLINK_PIC18_LT_Branch_3_42\pic18-lt\cxx-framework\src\traditional\proc\p18f97j60.asm
              ERXFCONbits   0x000ed8       data     extern E:\MPASM_MPLINK_PIC18_LT_Branch_3_42\pic18-lt\cxx-framework\src\traditional\proc\p18f97j60.asm
                    ERXND   0x000eea       data     extern E:\MPASM_MPLINK_PIC18_LT_Branch_3_42\pic18-lt\cxx-framework\src\traditional\proc\p18f97j60.asm
                   ERXNDH   0x000eeb       data     extern E:\MPASM_MPLINK_PIC18_LT_Branch_3_42\pic18-lt\cxx-framework\src\traditional\proc\p18f97j60.asm
                   ERXNDL   0x000eea       data     extern E:\MPASM_MPLINK_PIC18_LT_Branch_3_42\pic18-lt\cxx-framework\src\traditional\proc\p18f97j60.asm
                  ERXRDPT   0x000eec       data     extern E:\MPASM_MPLINK_PIC18_LT_Branch_3_42\pic18-lt\cxx-framework\src\traditional\proc\p18f97j60.asm
                 ERXRDPTH   0x000eed       data     extern E:\MPASM_MPLINK_PIC18_LT_Branch_3_42\pic18-lt\cxx-framework\src\traditional\proc\p18f97j60.asm
                 ERXRDPTL   0x000eec       data     extern E:\MPASM_MPLINK_PIC18_LT_Branch_3_42\pic18-lt\cxx-framework\src\traditional\proc\p18f97j60.asm
                    ERXST   0x000ee8       data     extern E:\MPASM_MPLINK_PIC18_LT_Branch_3_42\pic18-lt\cxx-framework\src\traditional\proc\p18f97j60.asm
                   ERXSTH   0x000ee9       data     extern E:\MPASM_MPLINK_PIC18_LT_Branch_3_42\pic18-lt\cxx-framework\src\traditional\proc\p18f97j60.asm
                   ERXSTL   0x000ee8       data     extern E:\MPASM_MPLINK_PIC18_LT_Branch_3_42\pic18-lt\cxx-framework\src\traditional\proc\p18f97j60.asm
                  ERXWRPT   0x000eee       data     extern E:\MPASM_MPLINK_PIC18_LT_Branch_3_42\pic18-lt\cxx-framework\src\traditional\proc\p18f97j60.asm
                 ERXWRPTH   0x000eef       data     extern E:\MPASM_MPLINK_PIC18_LT_Branch_3_42\pic18-lt\cxx-framework\src\traditional\proc\p18f97j60.asm
                 ERXWRPTL   0x000eee       data     extern E:\MPASM_MPLINK_PIC18_LT_Branch_3_42\pic18-lt\cxx-framework\src\traditional\proc\p18f97j60.asm
                       ES   0x000688       data     static C:\Users\LFRAD\Documents\CMS2Luc\ProjetsNettoyesCMSGit\ProjetCarteIO\project\MainDemoV1.c
                    ESTAT   0x000efd       data     extern E:\MPASM_MPLINK_PIC18_LT_Branch_3_42\pic18-lt\cxx-framework\src\traditional\proc\p18f97j60.asm
                ESTATbits   0x000efd       data     extern E:\MPASM_MPLINK_PIC18_LT_Branch_3_42\pic18-lt\cxx-framework\src\traditional\proc\p18f97j60.asm
                     ETAT   0x00094c       data     extern C:\Users\LFRAD\Documents\CMS2Luc\ProjetsNettoyesCMSGit\ProjetCarteIO\project\MainDemoV1.c
                    ETAT1   0x0009eb       data     static C:\Users\LFRAD\Documents\CMS2Luc\ProjetsNettoyesCMSGit\ProjetCarteIO\project\MainDemoV1.c
     ETAT_CONNECT_MINITEL   0x000901       data     extern C:\Users\LFRAD\Documents\CMS2Luc\ProjetsNettoyesCMSGit\ProjetCarteIO\project\MainDemoV1.c
                  ETAT_M1   0x0009b0       data     extern C:\Users\LFRAD\Documents\CMS2Luc\ProjetsNettoyesCMSGit\ProjetCarteIO\project\MainDemoV1.c
                    ETXND   0x000ee6       data     extern E:\MPASM_MPLINK_PIC18_LT_Branch_3_42\pic18-lt\cxx-framework\src\traditional\proc\p18f97j60.asm
                   ETXNDH   0x000ee7       data     extern E:\MPASM_MPLINK_PIC18_LT_Branch_3_42\pic18-lt\cxx-framework\src\traditional\proc\p18f97j60.asm
                   ETXNDL   0x000ee6       data     extern E:\MPASM_MPLINK_PIC18_LT_Branch_3_42\pic18-lt\cxx-framework\src\traditional\proc\p18f97j60.asm
                    ETXST   0x000ee4       data     extern E:\MPASM_MPLINK_PIC18_LT_Branch_3_42\pic18-lt\cxx-framework\src\traditional\proc\p18f97j60.asm
                   ETXSTH   0x000ee5       data     extern E:\MPASM_MPLINK_PIC18_LT_Branch_3_42\pic18-lt\cxx-framework\src\traditional\proc\p18f97j60.asm
                   ETXSTL   0x000ee4       data     extern E:\MPASM_MPLINK_PIC18_LT_Branch_3_42\pic18-lt\cxx-framework\src\traditional\proc\p18f97j60.asm
                     ET_C   0x00099d       data     extern C:\Users\LFRAD\Documents\CMS2Luc\ProjetsNettoyesCMSGit\ProjetCarteIO\project\MainDemoV1.c
                     ET_F   0x0009a1       data     extern C:\Users\LFRAD\Documents\CMS2Luc\ProjetsNettoyesCMSGit\ProjetCarteIO\project\MainDemoV1.c
                    ET_GR   0x00098d       data     extern C:\Users\LFRAD\Documents\CMS2Luc\ProjetsNettoyesCMSGit\ProjetCarteIO\project\MainDemoV1.c
                     ET_I   0x000999       data     extern C:\Users\LFRAD\Documents\CMS2Luc\ProjetsNettoyesCMSGit\ProjetCarteIO\project\MainDemoV1.c
                    ET_TD   0x000989       data     extern C:\Users\LFRAD\Documents\CMS2Luc\ProjetsNettoyesCMSGit\ProjetCarteIO\project\MainDemoV1.c
                    ET_TP   0x000991       data     extern C:\Users\LFRAD\Documents\CMS2Luc\ProjetsNettoyesCMSGit\ProjetCarteIO\project\MainDemoV1.c
                    ET_TR   0x000995       data     extern C:\Users\LFRAD\Documents\CMS2Luc\ProjetsNettoyesCMSGit\ProjetCarteIO\project\MainDemoV1.c
                    EWRPT   0x000ee2       data     extern E:\MPASM_MPLINK_PIC18_LT_Branch_3_42\pic18-lt\cxx-framework\src\traditional\proc\p18f97j60.asm
                   EWRPTH   0x000ee3       data     extern E:\MPASM_MPLINK_PIC18_LT_Branch_3_42\pic18-lt\cxx-framework\src\traditional\proc\p18f97j60.asm
                   EWRPTL   0x000ee2       data     extern E:\MPASM_MPLINK_PIC18_LT_Branch_3_42\pic18-lt\cxx-framework\src\traditional\proc\p18f97j60.asm
                 FONCTION   0x000a40       data     extern C:\Users\LFRAD\Documents\CMS2Luc\ProjetsNettoyesCMSGit\ProjetCarteIO\project\MainDemoV1.c
                     FSR0   0x000fe9       data     extern E:\MPASM_MPLINK_PIC18_LT_Branch_3_42\pic18-lt\cxx-framework\src\traditional\proc\p18f97j60.asm
                    FSR0H   0x000fea       data     extern E:\MPASM_MPLINK_PIC18_LT_Branch_3_42\pic18-lt\cxx-framework\src\traditional\proc\p18f97j60.asm
                    FSR0L   0x000fe9       data     extern E:\MPASM_MPLINK_PIC18_LT_Branch_3_42\pic18-lt\cxx-framework\src\traditional\proc\p18f97j60.asm
                     FSR1   0x000fe1       data     extern E:\MPASM_MPLINK_PIC18_LT_Branch_3_42\pic18-lt\cxx-framework\src\traditional\proc\p18f97j60.asm
                    FSR1H   0x000fe2       data     extern E:\MPASM_MPLINK_PIC18_LT_Branch_3_42\pic18-lt\cxx-framework\src\traditional\proc\p18f97j60.asm
                    FSR1L   0x000fe1       data     extern E:\MPASM_MPLINK_PIC18_LT_Branch_3_42\pic18-lt\cxx-framework\src\traditional\proc\p18f97j60.asm
                     FSR2   0x000fd9       data     extern E:\MPASM_MPLINK_PIC18_LT_Branch_3_42\pic18-lt\cxx-framework\src\traditional\proc\p18f97j60.asm
                    FSR2H   0x000fda       data     extern E:\MPASM_MPLINK_PIC18_LT_Branch_3_42\pic18-lt\cxx-framework\src\traditional\proc\p18f97j60.asm
                    FSR2L   0x000fd9       data     extern E:\MPASM_MPLINK_PIC18_LT_Branch_3_42\pic18-lt\cxx-framework\src\traditional\proc\p18f97j60.asm
                    Flags   0x0004c1       data     static C:\Users\LFRAD\Documents\CMS2Luc\ProjetsNettoyesCMSGit\ProjetCarteIO\project\UDP.c
                    Flags   0x000e6c       data     static C:\Users\LFRAD\Documents\CMS2Luc\ProjetsNettoyesCMSGit\ProjetCarteIO\project\DNS.c
                  GIESave   0x000b00       data     static C:\Users\LFRAD\Documents\CMS2Luc\ProjetsNettoyesCMSGit\ProjetCarteIO\project\ETH97J60.c
   GenericTCPExampleState   0x000e6a       data     static C:\Users\LFRAD\Documents\CMS2Luc\ProjetsNettoyesCMSGit\ProjetCarteIO\project\GenericTCPClient.c
                    HEURE   0x000b00       data     static C:\Users\LFRAD\Documents\CMS2Luc\ProjetsNettoyesCMSGit\ProjetCarteIO\project\MainDemoV1.c
                    HEURE   0x000b00       data     static C:\Users\LFRAD\Documents\CMS2Luc\ProjetsNettoyesCMSGit\ProjetCarteIO\project\MainDemoV1.c
                       HH   0x000934       data     extern C:\Users\LFRAD\Documents\CMS2Luc\ProjetsNettoyesCMSGit\ProjetCarteIO\project\MainDemoV1.c
                 HORLOGET   0x0000d5       data     extern C:\Users\LFRAD\Documents\CMS2Luc\ProjetsNettoyesCMSGit\ProjetCarteIO\project\MainDemoV1.c
                   HostIP   0x0007e6       data     static C:\Users\LFRAD\Documents\CMS2Luc\ProjetsNettoyesCMSGit\ProjetCarteIO\project\DNS.c
                 Hostname   0x0007e2       data     static C:\Users\LFRAD\Documents\CMS2Luc\ProjetsNettoyesCMSGit\ProjetCarteIO\project\DNS.c
                 Hostname   0x0007df       data     static C:\Users\LFRAD\Documents\CMS2Luc\ProjetsNettoyesCMSGit\ProjetCarteIO\project\DNS.c
                ICMPFlags   0x0009ff       data     static C:\Users\LFRAD\Documents\CMS2Luc\ProjetsNettoyesCMSGit\ProjetCarteIO\project\MainDemoV1.c
                      ID1   0x000a3c       data     extern C:\Users\LFRAD\Documents\CMS2Luc\ProjetsNettoyesCMSGit\ProjetCarteIO\project\MainDemoV1.c
                      ID2   0x000a3e       data     extern C:\Users\LFRAD\Documents\CMS2Luc\ProjetsNettoyesCMSGit\ProjetCarteIO\project\MainDemoV1.c
                  ID_rack   0x0000b1       data     extern C:\Users\LFRAD\Documents\CMS2Luc\ProjetsNettoyesCMSGit\ProjetCarteIO\project\MainDemoV1.c
                    INDF0   0x000fef       data     extern E:\MPASM_MPLINK_PIC18_LT_Branch_3_42\pic18-lt\cxx-framework\src\traditional\proc\p18f97j60.asm
                    INDF1   0x000fe7       data     extern E:\MPASM_MPLINK_PIC18_LT_Branch_3_42\pic18-lt\cxx-framework\src\traditional\proc\p18f97j60.asm
                    INDF2   0x000fdf       data     extern E:\MPASM_MPLINK_PIC18_LT_Branch_3_42\pic18-lt\cxx-framework\src\traditional\proc\p18f97j60.asm
       INFORMATION_ERREUR   0x000a57       data     extern C:\Users\LFRAD\Documents\CMS2Luc\ProjetsNettoyesCMSGit\ProjetCarteIO\project\MainDemoV1.c
                   INTCON   0x000ff2       data     extern E:\MPASM_MPLINK_PIC18_LT_Branch_3_42\pic18-lt\cxx-framework\src\traditional\proc\p18f97j60.asm
                  INTCON2   0x000ff1       data     extern E:\MPASM_MPLINK_PIC18_LT_Branch_3_42\pic18-lt\cxx-framework\src\traditional\proc\p18f97j60.asm
              INTCON2bits   0x000ff1       data     extern E:\MPASM_MPLINK_PIC18_LT_Branch_3_42\pic18-lt\cxx-framework\src\traditional\proc\p18f97j60.asm
                  INTCON3   0x000ff0       data     extern E:\MPASM_MPLINK_PIC18_LT_Branch_3_42\pic18-lt\cxx-framework\src\traditional\proc\p18f97j60.asm
              INTCON3bits   0x000ff0       data     extern E:\MPASM_MPLINK_PIC18_LT_Branch_3_42\pic18-lt\cxx-framework\src\traditional\proc\p18f97j60.asm
               INTCONbits   0x000ff2       data     extern E:\MPASM_MPLINK_PIC18_LT_Branch_3_42\pic18-lt\cxx-framework\src\traditional\proc\p18f97j60.asm
                   IPAddr   0x0006f6       data     static C:\Users\LFRAD\Documents\CMS2Luc\ProjetsNettoyesCMSGit\ProjetCarteIO\project\ARP.c
                   IPAddr   0x0006f4       data     static C:\Users\LFRAD\Documents\CMS2Luc\ProjetsNettoyesCMSGit\ProjetCarteIO\project\ARP.c
                IPAddress   0x000a06       data     static C:\Users\LFRAD\Documents\CMS2Luc\ProjetsNettoyesCMSGit\ProjetCarteIO\project\Helpers.c
                IPAddress   0x000a0b       data     static C:\Users\LFRAD\Documents\CMS2Luc\ProjetsNettoyesCMSGit\ProjetCarteIO\project\Helpers.c
                  IPDigit   0x000b06       data     static C:\Users\LFRAD\Documents\CMS2Luc\ProjetsNettoyesCMSGit\ProjetCarteIO\project\MainDemoV1.c
              IPHeaderLen   0x0005ea       data     static C:\Users\LFRAD\Documents\CMS2Luc\ProjetsNettoyesCMSGit\ProjetCarteIO\project\IP.c
                     IPR1   0x000f9f       data     extern E:\MPASM_MPLINK_PIC18_LT_Branch_3_42\pic18-lt\cxx-framework\src\traditional\proc\p18f97j60.asm
                 IPR1bits   0x000f9f       data     extern E:\MPASM_MPLINK_PIC18_LT_Branch_3_42\pic18-lt\cxx-framework\src\traditional\proc\p18f97j60.asm
                     IPR2   0x000fa2       data     extern E:\MPASM_MPLINK_PIC18_LT_Branch_3_42\pic18-lt\cxx-framework\src\traditional\proc\p18f97j60.asm
                 IPR2bits   0x000fa2       data     extern E:\MPASM_MPLINK_PIC18_LT_Branch_3_42\pic18-lt\cxx-framework\src\traditional\proc\p18f97j60.asm
                     IPR3   0x000fa5       data     extern E:\MPASM_MPLINK_PIC18_LT_Branch_3_42\pic18-lt\cxx-framework\src\traditional\proc\p18f97j60.asm
                 IPR3bits   0x000fa5       data     extern E:\MPASM_MPLINK_PIC18_LT_Branch_3_42\pic18-lt\cxx-framework\src\traditional\proc\p18f97j60.asm
                    IPVal   0x00066f       data     static C:\Users\LFRAD\Documents\CMS2Luc\ProjetsNettoyesCMSGit\ProjetCarteIO\project\MainDemoV1.c
                       JJ   0x00092c       data     extern C:\Users\LFRAD\Documents\CMS2Luc\ProjetsNettoyesCMSGit\ProjetCarteIO\project\MainDemoV1.c
                     JOUR   0x000b04       data     static C:\Users\LFRAD\Documents\CMS2Luc\ProjetsNettoyesCMSGit\ProjetCarteIO\project\MainDemoV1.c
                     JOUR   0x000b04       data     static C:\Users\LFRAD\Documents\CMS2Luc\ProjetsNettoyesCMSGit\ProjetCarteIO\project\MainDemoV1.c
                     LATA   0x000f89       data     extern E:\MPASM_MPLINK_PIC18_LT_Branch_3_42\pic18-lt\cxx-framework\src\traditional\proc\p18f97j60.asm
                 LATAbits   0x000f89       data     extern E:\MPASM_MPLINK_PIC18_LT_Branch_3_42\pic18-lt\cxx-framework\src\traditional\proc\p18f97j60.asm
                     LATB   0x000f8a       data     extern E:\MPASM_MPLINK_PIC18_LT_Branch_3_42\pic18-lt\cxx-framework\src\traditional\proc\p18f97j60.asm
                 LATBbits   0x000f8a       data     extern E:\MPASM_MPLINK_PIC18_LT_Branch_3_42\pic18-lt\cxx-framework\src\traditional\proc\p18f97j60.asm
                     LATC   0x000f8b       data     extern E:\MPASM_MPLINK_PIC18_LT_Branch_3_42\pic18-lt\cxx-framework\src\traditional\proc\p18f97j60.asm
                 LATCbits   0x000f8b       data     extern E:\MPASM_MPLINK_PIC18_LT_Branch_3_42\pic18-lt\cxx-framework\src\traditional\proc\p18f97j60.asm
                     LATD   0x000f8c       data     extern E:\MPASM_MPLINK_PIC18_LT_Branch_3_42\pic18-lt\cxx-framework\src\traditional\proc\p18f97j60.asm
                 LATDbits   0x000f8c       data     extern E:\MPASM_MPLINK_PIC18_LT_Branch_3_42\pic18-lt\cxx-framework\src\traditional\proc\p18f97j60.asm
                     LATE   0x000f8d       data     extern E:\MPASM_MPLINK_PIC18_LT_Branch_3_42\pic18-lt\cxx-framework\src\traditional\proc\p18f97j60.asm
                 LATEbits   0x000f8d       data     extern E:\MPASM_MPLINK_PIC18_LT_Branch_3_42\pic18-lt\cxx-framework\src\traditional\proc\p18f97j60.asm
                     LATF   0x000f8e       data     extern E:\MPASM_MPLINK_PIC18_LT_Branch_3_42\pic18-lt\cxx-framework\src\traditional\proc\p18f97j60.asm
                 LATFbits   0x000f8e       data     extern E:\MPASM_MPLINK_PIC18_LT_Branch_3_42\pic18-lt\cxx-framework\src\traditional\proc\p18f97j60.asm
                     LATG   0x000f8f       data     extern E:\MPASM_MPLINK_PIC18_LT_Branch_3_42\pic18-lt\cxx-framework\src\traditional\proc\p18f97j60.asm
                 LATGbits   0x000f8f       data     extern E:\MPASM_MPLINK_PIC18_LT_Branch_3_42\pic18-lt\cxx-framework\src\traditional\proc\p18f97j60.asm
                     LATH   0x000f90       data     extern E:\MPASM_MPLINK_PIC18_LT_Branch_3_42\pic18-lt\cxx-framework\src\traditional\proc\p18f97j60.asm
                 LATHbits   0x000f90       data     extern E:\MPASM_MPLINK_PIC18_LT_Branch_3_42\pic18-lt\cxx-framework\src\traditional\proc\p18f97j60.asm
                     LATJ   0x000f91       data     extern E:\MPASM_MPLINK_PIC18_LT_Branch_3_42\pic18-lt\cxx-framework\src\traditional\proc\p18f97j60.asm
                 LATJbits   0x000f91       data     extern E:\MPASM_MPLINK_PIC18_LT_Branch_3_42\pic18-lt\cxx-framework\src\traditional\proc\p18f97j60.asm
            LastPutSocket   0x0000fe       data     static C:\Users\LFRAD\Documents\CMS2Luc\ProjetsNettoyesCMSGit\ProjetCarteIO\project\UDP.c
                      Len   0x000b04       data     static C:\Users\LFRAD\Documents\CMS2Luc\ProjetsNettoyesCMSGit\ProjetCarteIO\project\DNS.c
                      Len   0x000b03       data     static C:\Users\LFRAD\Documents\CMS2Luc\ProjetsNettoyesCMSGit\ProjetCarteIO\project\DNS.c
                   MAADR1   0x000e84       data     extern E:\MPASM_MPLINK_PIC18_LT_Branch_3_42\pic18-lt\cxx-framework\src\traditional\proc\p18f97j60.asm
                   MAADR2   0x000e85       data     extern E:\MPASM_MPLINK_PIC18_LT_Branch_3_42\pic18-lt\cxx-framework\src\traditional\proc\p18f97j60.asm
                   MAADR3   0x000e82       data     extern E:\MPASM_MPLINK_PIC18_LT_Branch_3_42\pic18-lt\cxx-framework\src\traditional\proc\p18f97j60.asm
                   MAADR4   0x000e83       data     extern E:\MPASM_MPLINK_PIC18_LT_Branch_3_42\pic18-lt\cxx-framework\src\traditional\proc\p18f97j60.asm
                   MAADR5   0x000e80       data     extern E:\MPASM_MPLINK_PIC18_LT_Branch_3_42\pic18-lt\cxx-framework\src\traditional\proc\p18f97j60.asm
                   MAADR6   0x000e81       data     extern E:\MPASM_MPLINK_PIC18_LT_Branch_3_42\pic18-lt\cxx-framework\src\traditional\proc\p18f97j60.asm
                  MABBIPG   0x000ea4       data     extern E:\MPASM_MPLINK_PIC18_LT_Branch_3_42\pic18-lt\cxx-framework\src\traditional\proc\p18f97j60.asm
              MABBIPGbits   0x000ea4       data     extern E:\MPASM_MPLINK_PIC18_LT_Branch_3_42\pic18-lt\cxx-framework\src\traditional\proc\p18f97j60.asm
                  MACAddr   0x0006f8       data     static C:\Users\LFRAD\Documents\CMS2Luc\ProjetsNettoyesCMSGit\ProjetCarteIO\project\ARP.c
                   MACON1   0x000ea0       data     extern E:\MPASM_MPLINK_PIC18_LT_Branch_3_42\pic18-lt\cxx-framework\src\traditional\proc\p18f97j60.asm
               MACON1bits   0x000ea0       data     extern E:\MPASM_MPLINK_PIC18_LT_Branch_3_42\pic18-lt\cxx-framework\src\traditional\proc\p18f97j60.asm
                   MACON3   0x000ea2       data     extern E:\MPASM_MPLINK_PIC18_LT_Branch_3_42\pic18-lt\cxx-framework\src\traditional\proc\p18f97j60.asm
               MACON3bits   0x000ea2       data     extern E:\MPASM_MPLINK_PIC18_LT_Branch_3_42\pic18-lt\cxx-framework\src\traditional\proc\p18f97j60.asm
                   MACON4   0x000ea3       data     extern E:\MPASM_MPLINK_PIC18_LT_Branch_3_42\pic18-lt\cxx-framework\src\traditional\proc\p18f97j60.asm
               MACON4bits   0x000ea3       data     extern E:\MPASM_MPLINK_PIC18_LT_Branch_3_42\pic18-lt\cxx-framework\src\traditional\proc\p18f97j60.asm
                    MAIPG   0x000ea6       data     extern E:\MPASM_MPLINK_PIC18_LT_Branch_3_42\pic18-lt\cxx-framework\src\traditional\proc\p18f97j60.asm
                   MAIPGH   0x000ea7       data     extern E:\MPASM_MPLINK_PIC18_LT_Branch_3_42\pic18-lt\cxx-framework\src\traditional\proc\p18f97j60.asm
                   MAIPGL   0x000ea6       data     extern E:\MPASM_MPLINK_PIC18_LT_Branch_3_42\pic18-lt\cxx-framework\src\traditional\proc\p18f97j60.asm
                  MAJBLOC   0x000669       data     extern C:\Users\LFRAD\Documents\CMS2Luc\ProjetsNettoyesCMSGit\ProjetCarteIO\project\MainDemoV1.c
                   MAMXFL   0x000eaa       data     extern E:\MPASM_MPLINK_PIC18_LT_Branch_3_42\pic18-lt\cxx-framework\src\traditional\proc\p18f97j60.asm
                  MAMXFLH   0x000eab       data     extern E:\MPASM_MPLINK_PIC18_LT_Branch_3_42\pic18-lt\cxx-framework\src\traditional\proc\p18f97j60.asm
                  MAMXFLL   0x000eaa       data     extern E:\MPASM_MPLINK_PIC18_LT_Branch_3_42\pic18-lt\cxx-framework\src\traditional\proc\p18f97j60.asm
                   MEMCON   0x000f9c       data     extern E:\MPASM_MPLINK_PIC18_LT_Branch_3_42\pic18-lt\cxx-framework\src\traditional\proc\p18f97j60.asm
               MEMCONbits   0x000f9c       data     extern E:\MPASM_MPLINK_PIC18_LT_Branch_3_42\pic18-lt\cxx-framework\src\traditional\proc\p18f97j60.asm
                    MICMD   0x000eb2       data     extern E:\MPASM_MPLINK_PIC18_LT_Branch_3_42\pic18-lt\cxx-framework\src\traditional\proc\p18f97j60.asm
                MICMDbits   0x000eb2       data     extern E:\MPASM_MPLINK_PIC18_LT_Branch_3_42\pic18-lt\cxx-framework\src\traditional\proc\p18f97j60.asm
                   MINUTE   0x000b01       data     static C:\Users\LFRAD\Documents\CMS2Luc\ProjetsNettoyesCMSGit\ProjetCarteIO\project\MainDemoV1.c
                   MINUTE   0x000b01       data     static C:\Users\LFRAD\Documents\CMS2Luc\ProjetsNettoyesCMSGit\ProjetCarteIO\project\MainDemoV1.c
                     MIRD   0x000eb8       data     extern E:\MPASM_MPLINK_PIC18_LT_Branch_3_42\pic18-lt\cxx-framework\src\traditional\proc\p18f97j60.asm
                    MIRDH   0x000eb9       data     extern E:\MPASM_MPLINK_PIC18_LT_Branch_3_42\pic18-lt\cxx-framework\src\traditional\proc\p18f97j60.asm
                    MIRDL   0x000eb8       data     extern E:\MPASM_MPLINK_PIC18_LT_Branch_3_42\pic18-lt\cxx-framework\src\traditional\proc\p18f97j60.asm
                 MIREGADR   0x000eb4       data     extern E:\MPASM_MPLINK_PIC18_LT_Branch_3_42\pic18-lt\cxx-framework\src\traditional\proc\p18f97j60.asm
                   MISTAT   0x000e8a       data     extern E:\MPASM_MPLINK_PIC18_LT_Branch_3_42\pic18-lt\cxx-framework\src\traditional\proc\p18f97j60.asm
               MISTATbits   0x000e8a       data     extern E:\MPASM_MPLINK_PIC18_LT_Branch_3_42\pic18-lt\cxx-framework\src\traditional\proc\p18f97j60.asm
                     MIWR   0x000eb6       data     extern E:\MPASM_MPLINK_PIC18_LT_Branch_3_42\pic18-lt\cxx-framework\src\traditional\proc\p18f97j60.asm
                    MIWRH   0x000eb7       data     extern E:\MPASM_MPLINK_PIC18_LT_Branch_3_42\pic18-lt\cxx-framework\src\traditional\proc\p18f97j60.asm
                    MIWRL   0x000eb6       data     extern E:\MPASM_MPLINK_PIC18_LT_Branch_3_42\pic18-lt\cxx-framework\src\traditional\proc\p18f97j60.asm
                       MM   0x00092e       data     extern C:\Users\LFRAD\Documents\CMS2Luc\ProjetsNettoyesCMSGit\ProjetCarteIO\project\MainDemoV1.c
                MODERAPID   0x000a3a       data     extern C:\Users\LFRAD\Documents\CMS2Luc\ProjetsNettoyesCMSGit\ProjetCarteIO\project\MainDemoV1.c
                     MOIS   0x000b03       data     static C:\Users\LFRAD\Documents\CMS2Luc\ProjetsNettoyesCMSGit\ProjetCarteIO\project\MainDemoV1.c
                     MOIS   0x000b03       data     static C:\Users\LFRAD\Documents\CMS2Luc\ProjetsNettoyesCMSGit\ProjetCarteIO\project\MainDemoV1.c
                      Mil   0x000b00       data     static C:\Users\LFRAD\Documents\CMS2Luc\ProjetsNettoyesCMSGit\ProjetCarteIO\project\GenericTCPClient.c
                      Mil   0x000b00       data     static C:\Users\LFRAD\Documents\CMS2Luc\ProjetsNettoyesCMSGit\ProjetCarteIO\project\MainDemoV1.c
                      Mil   0x000b00       data     static C:\Users\LFRAD\Documents\CMS2Luc\ProjetsNettoyesCMSGit\ProjetCarteIO\project\MainDemoV1.c
                 MySocket   0x000e6b       data     static C:\Users\LFRAD\Documents\CMS2Luc\ProjetsNettoyesCMSGit\ProjetCarteIO\project\DNS.c
                 MySocket   0x0008f1       data     static C:\Users\LFRAD\Documents\CMS2Luc\ProjetsNettoyesCMSGit\ProjetCarteIO\project\GenericTCPClient.c
                 MySocket   0x000e69       data     static C:\Users\LFRAD\Documents\CMS2Luc\ProjetsNettoyesCMSGit\ProjetCarteIO\project\GenericTCPClient.c
                 MySocket   0x0000f3       data     extern C:\Users\LFRAD\Documents\CMS2Luc\ProjetsNettoyesCMSGit\ProjetCarteIO\project\GenericTCPServer.c
                 MySocket   0x0006cf       data     static C:\Users\LFRAD\Documents\CMS2Luc\ProjetsNettoyesCMSGit\ProjetCarteIO\project\MainDemoV1.c
                    MyTCB   0x000702       data     static C:\Users\LFRAD\Documents\CMS2Luc\ProjetsNettoyesCMSGit\ProjetCarteIO\project\TCP.c
                MyTCBStub   0x000729       data     static C:\Users\LFRAD\Documents\CMS2Luc\ProjetsNettoyesCMSGit\ProjetCarteIO\project\TCP.c
                    NBCOM   0x000a71       data     extern C:\Users\LFRAD\Documents\CMS2Luc\ProjetsNettoyesCMSGit\ProjetCarteIO\project\MainDemoV1.c
       NBRECAPTEURS_CABLE   0x000e3d       data     extern C:\Users\LFRAD\Documents\CMS2Luc\ProjetsNettoyesCMSGit\ProjetCarteIO\project\MainDemoV1.c
              NORECEPTION   0x000a6b       data     extern C:\Users\LFRAD\Documents\CMS2Luc\ProjetsNettoyesCMSGit\ProjetCarteIO\project\MainDemoV1.c
                  NUMDNS1   0x00089c       data     extern C:\Users\LFRAD\Documents\CMS2Luc\ProjetsNettoyesCMSGit\ProjetCarteIO\project\MainDemoV1.c
                  NUMDNS2   0x000898       data     extern C:\Users\LFRAD\Documents\CMS2Luc\ProjetsNettoyesCMSGit\ProjetCarteIO\project\MainDemoV1.c
                  NUMDNS3   0x000894       data     extern C:\Users\LFRAD\Documents\CMS2Luc\ProjetsNettoyesCMSGit\ProjetCarteIO\project\MainDemoV1.c
                  NUMDNS4   0x000890       data     extern C:\Users\LFRAD\Documents\CMS2Luc\ProjetsNettoyesCMSGit\ProjetCarteIO\project\MainDemoV1.c
                   NUMIP1   0x00088c       data     extern C:\Users\LFRAD\Documents\CMS2Luc\ProjetsNettoyesCMSGit\ProjetCarteIO\project\MainDemoV1.c
                   NUMIP2   0x000888       data     extern C:\Users\LFRAD\Documents\CMS2Luc\ProjetsNettoyesCMSGit\ProjetCarteIO\project\MainDemoV1.c
                   NUMIP3   0x000884       data     extern C:\Users\LFRAD\Documents\CMS2Luc\ProjetsNettoyesCMSGit\ProjetCarteIO\project\MainDemoV1.c
                   NUMIP4   0x000880       data     extern C:\Users\LFRAD\Documents\CMS2Luc\ProjetsNettoyesCMSGit\ProjetCarteIO\project\MainDemoV1.c
                NUMPASSE1   0x0008ac       data     extern C:\Users\LFRAD\Documents\CMS2Luc\ProjetsNettoyesCMSGit\ProjetCarteIO\project\MainDemoV1.c
                NUMPASSE2   0x0008a8       data     extern C:\Users\LFRAD\Documents\CMS2Luc\ProjetsNettoyesCMSGit\ProjetCarteIO\project\MainDemoV1.c
                NUMPASSE3   0x0008a4       data     extern C:\Users\LFRAD\Documents\CMS2Luc\ProjetsNettoyesCMSGit\ProjetCarteIO\project\MainDemoV1.c
                NUMPASSE4   0x0008a0       data     extern C:\Users\LFRAD\Documents\CMS2Luc\ProjetsNettoyesCMSGit\ProjetCarteIO\project\MainDemoV1.c
                     Name   0x000a2d       data     static C:\Users\LFRAD\Documents\CMS2Luc\ProjetsNettoyesCMSGit\ProjetCarteIO\project\Helpers.c
                  Nchamps   0x000695       data     static C:\Users\LFRAD\Documents\CMS2Luc\ProjetsNettoyesCMSGit\ProjetCarteIO\project\MainDemoV1.c
          NewRXRDLocation   0x000b25       data     static C:\Users\LFRAD\Documents\CMS2Luc\ProjetsNettoyesCMSGit\ProjetCarteIO\project\ETH97J60.c
       NextPacketLocation   0x000a72       data     static C:\Users\LFRAD\Documents\CMS2Luc\ProjetsNettoyesCMSGit\ProjetCarteIO\project\ETH97J60.c
                 NextPort   0x0004cb       data     static C:\Users\LFRAD\Documents\CMS2Luc\ProjetsNettoyesCMSGit\ProjetCarteIO\project\UDP.c
                 NextPort   0x000700       data     static C:\Users\LFRAD\Documents\CMS2Luc\ProjetsNettoyesCMSGit\ProjetCarteIO\project\TCP.c
                    Npage   0x000694       data     static C:\Users\LFRAD\Documents\CMS2Luc\ProjetsNettoyesCMSGit\ProjetCarteIO\project\MainDemoV1.c
                  NumeroH   0x0006c0       data     static C:\Users\LFRAD\Documents\CMS2Luc\ProjetsNettoyesCMSGit\ProjetCarteIO\project\MainDemoV1.c
                  NumeroH   0x0006bb       data     static C:\Users\LFRAD\Documents\CMS2Luc\ProjetsNettoyesCMSGit\ProjetCarteIO\project\MainDemoV1.c
                   OSCCON   0x000fd3       data     extern E:\MPASM_MPLINK_PIC18_LT_Branch_3_42\pic18-lt\cxx-framework\src\traditional\proc\p18f97j60.asm
               OSCCONbits   0x000fd3       data     extern E:\MPASM_MPLINK_PIC18_LT_Branch_3_42\pic18-lt\cxx-framework\src\traditional\proc\p18f97j60.asm
                  OSCTUNE   0x000f9b       data     extern E:\MPASM_MPLINK_PIC18_LT_Branch_3_42\pic18-lt\cxx-framework\src\traditional\proc\p18f97j60.asm
              OSCTUNEbits   0x000f9b       data     extern E:\MPASM_MPLINK_PIC18_LT_Branch_3_42\pic18-lt\cxx-framework\src\traditional\proc\p18f97j60.asm
              OUVERTUREIP   0x00087d       data     extern C:\Users\LFRAD\Documents\CMS2Luc\ProjetsNettoyesCMSGit\ProjetCarteIO\project\MainDemoV1.c
                   Offset   0x0005f8       data     static C:\Users\LFRAD\Documents\CMS2Luc\ProjetsNettoyesCMSGit\ProjetCarteIO\project\IP.c
PASDEDEMANDECONNECTIONTCPIP   0x00087e       data     extern C:\Users\LFRAD\Documents\CMS2Luc\ProjetsNettoyesCMSGit\ProjetCarteIO\project\MainDemoV1.c
                       PC   0x000ff9       data     extern E:\MPASM_MPLINK_PIC18_LT_Branch_3_42\pic18-lt\cxx-framework\src\traditional\proc\p18f97j60.asm
                      PCL   0x000ff9       data     extern E:\MPASM_MPLINK_PIC18_LT_Branch_3_42\pic18-lt\cxx-framework\src\traditional\proc\p18f97j60.asm
                   PCLATH   0x000ffa       data     extern E:\MPASM_MPLINK_PIC18_LT_Branch_3_42\pic18-lt\cxx-framework\src\traditional\proc\p18f97j60.asm
                   PCLATU   0x000ffb       data     extern E:\MPASM_MPLINK_PIC18_LT_Branch_3_42\pic18-lt\cxx-framework\src\traditional\proc\p18f97j60.asm
                     PIE1   0x000f9d       data     extern E:\MPASM_MPLINK_PIC18_LT_Branch_3_42\pic18-lt\cxx-framework\src\traditional\proc\p18f97j60.asm
                 PIE1bits   0x000f9d       data     extern E:\MPASM_MPLINK_PIC18_LT_Branch_3_42\pic18-lt\cxx-framework\src\traditional\proc\p18f97j60.asm
                     PIE2   0x000fa0       data     extern E:\MPASM_MPLINK_PIC18_LT_Branch_3_42\pic18-lt\cxx-framework\src\traditional\proc\p18f97j60.asm
                 PIE2bits   0x000fa0       data     extern E:\MPASM_MPLINK_PIC18_LT_Branch_3_42\pic18-lt\cxx-framework\src\traditional\proc\p18f97j60.asm
                     PIE3   0x000fa3       data     extern E:\MPASM_MPLINK_PIC18_LT_Branch_3_42\pic18-lt\cxx-framework\src\traditional\proc\p18f97j60.asm
                 PIE3bits   0x000fa3       data     extern E:\MPASM_MPLINK_PIC18_LT_Branch_3_42\pic18-lt\cxx-framework\src\traditional\proc\p18f97j60.asm
                     PIR1   0x000f9e       data     extern E:\MPASM_MPLINK_PIC18_LT_Branch_3_42\pic18-lt\cxx-framework\src\traditional\proc\p18f97j60.asm
                 PIR1bits   0x000f9e       data     extern E:\MPASM_MPLINK_PIC18_LT_Branch_3_42\pic18-lt\cxx-framework\src\traditional\proc\p18f97j60.asm
                     PIR2   0x000fa1       data     extern E:\MPASM_MPLINK_PIC18_LT_Branch_3_42\pic18-lt\cxx-framework\src\traditional\proc\p18f97j60.asm
                 PIR2bits   0x000fa1       data     extern E:\MPASM_MPLINK_PIC18_LT_Branch_3_42\pic18-lt\cxx-framework\src\traditional\proc\p18f97j60.asm
                     PIR3   0x000fa4       data     extern E:\MPASM_MPLINK_PIC18_LT_Branch_3_42\pic18-lt\cxx-framework\src\traditional\proc\p18f97j60.asm
                 PIR3bits   0x000fa4       data     extern E:\MPASM_MPLINK_PIC18_LT_Branch_3_42\pic18-lt\cxx-framework\src\traditional\proc\p18f97j60.asm
                   PLUSW0   0x000feb       data     extern E:\MPASM_MPLINK_PIC18_LT_Branch_3_42\pic18-lt\cxx-framework\src\traditional\proc\p18f97j60.asm
                   PLUSW1   0x000fe3       data     extern E:\MPASM_MPLINK_PIC18_LT_Branch_3_42\pic18-lt\cxx-framework\src\traditional\proc\p18f97j60.asm
                   PLUSW2   0x000fdb       data     extern E:\MPASM_MPLINK_PIC18_LT_Branch_3_42\pic18-lt\cxx-framework\src\traditional\proc\p18f97j60.asm
              POINT_ROSEE   0x0005aa       data     extern C:\Users\LFRAD\Documents\CMS2Luc\ProjetsNettoyesCMSGit\ProjetCarteIO\project\MainDemoV1.c
                    PORTA   0x000f80       data     extern E:\MPASM_MPLINK_PIC18_LT_Branch_3_42\pic18-lt\cxx-framework\src\traditional\proc\p18f97j60.asm
                PORTAbits   0x000f80       data     extern E:\MPASM_MPLINK_PIC18_LT_Branch_3_42\pic18-lt\cxx-framework\src\traditional\proc\p18f97j60.asm
                    PORTB   0x000f81       data     extern E:\MPASM_MPLINK_PIC18_LT_Branch_3_42\pic18-lt\cxx-framework\src\traditional\proc\p18f97j60.asm
                PORTBbits   0x000f81       data     extern E:\MPASM_MPLINK_PIC18_LT_Branch_3_42\pic18-lt\cxx-framework\src\traditional\proc\p18f97j60.asm
                    PORTC   0x000f82       data     extern E:\MPASM_MPLINK_PIC18_LT_Branch_3_42\pic18-lt\cxx-framework\src\traditional\proc\p18f97j60.asm
                PORTCbits   0x000f82       data     extern E:\MPASM_MPLINK_PIC18_LT_Branch_3_42\pic18-lt\cxx-framework\src\traditional\proc\p18f97j60.asm
                    PORTD   0x000f83       data     extern E:\MPASM_MPLINK_PIC18_LT_Branch_3_42\pic18-lt\cxx-framework\src\traditional\proc\p18f97j60.asm
                PORTDbits   0x000f83       data     extern E:\MPASM_MPLINK_PIC18_LT_Branch_3_42\pic18-lt\cxx-framework\src\traditional\proc\p18f97j60.asm
                    PORTE   0x000f84       data     extern E:\MPASM_MPLINK_PIC18_LT_Branch_3_42\pic18-lt\cxx-framework\src\traditional\proc\p18f97j60.asm
                PORTEbits   0x000f84       data     extern E:\MPASM_MPLINK_PIC18_LT_Branch_3_42\pic18-lt\cxx-framework\src\traditional\proc\p18f97j60.asm
                    PORTF   0x000f85       data     extern E:\MPASM_MPLINK_PIC18_LT_Branch_3_42\pic18-lt\cxx-framework\src\traditional\proc\p18f97j60.asm
                PORTFbits   0x000f85       data     extern E:\MPASM_MPLINK_PIC18_LT_Branch_3_42\pic18-lt\cxx-framework\src\traditional\proc\p18f97j60.asm
                    PORTG   0x000f86       data     extern E:\MPASM_MPLINK_PIC18_LT_Branch_3_42\pic18-lt\cxx-framework\src\traditional\proc\p18f97j60.asm
                PORTGbits   0x000f86       data     extern E:\MPASM_MPLINK_PIC18_LT_Branch_3_42\pic18-lt\cxx-framework\src\traditional\proc\p18f97j60.asm
                    PORTH   0x000f87       data     extern E:\MPASM_MPLINK_PIC18_LT_Branch_3_42\pic18-lt\cxx-framework\src\traditional\proc\p18f97j60.asm
                PORTHbits   0x000f87       data     extern E:\MPASM_MPLINK_PIC18_LT_Branch_3_42\pic18-lt\cxx-framework\src\traditional\proc\p18f97j60.asm
                    PORTJ   0x000f88       data     extern E:\MPASM_MPLINK_PIC18_LT_Branch_3_42\pic18-lt\cxx-framework\src\traditional\proc\p18f97j60.asm
                PORTJbits   0x000f88       data     extern E:\MPASM_MPLINK_PIC18_LT_Branch_3_42\pic18-lt\cxx-framework\src\traditional\proc\p18f97j60.asm
                      POS   0x000904       data     extern C:\Users\LFRAD\Documents\CMS2Luc\ProjetsNettoyesCMSGit\ProjetCarteIO\project\MainDemoV1.c
                 POSTDEC0   0x000fed       data     extern E:\MPASM_MPLINK_PIC18_LT_Branch_3_42\pic18-lt\cxx-framework\src\traditional\proc\p18f97j60.asm
                 POSTDEC1   0x000fe5       data     extern E:\MPASM_MPLINK_PIC18_LT_Branch_3_42\pic18-lt\cxx-framework\src\traditional\proc\p18f97j60.asm
                 POSTDEC2   0x000fdd       data     extern E:\MPASM_MPLINK_PIC18_LT_Branch_3_42\pic18-lt\cxx-framework\src\traditional\proc\p18f97j60.asm
                 POSTINC0   0x000fee       data     extern E:\MPASM_MPLINK_PIC18_LT_Branch_3_42\pic18-lt\cxx-framework\src\traditional\proc\p18f97j60.asm
                 POSTINC1   0x000fe6       data     extern E:\MPASM_MPLINK_PIC18_LT_Branch_3_42\pic18-lt\cxx-framework\src\traditional\proc\p18f97j60.asm
                 POSTINC2   0x000fde       data     extern E:\MPASM_MPLINK_PIC18_LT_Branch_3_42\pic18-lt\cxx-framework\src\traditional\proc\p18f97j60.asm
                      PR2   0x000fcb       data     extern E:\MPASM_MPLINK_PIC18_LT_Branch_3_42\pic18-lt\cxx-framework\src\traditional\proc\p18f97j60.asm
                      PR4   0x000f77       data     extern E:\MPASM_MPLINK_PIC18_LT_Branch_3_42\pic18-lt\cxx-framework\src\traditional\proc\p18f97j60.asm
                  PREINC0   0x000fec       data     extern E:\MPASM_MPLINK_PIC18_LT_Branch_3_42\pic18-lt\cxx-framework\src\traditional\proc\p18f97j60.asm
                  PREINC1   0x000fe4       data     extern E:\MPASM_MPLINK_PIC18_LT_Branch_3_42\pic18-lt\cxx-framework\src\traditional\proc\p18f97j60.asm
                  PREINC2   0x000fdc       data     extern E:\MPASM_MPLINK_PIC18_LT_Branch_3_42\pic18-lt\cxx-framework\src\traditional\proc\p18f97j60.asm
            PRESENCE_220V   0x0005de       data     extern C:\Users\LFRAD\Documents\CMS2Luc\ProjetsNettoyesCMSGit\ProjetCarteIO\project\MainDemoV1.c
             PRESENCE_48V   0x0005e4       data     extern C:\Users\LFRAD\Documents\CMS2Luc\ProjetsNettoyesCMSGit\ProjetCarteIO\project\MainDemoV1.c
                     PROD   0x000ff3       data     extern E:\MPASM_MPLINK_PIC18_LT_Branch_3_42\pic18-lt\cxx-framework\src\traditional\proc\p18f97j60.asm
                    PRODH   0x000ff4       data     extern E:\MPASM_MPLINK_PIC18_LT_Branch_3_42\pic18-lt\cxx-framework\src\traditional\proc\p18f97j60.asm
                    PRODL   0x000ff3       data     extern E:\MPASM_MPLINK_PIC18_LT_Branch_3_42\pic18-lt\cxx-framework\src\traditional\proc\p18f97j60.asm
                   PSPCON   0x000fb0       data     extern E:\MPASM_MPLINK_PIC18_LT_Branch_3_42\pic18-lt\cxx-framework\src\traditional\proc\p18f97j60.asm
               PSPCONbits   0x000fb0       data     extern E:\MPASM_MPLINK_PIC18_LT_Branch_3_42\pic18-lt\cxx-framework\src\traditional\proc\p18f97j60.asm
              P_RESERVOIR   0x00057d       data     extern C:\Users\LFRAD\Documents\CMS2Luc\ProjetsNettoyesCMSGit\ProjetCarteIO\project\MainDemoV1.c
                P_SECOURS   0x00059b       data     extern C:\Users\LFRAD\Documents\CMS2Luc\ProjetsNettoyesCMSGit\ProjetCarteIO\project\MainDemoV1.c
                 P_SORTIE   0x00058c       data     extern C:\Users\LFRAD\Documents\CMS2Luc\ProjetsNettoyesCMSGit\ProjetCarteIO\project\MainDemoV1.c
                 PageSize   0x000b0d       data     static C:\Users\LFRAD\Documents\CMS2Luc\ProjetsNettoyesCMSGit\ProjetCarteIO\project\MainDemoV1.c
                Precision   0x0006d4       data     static C:\Users\LFRAD\Documents\CMS2Luc\ProjetsNettoyesCMSGit\ProjetCarteIO\project\MainDemoV1.c
                Precision   0x0008fa       data     static C:\Users\LFRAD\Documents\CMS2Luc\ProjetsNettoyesCMSGit\ProjetCarteIO\project\GenericTCPClient.c
                Precision   0x000677       data     static C:\Users\LFRAD\Documents\CMS2Luc\ProjetsNettoyesCMSGit\ProjetCarteIO\project\MainDemoV1.c
                  Printed   0x000b05       data     static C:\Users\LFRAD\Documents\CMS2Luc\ProjetsNettoyesCMSGit\ProjetCarteIO\project\Helpers.c
                        R   0x0006ae       data     static C:\Users\LFRAD\Documents\CMS2Luc\ProjetsNettoyesCMSGit\ProjetCarteIO\project\MainDemoV1.c
                     RCON   0x000fd0       data     extern E:\MPASM_MPLINK_PIC18_LT_Branch_3_42\pic18-lt\cxx-framework\src\traditional\proc\p18f97j60.asm
                 RCONbits   0x000fd0       data     extern E:\MPASM_MPLINK_PIC18_LT_Branch_3_42\pic18-lt\cxx-framework\src\traditional\proc\p18f97j60.asm
                    RCREG   0x000fae       data     extern E:\MPASM_MPLINK_PIC18_LT_Branch_3_42\pic18-lt\cxx-framework\src\traditional\proc\p18f97j60.asm
                   RCREG1   0x000fae       data     extern E:\MPASM_MPLINK_PIC18_LT_Branch_3_42\pic18-lt\cxx-framework\src\traditional\proc\p18f97j60.asm
                   RCREG2   0x000f6e       data     extern E:\MPASM_MPLINK_PIC18_LT_Branch_3_42\pic18-lt\cxx-framework\src\traditional\proc\p18f97j60.asm
                    RCSTA   0x000fab       data     extern E:\MPASM_MPLINK_PIC18_LT_Branch_3_42\pic18-lt\cxx-framework\src\traditional\proc\p18f97j60.asm
                   RCSTA1   0x000fab       data     extern E:\MPASM_MPLINK_PIC18_LT_Branch_3_42\pic18-lt\cxx-framework\src\traditional\proc\p18f97j60.asm
               RCSTA1bits   0x000fab       data     extern E:\MPASM_MPLINK_PIC18_LT_Branch_3_42\pic18-lt\cxx-framework\src\traditional\proc\p18f97j60.asm
                   RCSTA2   0x000f6b       data     extern E:\MPASM_MPLINK_PIC18_LT_Branch_3_42\pic18-lt\cxx-framework\src\traditional\proc\p18f97j60.asm
               RCSTA2bits   0x000f6b       data     extern E:\MPASM_MPLINK_PIC18_LT_Branch_3_42\pic18-lt\cxx-framework\src\traditional\proc\p18f97j60.asm
                RCSTAbits   0x000fab       data     extern E:\MPASM_MPLINK_PIC18_LT_Branch_3_42\pic18-lt\cxx-framework\src\traditional\proc\p18f97j60.asm
                   RDSave   0x000b18       data     static C:\Users\LFRAD\Documents\CMS2Luc\ProjetsNettoyesCMSGit\ProjetCarteIO\project\ETH97J60.c
            REA_DESACTIVE   0x0000e2       data     extern C:\Users\LFRAD\Documents\CMS2Luc\ProjetsNettoyesCMSGit\ProjetCarteIO\project\MainDemoV1.c
                 REBOOTIP   0x0009e5       data     extern C:\Users\LFRAD\Documents\CMS2Luc\ProjetsNettoyesCMSGit\ProjetCarteIO\project\MainDemoV1.c
                      ROB   0x000e4b       data     extern C:\Users\LFRAD\Documents\CMS2Luc\ProjetsNettoyesCMSGit\ProjetCarteIO\project\MainDemoV1.c
                   ReadPT   0x000b25       data     static C:\Users\LFRAD\Documents\CMS2Luc\ProjetsNettoyesCMSGit\ProjetCarteIO\project\ETH97J60.c
                   ReadPT   0x000b29       data     static C:\Users\LFRAD\Documents\CMS2Luc\ProjetsNettoyesCMSGit\ProjetCarteIO\project\ETH97J60.c
                 ReadSave   0x000b2b       data     static C:\Users\LFRAD\Documents\CMS2Luc\ProjetsNettoyesCMSGit\ProjetCarteIO\project\ETH97J60.c
               RecordType   0x0007d4       data     static C:\Users\LFRAD\Documents\CMS2Luc\ProjetsNettoyesCMSGit\ProjetCarteIO\project\DNS.c
                 Register   0x000aa4       data     static C:\Users\LFRAD\Documents\CMS2Luc\ProjetsNettoyesCMSGit\ProjetCarteIO\project\ETH97J60.c
                 Register   0x000aa5       data     static C:\Users\LFRAD\Documents\CMS2Luc\ProjetsNettoyesCMSGit\ProjetCarteIO\project\ETH97J60.c
               RemoteInfo   0x000753       data     static C:\Users\LFRAD\Documents\CMS2Luc\ProjetsNettoyesCMSGit\ProjetCarteIO\project\TCP.c
             ResolvedInfo   0x0007d5       data     static C:\Users\LFRAD\Documents\CMS2Luc\ProjetsNettoyesCMSGit\ProjetCarteIO\project\DNS.c
                   Result   0x000b14       data     static C:\Users\LFRAD\Documents\CMS2Luc\ProjetsNettoyesCMSGit\ProjetCarteIO\project\ETH97J60.c
                 RightLen   0x000b02       data     static C:\Users\LFRAD\Documents\CMS2Luc\ProjetsNettoyesCMSGit\ProjetCarteIO\project\TCP.c
                 RightPtr   0x000b00       data     static C:\Users\LFRAD\Documents\CMS2Luc\ProjetsNettoyesCMSGit\ProjetCarteIO\project\DNS.c
                 RightPtr   0x000b00       data     static C:\Users\LFRAD\Documents\CMS2Luc\ProjetsNettoyesCMSGit\ProjetCarteIO\project\DNS.c
                  SALARME   0x000c08       data     static C:\Users\LFRAD\Documents\CMS2Luc\ProjetsNettoyesCMSGit\ProjetCarteIO\project\MainDemoV1.c
                  SECONDE   0x000b02       data     static C:\Users\LFRAD\Documents\CMS2Luc\ProjetsNettoyesCMSGit\ProjetCarteIO\project\MainDemoV1.c
                  SECONDE   0x000b02       data     static C:\Users\LFRAD\Documents\CMS2Luc\ProjetsNettoyesCMSGit\ProjetCarteIO\project\MainDemoV1.c
                 SERVERIP   0x0000e3       data     extern C:\Users\LFRAD\Documents\CMS2Luc\ProjetsNettoyesCMSGit\ProjetCarteIO\project\MainDemoV1.c
                    SEUIL   0x000955       data     extern C:\Users\LFRAD\Documents\CMS2Luc\ProjetsNettoyesCMSGit\ProjetCarteIO\project\MainDemoV1.c
                   SEUIL2   0x000972       data     extern C:\Users\LFRAD\Documents\CMS2Luc\ProjetsNettoyesCMSGit\ProjetCarteIO\project\MainDemoV1.c
                     SIGN   0x000000       data     extern E:\MPASM_MPLINK_PIC18_LT_Branch_3_42\pic18-lt\cxx-framework\src\traditional\math\cmath18.asm
                    SPBRG   0x000faf       data     extern E:\MPASM_MPLINK_PIC18_LT_Branch_3_42\pic18-lt\cxx-framework\src\traditional\proc\p18f97j60.asm
                   SPBRG1   0x000faf       data     extern E:\MPASM_MPLINK_PIC18_LT_Branch_3_42\pic18-lt\cxx-framework\src\traditional\proc\p18f97j60.asm
                   SPBRG2   0x000f6f       data     extern E:\MPASM_MPLINK_PIC18_LT_Branch_3_42\pic18-lt\cxx-framework\src\traditional\proc\p18f97j60.asm
                   SPBRGH   0x000f7f       data     extern E:\MPASM_MPLINK_PIC18_LT_Branch_3_42\pic18-lt\cxx-framework\src\traditional\proc\p18f97j60.asm
                  SPBRGH1   0x000f7f       data     extern E:\MPASM_MPLINK_PIC18_LT_Branch_3_42\pic18-lt\cxx-framework\src\traditional\proc\p18f97j60.asm
                  SPBRGH2   0x000f7d       data     extern E:\MPASM_MPLINK_PIC18_LT_Branch_3_42\pic18-lt\cxx-framework\src\traditional\proc\p18f97j60.asm
                    SPEED   0x000b00       data     static C:\Users\LFRAD\Documents\CMS2Luc\ProjetsNettoyesCMSGit\ProjetCarteIO\project\MainDemoV1.c
                  SSP1ADD   0x000fc8       data     extern E:\MPASM_MPLINK_PIC18_LT_Branch_3_42\pic18-lt\cxx-framework\src\traditional\proc\p18f97j60.asm
                  SSP1BUF   0x000fc9       data     extern E:\MPASM_MPLINK_PIC18_LT_Branch_3_42\pic18-lt\cxx-framework\src\traditional\proc\p18f97j60.asm
                 SSP1CON1   0x000fc6       data     extern E:\MPASM_MPLINK_PIC18_LT_Branch_3_42\pic18-lt\cxx-framework\src\traditional\proc\p18f97j60.asm
             SSP1CON1bits   0x000fc6       data     extern E:\MPASM_MPLINK_PIC18_LT_Branch_3_42\pic18-lt\cxx-framework\src\traditional\proc\p18f97j60.asm
                 SSP1CON2   0x000fc5       data     extern E:\MPASM_MPLINK_PIC18_LT_Branch_3_42\pic18-lt\cxx-framework\src\traditional\proc\p18f97j60.asm
             SSP1CON2bits   0x000fc5       data     extern E:\MPASM_MPLINK_PIC18_LT_Branch_3_42\pic18-lt\cxx-framework\src\traditional\proc\p18f97j60.asm
                 SSP1STAT   0x000fc7       data     extern E:\MPASM_MPLINK_PIC18_LT_Branch_3_42\pic18-lt\cxx-framework\src\traditional\proc\p18f97j60.asm
             SSP1STATbits   0x000fc7       data     extern E:\MPASM_MPLINK_PIC18_LT_Branch_3_42\pic18-lt\cxx-framework\src\traditional\proc\p18f97j60.asm
                  SSP2ADD   0x000f65       data     extern E:\MPASM_MPLINK_PIC18_LT_Branch_3_42\pic18-lt\cxx-framework\src\traditional\proc\p18f97j60.asm
                  SSP2BUF   0x000f66       data     extern E:\MPASM_MPLINK_PIC18_LT_Branch_3_42\pic18-lt\cxx-framework\src\traditional\proc\p18f97j60.asm
                 SSP2CON1   0x000f63       data     extern E:\MPASM_MPLINK_PIC18_LT_Branch_3_42\pic18-lt\cxx-framework\src\traditional\proc\p18f97j60.asm
             SSP2CON1bits   0x000f63       data     extern E:\MPASM_MPLINK_PIC18_LT_Branch_3_42\pic18-lt\cxx-framework\src\traditional\proc\p18f97j60.asm
                 SSP2CON2   0x000f62       data     extern E:\MPASM_MPLINK_PIC18_LT_Branch_3_42\pic18-lt\cxx-framework\src\traditional\proc\p18f97j60.asm
             SSP2CON2bits   0x000f62       data     extern E:\MPASM_MPLINK_PIC18_LT_Branch_3_42\pic18-lt\cxx-framework\src\traditional\proc\p18f97j60.asm
                 SSP2STAT   0x000f64       data     extern E:\MPASM_MPLINK_PIC18_LT_Branch_3_42\pic18-lt\cxx-framework\src\traditional\proc\p18f97j60.asm
             SSP2STATbits   0x000f64       data     extern E:\MPASM_MPLINK_PIC18_LT_Branch_3_42\pic18-lt\cxx-framework\src\traditional\proc\p18f97j60.asm
                   SSPADD   0x000fc8       data     extern E:\MPASM_MPLINK_PIC18_LT_Branch_3_42\pic18-lt\cxx-framework\src\traditional\proc\p18f97j60.asm
                   SSPBUF   0x000fc9       data     extern E:\MPASM_MPLINK_PIC18_LT_Branch_3_42\pic18-lt\cxx-framework\src\traditional\proc\p18f97j60.asm
                  SSPCON1   0x000fc6       data     extern E:\MPASM_MPLINK_PIC18_LT_Branch_3_42\pic18-lt\cxx-framework\src\traditional\proc\p18f97j60.asm
              SSPCON1bits   0x000fc6       data     extern E:\MPASM_MPLINK_PIC18_LT_Branch_3_42\pic18-lt\cxx-framework\src\traditional\proc\p18f97j60.asm
                  SSPCON2   0x000fc5       data     extern E:\MPASM_MPLINK_PIC18_LT_Branch_3_42\pic18-lt\cxx-framework\src\traditional\proc\p18f97j60.asm
              SSPCON2bits   0x000fc5       data     extern E:\MPASM_MPLINK_PIC18_LT_Branch_3_42\pic18-lt\cxx-framework\src\traditional\proc\p18f97j60.asm
                  SSPSTAT   0x000fc7       data     extern E:\MPASM_MPLINK_PIC18_LT_Branch_3_42\pic18-lt\cxx-framework\src\traditional\proc\p18f97j60.asm
              SSPSTATbits   0x000fc7       data     extern E:\MPASM_MPLINK_PIC18_LT_Branch_3_42\pic18-lt\cxx-framework\src\traditional\proc\p18f97j60.asm
                    START   0x000a3b       data     extern C:\Users\LFRAD\Documents\CMS2Luc\ProjetsNettoyesCMSGit\ProjetCarteIO\project\MainDemoV1.c
                   STATUS   0x000fd8       data     extern E:\MPASM_MPLINK_PIC18_LT_Branch_3_42\pic18-lt\cxx-framework\src\traditional\proc\p18f97j60.asm
               STATUSbits   0x000fd8       data     extern E:\MPASM_MPLINK_PIC18_LT_Branch_3_42\pic18-lt\cxx-framework\src\traditional\proc\p18f97j60.asm
                   STKPTR   0x000ffc       data     extern E:\MPASM_MPLINK_PIC18_LT_Branch_3_42\pic18-lt\cxx-framework\src\traditional\proc\p18f97j60.asm
               STKPTRbits   0x000ffc       data     extern E:\MPASM_MPLINK_PIC18_LT_Branch_3_42\pic18-lt\cxx-framework\src\traditional\proc\p18f97j60.asm
                     STOP   0x000a48       data     extern C:\Users\LFRAD\Documents\CMS2Luc\ProjetsNettoyesCMSGit\ProjetCarteIO\project\MainDemoV1.c
              STOPMINITEL   0x00006c       data     extern C:\Users\LFRAD\Documents\CMS2Luc\ProjetsNettoyesCMSGit\ProjetCarteIO\project\MainDemoV1.c
                 SYNQueue   0x000f00       data     static C:\Users\LFRAD\Documents\CMS2Luc\ProjetsNettoyesCMSGit\ProjetCarteIO\project\TCP.c
        SentTransactionID   0x0007ec       data     static C:\Users\LFRAD\Documents\CMS2Luc\ProjetsNettoyesCMSGit\ProjetCarteIO\project\DNS.c
               ServerName   0x000e63       data     static C:\Users\LFRAD\Documents\CMS2Luc\ProjetsNettoyesCMSGit\ProjetCarteIO\project\GenericTCPClient.c
             ServerNameio   0x0009fb       data     static C:\Users\LFRAD\Documents\CMS2Luc\ProjetsNettoyesCMSGit\ProjetCarteIO\project\MainDemoV1.c
               ServerPort   0x000e67       data     static C:\Users\LFRAD\Documents\CMS2Luc\ProjetsNettoyesCMSGit\ProjetCarteIO\project\GenericTCPClient.c
         SocketWithRxData   0x0000ff       data     static C:\Users\LFRAD\Documents\CMS2Luc\ProjetsNettoyesCMSGit\ProjetCarteIO\project\UDP.c
                SrcIPAddr   0x0006df       data     static C:\Users\LFRAD\Documents\CMS2Luc\ProjetsNettoyesCMSGit\ProjetCarteIO\project\ARP.c
                    Start   0x000b25       data     static C:\Users\LFRAD\Documents\CMS2Luc\ProjetsNettoyesCMSGit\ProjetCarteIO\project\ETH97J60.c
                StartTime   0x0007e8       data     static C:\Users\LFRAD\Documents\CMS2Luc\ProjetsNettoyesCMSGit\ProjetCarteIO\project\DNS.c
                   String   0x0007f2       data     static C:\Users\LFRAD\Documents\CMS2Luc\ProjetsNettoyesCMSGit\ProjetCarteIO\project\DNS.c
                   String   0x0007f0       data     static C:\Users\LFRAD\Documents\CMS2Luc\ProjetsNettoyesCMSGit\ProjetCarteIO\project\DNS.c
                    T0CON   0x000fd5       data     extern E:\MPASM_MPLINK_PIC18_LT_Branch_3_42\pic18-lt\cxx-framework\src\traditional\proc\p18f97j60.asm
                T0CONSave   0x000b11       data     static C:\Users\LFRAD\Documents\CMS2Luc\ProjetsNettoyesCMSGit\ProjetCarteIO\project\Helpers.c
                T0CONbits   0x000fd5       data     extern E:\MPASM_MPLINK_PIC18_LT_Branch_3_42\pic18-lt\cxx-framework\src\traditional\proc\p18f97j60.asm
                    T1CON   0x000fcd       data     extern E:\MPASM_MPLINK_PIC18_LT_Branch_3_42\pic18-lt\cxx-framework\src\traditional\proc\p18f97j60.asm
                T1CONbits   0x000fcd       data     extern E:\MPASM_MPLINK_PIC18_LT_Branch_3_42\pic18-lt\cxx-framework\src\traditional\proc\p18f97j60.asm
                    T2CON   0x000fca       data     extern E:\MPASM_MPLINK_PIC18_LT_Branch_3_42\pic18-lt\cxx-framework\src\traditional\proc\p18f97j60.asm
                T2CONbits   0x000fca       data     extern E:\MPASM_MPLINK_PIC18_LT_Branch_3_42\pic18-lt\cxx-framework\src\traditional\proc\p18f97j60.asm
                    T3CON   0x000fb1       data     extern E:\MPASM_MPLINK_PIC18_LT_Branch_3_42\pic18-lt\cxx-framework\src\traditional\proc\p18f97j60.asm
                T3CONbits   0x000fb1       data     extern E:\MPASM_MPLINK_PIC18_LT_Branch_3_42\pic18-lt\cxx-framework\src\traditional\proc\p18f97j60.asm
                    T4CON   0x000f76       data     extern E:\MPASM_MPLINK_PIC18_LT_Branch_3_42\pic18-lt\cxx-framework\src\traditional\proc\p18f97j60.asm
                T4CONbits   0x000f76       data     extern E:\MPASM_MPLINK_PIC18_LT_Branch_3_42\pic18-lt\cxx-framework\src\traditional\proc\p18f97j60.asm
                   TABLAT   0x000ff5       data     extern E:\MPASM_MPLINK_PIC18_LT_Branch_3_42\pic18-lt\cxx-framework\src\traditional\proc\p18f97j60.asm
                   TBLPTR   0x000ff6       data     extern E:\MPASM_MPLINK_PIC18_LT_Branch_3_42\pic18-lt\cxx-framework\src\traditional\proc\p18f97j60.asm
                  TBLPTRH   0x000ff7       data     extern E:\MPASM_MPLINK_PIC18_LT_Branch_3_42\pic18-lt\cxx-framework\src\traditional\proc\p18f97j60.asm
                  TBLPTRL   0x000ff6       data     extern E:\MPASM_MPLINK_PIC18_LT_Branch_3_42\pic18-lt\cxx-framework\src\traditional\proc\p18f97j60.asm
                  TBLPTRU   0x000ff8       data     extern E:\MPASM_MPLINK_PIC18_LT_Branch_3_42\pic18-lt\cxx-framework\src\traditional\proc\p18f97j60.asm
                 TCBStubs   0x000100       data     static C:\Users\LFRAD\Documents\CMS2Luc\ProjetsNettoyesCMSGit\ProjetCarteIO\project\TCP.c
                TCPHeader   0x000b00       data     static C:\Users\LFRAD\Documents\CMS2Luc\ProjetsNettoyesCMSGit\ProjetCarteIO\project\TCP.c
           TCPServerState   0x000e73       data     static C:\Users\LFRAD\Documents\CMS2Luc\ProjetsNettoyesCMSGit\ProjetCarteIO\project\GenericTCPServer.c
                   TEMPS1   0x000b01       data     static C:\Users\LFRAD\Documents\CMS2Luc\ProjetsNettoyesCMSGit\ProjetCarteIO\project\MainDemoV1.c
                   TEMPS2   0x000b03       data     static C:\Users\LFRAD\Documents\CMS2Luc\ProjetsNettoyesCMSGit\ProjetCarteIO\project\MainDemoV1.c
       TEMPS_CYCLE_MOTEUR   0x0005c0       data     extern C:\Users\LFRAD\Documents\CMS2Luc\ProjetsNettoyesCMSGit\ProjetCarteIO\project\MainDemoV1.c
             TEMPS_MOTEUR   0x0005cb       data     extern C:\Users\LFRAD\Documents\CMS2Luc\ProjetsNettoyesCMSGit\ProjetCarteIO\project\MainDemoV1.c
            TERMINEACTION   0x000903       data     extern C:\Users\LFRAD\Documents\CMS2Luc\ProjetsNettoyesCMSGit\ProjetCarteIO\project\MainDemoV1.c
                      TMP   0x000500       data     extern C:\Users\LFRAD\Documents\CMS2Luc\ProjetsNettoyesCMSGit\ProjetCarteIO\project\MainDemoV1.c
                      TMP   0x000b07       data     static C:\Users\LFRAD\Documents\CMS2Luc\ProjetsNettoyesCMSGit\ProjetCarteIO\project\MainDemoV1.c
                      TMP   0x000b08       data     static C:\Users\LFRAD\Documents\CMS2Luc\ProjetsNettoyesCMSGit\ProjetCarteIO\project\MainDemoV1.c
                      TMP   0x000b01       data     static C:\Users\LFRAD\Documents\CMS2Luc\ProjetsNettoyesCMSGit\ProjetCarteIO\project\MainDemoV1.c
                     TMP2   0x000b00       data     static C:\Users\LFRAD\Documents\CMS2Luc\ProjetsNettoyesCMSGit\ProjetCarteIO\project\MainDemoV1.c
                     TMP2   0x000b14       data     static C:\Users\LFRAD\Documents\CMS2Luc\ProjetsNettoyesCMSGit\ProjetCarteIO\project\MainDemoV1.c
                     TMP4   0x000b15       data     static C:\Users\LFRAD\Documents\CMS2Luc\ProjetsNettoyesCMSGit\ProjetCarteIO\project\MainDemoV1.c
                   TMPTDA   0x000b78       data     static C:\Users\LFRAD\Documents\CMS2Luc\ProjetsNettoyesCMSGit\ProjetCarteIO\project\MainDemoV1.c
                    TMR0H   0x000fd7       data     extern E:\MPASM_MPLINK_PIC18_LT_Branch_3_42\pic18-lt\cxx-framework\src\traditional\proc\p18f97j60.asm
                TMR0HSave   0x000b12       data     static C:\Users\LFRAD\Documents\CMS2Luc\ProjetsNettoyesCMSGit\ProjetCarteIO\project\Helpers.c
                    TMR0L   0x000fd6       data     extern E:\MPASM_MPLINK_PIC18_LT_Branch_3_42\pic18-lt\cxx-framework\src\traditional\proc\p18f97j60.asm
                TMR0LSave   0x000b13       data     static C:\Users\LFRAD\Documents\CMS2Luc\ProjetsNettoyesCMSGit\ProjetCarteIO\project\Helpers.c
                    TMR1H   0x000fcf       data     extern E:\MPASM_MPLINK_PIC18_LT_Branch_3_42\pic18-lt\cxx-framework\src\traditional\proc\p18f97j60.asm
                    TMR1L   0x000fce       data     extern E:\MPASM_MPLINK_PIC18_LT_Branch_3_42\pic18-lt\cxx-framework\src\traditional\proc\p18f97j60.asm
                     TMR2   0x000fcc       data     extern E:\MPASM_MPLINK_PIC18_LT_Branch_3_42\pic18-lt\cxx-framework\src\traditional\proc\p18f97j60.asm
                    TMR3H   0x000fb3       data     extern E:\MPASM_MPLINK_PIC18_LT_Branch_3_42\pic18-lt\cxx-framework\src\traditional\proc\p18f97j60.asm
                    TMR3L   0x000fb2       data     extern E:\MPASM_MPLINK_PIC18_LT_Branch_3_42\pic18-lt\cxx-framework\src\traditional\proc\p18f97j60.asm
                     TMR4   0x000f78       data     extern E:\MPASM_MPLINK_PIC18_LT_Branch_3_42\pic18-lt\cxx-framework\src\traditional\proc\p18f97j60.asm
                      TOS   0x000ffd       data     extern E:\MPASM_MPLINK_PIC18_LT_Branch_3_42\pic18-lt\cxx-framework\src\traditional\proc\p18f97j60.asm
                     TOSH   0x000ffe       data     extern E:\MPASM_MPLINK_PIC18_LT_Branch_3_42\pic18-lt\cxx-framework\src\traditional\proc\p18f97j60.asm
                     TOSL   0x000ffd       data     extern E:\MPASM_MPLINK_PIC18_LT_Branch_3_42\pic18-lt\cxx-framework\src\traditional\proc\p18f97j60.asm
                     TOSU   0x000fff       data     extern E:\MPASM_MPLINK_PIC18_LT_Branch_3_42\pic18-lt\cxx-framework\src\traditional\proc\p18f97j60.asm
                      TRA   0x000982       data     extern C:\Users\LFRAD\Documents\CMS2Luc\ProjetsNettoyesCMSGit\ProjetCarteIO\project\MainDemoV1.c
                  TRAMEIN   0x000800       data     extern C:\Users\LFRAD\Documents\CMS2Luc\ProjetsNettoyesCMSGit\ProjetCarteIO\project\MainDemoV1.c
                 TRAMEOUT   0x000200       data     extern C:\Users\LFRAD\Documents\CMS2Luc\ProjetsNettoyesCMSGit\ProjetCarteIO\project\MainDemoV1.c
               TRANSALARM   0x000667       data     extern C:\Users\LFRAD\Documents\CMS2Luc\ProjetsNettoyesCMSGit\ProjetCarteIO\project\MainDemoV1.c
         TRANSSORTIEALARM   0x000668       data     extern C:\Users\LFRAD\Documents\CMS2Luc\ProjetsNettoyesCMSGit\ProjetCarteIO\project\MainDemoV1.c
                    TRISA   0x000f92       data     extern E:\MPASM_MPLINK_PIC18_LT_Branch_3_42\pic18-lt\cxx-framework\src\traditional\proc\p18f97j60.asm
                TRISAbits   0x000f92       data     extern E:\MPASM_MPLINK_PIC18_LT_Branch_3_42\pic18-lt\cxx-framework\src\traditional\proc\p18f97j60.asm
                    TRISB   0x000f93       data     extern E:\MPASM_MPLINK_PIC18_LT_Branch_3_42\pic18-lt\cxx-framework\src\traditional\proc\p18f97j60.asm
                TRISBbits   0x000f93       data     extern E:\MPASM_MPLINK_PIC18_LT_Branch_3_42\pic18-lt\cxx-framework\src\traditional\proc\p18f97j60.asm
                    TRISC   0x000f94       data     extern E:\MPASM_MPLINK_PIC18_LT_Branch_3_42\pic18-lt\cxx-framework\src\traditional\proc\p18f97j60.asm
                TRISCbits   0x000f94       data     extern E:\MPASM_MPLINK_PIC18_LT_Branch_3_42\pic18-lt\cxx-framework\src\traditional\proc\p18f97j60.asm
                    TRISD   0x000f95       data     extern E:\MPASM_MPLINK_PIC18_LT_Branch_3_42\pic18-lt\cxx-framework\src\traditional\proc\p18f97j60.asm
                TRISDbits   0x000f95       data     extern E:\MPASM_MPLINK_PIC18_LT_Branch_3_42\pic18-lt\cxx-framework\src\traditional\proc\p18f97j60.asm
                    TRISE   0x000f96       data     extern E:\MPASM_MPLINK_PIC18_LT_Branch_3_42\pic18-lt\cxx-framework\src\traditional\proc\p18f97j60.asm
                TRISEbits   0x000f96       data     extern E:\MPASM_MPLINK_PIC18_LT_Branch_3_42\pic18-lt\cxx-framework\src\traditional\proc\p18f97j60.asm
                    TRISF   0x000f97       data     extern E:\MPASM_MPLINK_PIC18_LT_Branch_3_42\pic18-lt\cxx-framework\src\traditional\proc\p18f97j60.asm
                TRISFbits   0x000f97       data     extern E:\MPASM_MPLINK_PIC18_LT_Branch_3_42\pic18-lt\cxx-framework\src\traditional\proc\p18f97j60.asm
                    TRISG   0x000f98       data     extern E:\MPASM_MPLINK_PIC18_LT_Branch_3_42\pic18-lt\cxx-framework\src\traditional\proc\p18f97j60.asm
                TRISGbits   0x000f98       data     extern E:\MPASM_MPLINK_PIC18_LT_Branch_3_42\pic18-lt\cxx-framework\src\traditional\proc\p18f97j60.asm
                    TRISH   0x000f99       data     extern E:\MPASM_MPLINK_PIC18_LT_Branch_3_42\pic18-lt\cxx-framework\src\traditional\proc\p18f97j60.asm
                TRISHbits   0x000f99       data     extern E:\MPASM_MPLINK_PIC18_LT_Branch_3_42\pic18-lt\cxx-framework\src\traditional\proc\p18f97j60.asm
                    TRISJ   0x000f9a       data     extern E:\MPASM_MPLINK_PIC18_LT_Branch_3_42\pic18-lt\cxx-framework\src\traditional\proc\p18f97j60.asm
                TRISJbits   0x000f9a       data     extern E:\MPASM_MPLINK_PIC18_LT_Branch_3_42\pic18-lt\cxx-framework\src\traditional\proc\p18f97j60.asm
                    TXREG   0x000fad       data     extern E:\MPASM_MPLINK_PIC18_LT_Branch_3_42\pic18-lt\cxx-framework\src\traditional\proc\p18f97j60.asm
                   TXREG1   0x000fad       data     extern E:\MPASM_MPLINK_PIC18_LT_Branch_3_42\pic18-lt\cxx-framework\src\traditional\proc\p18f97j60.asm
                   TXREG2   0x000f6d       data     extern E:\MPASM_MPLINK_PIC18_LT_Branch_3_42\pic18-lt\cxx-framework\src\traditional\proc\p18f97j60.asm
                    TXSTA   0x000fac       data     extern E:\MPASM_MPLINK_PIC18_LT_Branch_3_42\pic18-lt\cxx-framework\src\traditional\proc\p18f97j60.asm
                   TXSTA1   0x000fac       data     extern E:\MPASM_MPLINK_PIC18_LT_Branch_3_42\pic18-lt\cxx-framework\src\traditional\proc\p18f97j60.asm
               TXSTA1bits   0x000fac       data     extern E:\MPASM_MPLINK_PIC18_LT_Branch_3_42\pic18-lt\cxx-framework\src\traditional\proc\p18f97j60.asm
                   TXSTA2   0x000f6c       data     extern E:\MPASM_MPLINK_PIC18_LT_Branch_3_42\pic18-lt\cxx-framework\src\traditional\proc\p18f97j60.asm
               TXSTA2bits   0x000f6c       data     extern E:\MPASM_MPLINK_PIC18_LT_Branch_3_42\pic18-lt\cxx-framework\src\traditional\proc\p18f97j60.asm
                TXSTAbits   0x000fac       data     extern E:\MPASM_MPLINK_PIC18_LT_Branch_3_42\pic18-lt\cxx-framework\src\traditional\proc\p18f97j60.asm
                     TYPE   0x000959       data     extern C:\Users\LFRAD\Documents\CMS2Luc\ProjetsNettoyesCMSGit\ProjetCarteIO\project\MainDemoV1.c
                TYPECARTE   0x000a6c       data     extern C:\Users\LFRAD\Documents\CMS2Luc\ProjetsNettoyesCMSGit\ProjetCarteIO\project\MainDemoV1.c
          TYPEORDREALARME   0x000666       data     extern C:\Users\LFRAD\Documents\CMS2Luc\ProjetsNettoyesCMSGit\ProjetCarteIO\project\MainDemoV1.c
              TYPE_ERREUR   0x000a55       data     extern C:\Users\LFRAD\Documents\CMS2Luc\ProjetsNettoyesCMSGit\ProjetCarteIO\project\MainDemoV1.c
                 T_alarme   0x0000cf       data     extern C:\Users\LFRAD\Documents\CMS2Luc\ProjetsNettoyesCMSGit\ProjetCarteIO\project\MainDemoV1.c
                 T_sortie   0x0000d2       data     extern C:\Users\LFRAD\Documents\CMS2Luc\ProjetsNettoyesCMSGit\ProjetCarteIO\project\MainDemoV1.c
           Tab_Horodatage   0x000060       data     extern C:\Users\LFRAD\Documents\CMS2Luc\ProjetsNettoyesCMSGit\ProjetCarteIO\project\MainDemoV1.c
                   Target   0x0006ea       data     static C:\Users\LFRAD\Documents\CMS2Luc\ProjetsNettoyesCMSGit\ProjetCarteIO\project\ARP.c
                     Time   0x0006be       data     static C:\Users\LFRAD\Documents\CMS2Luc\ProjetsNettoyesCMSGit\ProjetCarteIO\project\MainDemoV1.c
                    Timer   0x0008f2       data     static C:\Users\LFRAD\Documents\CMS2Luc\ProjetsNettoyesCMSGit\ProjetCarteIO\project\GenericTCPClient.c
                 Timering   0x0006cb       data     static C:\Users\LFRAD\Documents\CMS2Luc\ProjetsNettoyesCMSGit\ProjetCarteIO\project\MainDemoV1.c
                     Type   0x0007e5       data     static C:\Users\LFRAD\Documents\CMS2Luc\ProjetsNettoyesCMSGit\ProjetCarteIO\project\DNS.c
                     Type   0x0007e1       data     static C:\Users\LFRAD\Documents\CMS2Luc\ProjetsNettoyesCMSGit\ProjetCarteIO\project\DNS.c
               UDPRxCount   0x0004bb       data     extern C:\Users\LFRAD\Documents\CMS2Luc\ProjetsNettoyesCMSGit\ProjetCarteIO\project\UDP.c
            UDPSocketInfo   0x000400       data     extern C:\Users\LFRAD\Documents\CMS2Luc\ProjetsNettoyesCMSGit\ProjetCarteIO\project\UDP.c
               UDPTxCount   0x0004b9       data     extern C:\Users\LFRAD\Documents\CMS2Luc\ProjetsNettoyesCMSGit\ProjetCarteIO\project\UDP.c
                     Unit   0x000b06       data     static C:\Users\LFRAD\Documents\CMS2Luc\ProjetsNettoyesCMSGit\ProjetCarteIO\project\MainDemoV1.c
                     Unit   0x000b06       data     static C:\Users\LFRAD\Documents\CMS2Luc\ProjetsNettoyesCMSGit\ProjetCarteIO\project\GenericTCPClient.c
                     Unit   0x000b06       data     static C:\Users\LFRAD\Documents\CMS2Luc\ProjetsNettoyesCMSGit\ProjetCarteIO\project\MainDemoV1.c
        UpdateReadPointer   0x000b30       data     static C:\Users\LFRAD\Documents\CMS2Luc\ProjetsNettoyesCMSGit\ProjetCarteIO\project\ETH97J60.c
       UpdateWritePointer   0x000b2f       data     static C:\Users\LFRAD\Documents\CMS2Luc\ProjetsNettoyesCMSGit\ProjetCarteIO\project\ETH97J60.c
                   VALEUR   0x00091a       data     extern C:\Users\LFRAD\Documents\CMS2Luc\ProjetsNettoyesCMSGit\ProjetCarteIO\project\MainDemoV1.c
                  VOIECOD   0x00093a       data     extern C:\Users\LFRAD\Documents\CMS2Luc\ProjetsNettoyesCMSGit\ProjetCarteIO\project\MainDemoV1.c
                    Value   0x000a0d       data     static C:\Users\LFRAD\Documents\CMS2Luc\ProjetsNettoyesCMSGit\ProjetCarteIO\project\Helpers.c
                   WDTCON   0x000fd1       data     extern E:\MPASM_MPLINK_PIC18_LT_Branch_3_42\pic18-lt\cxx-framework\src\traditional\proc\p18f97j60.asm
               WDTCONbits   0x000fd1       data     extern E:\MPASM_MPLINK_PIC18_LT_Branch_3_42\pic18-lt\cxx-framework\src\traditional\proc\p18f97j60.asm
                     WREG   0x000fe8       data     extern E:\MPASM_MPLINK_PIC18_LT_Branch_3_42\pic18-lt\cxx-framework\src\traditional\proc\p18f97j60.asm
                  WritePT   0x000b27       data     static C:\Users\LFRAD\Documents\CMS2Luc\ProjetsNettoyesCMSGit\ProjetCarteIO\project\ETH97J60.c
                WriteSave   0x000b2d       data     static C:\Users\LFRAD\Documents\CMS2Luc\ProjetsNettoyesCMSGit\ProjetCarteIO\project\ETH97J60.c
               ZPLENVOYEE   0x0009e7       data     extern C:\Users\LFRAD\Documents\CMS2Luc\ProjetsNettoyesCMSGit\ProjetCarteIO\project\MainDemoV1.c
              _Identifier   0x000e70       data     static C:\Users\LFRAD\Documents\CMS2Luc\ProjetsNettoyesCMSGit\ProjetCarteIO\project\IP.c
                 __AARGB0   0x000009       data     extern E:\MPASM_MPLINK_PIC18_LT_Branch_3_42\pic18-lt\cxx-framework\src\traditional\math\aarg.asm
                 __AARGB1   0x000008       data     extern E:\MPASM_MPLINK_PIC18_LT_Branch_3_42\pic18-lt\cxx-framework\src\traditional\math\aarg.asm
                 __AARGB2   0x000007       data     extern E:\MPASM_MPLINK_PIC18_LT_Branch_3_42\pic18-lt\cxx-framework\src\traditional\math\aarg.asm
                 __AARGB3   0x000006       data     extern E:\MPASM_MPLINK_PIC18_LT_Branch_3_42\pic18-lt\cxx-framework\src\traditional\math\aarg.asm
                 __AARGB4   0x000005       data     extern E:\MPASM_MPLINK_PIC18_LT_Branch_3_42\pic18-lt\cxx-framework\src\traditional\math\aarg.asm
                 __AARGB5   0x000004       data     extern E:\MPASM_MPLINK_PIC18_LT_Branch_3_42\pic18-lt\cxx-framework\src\traditional\math\aarg.asm
                 __AARGB6   0x000003       data     extern E:\MPASM_MPLINK_PIC18_LT_Branch_3_42\pic18-lt\cxx-framework\src\traditional\math\aarg.asm
                 __AARGB7   0x000002       data     extern E:\MPASM_MPLINK_PIC18_LT_Branch_3_42\pic18-lt\cxx-framework\src\traditional\math\aarg.asm
                   __AEXP   0x00000a       data     extern E:\MPASM_MPLINK_PIC18_LT_Branch_3_42\pic18-lt\cxx-framework\src\traditional\math\aarg.asm
        __ARPIsResolved:0   0x0006f6       data     extern C:\Users\LFRAD\Documents\CMS2Luc\ProjetsNettoyesCMSGit\ProjetCarteIO\project\ARP.c
        __ARPIsResolved:1   0x0006f8       data     extern C:\Users\LFRAD\Documents\CMS2Luc\ProjetsNettoyesCMSGit\ProjetCarteIO\project\ARP.c
               __ARPPut:0   0x0006e8       data     static C:\Users\LFRAD\Documents\CMS2Luc\ProjetsNettoyesCMSGit\ProjetCarteIO\project\ARP.c
           __ARPResolve:0   0x0006f4       data     extern C:\Users\LFRAD\Documents\CMS2Luc\ProjetsNettoyesCMSGit\ProjetCarteIO\project\ARP.c
           __ARPSendPkt:0   0x0006df       data     extern C:\Users\LFRAD\Documents\CMS2Luc\ProjetsNettoyesCMSGit\ProjetCarteIO\project\ARP.c
           __ARPSendPkt:1   0x0006e3       data     extern C:\Users\LFRAD\Documents\CMS2Luc\ProjetsNettoyesCMSGit\ProjetCarteIO\project\ARP.c
           __ARPSendPkt:2   0x0006e7       data     extern C:\Users\LFRAD\Documents\CMS2Luc\ProjetsNettoyesCMSGit\ProjetCarteIO\project\ARP.c
                 __BARGB0   0x00000e       data     extern E:\MPASM_MPLINK_PIC18_LT_Branch_3_42\pic18-lt\cxx-framework\src\traditional\math\barg.asm
                 __BARGB1   0x00000d       data     extern E:\MPASM_MPLINK_PIC18_LT_Branch_3_42\pic18-lt\cxx-framework\src\traditional\math\barg.asm
                 __BARGB2   0x00000c       data     extern E:\MPASM_MPLINK_PIC18_LT_Branch_3_42\pic18-lt\cxx-framework\src\traditional\math\barg.asm
                 __BARGB3   0x00000b       data     extern E:\MPASM_MPLINK_PIC18_LT_Branch_3_42\pic18-lt\cxx-framework\src\traditional\math\barg.asm
                   __BEXP   0x00000f       data     extern E:\MPASM_MPLINK_PIC18_LT_Branch_3_42\pic18-lt\cxx-framework\src\traditional\math\barg.asm
__CHERCHER_DONNNEES_CABLES:0   0x00069a       data     extern C:\Users\LFRAD\Documents\CMS2Luc\ProjetsNettoyesCMSGit\ProjetCarteIO\project\MainDemoV1.c
__CHERCHER_DONNNEES_CABLES:1   0x00069c       data     extern C:\Users\LFRAD\Documents\CMS2Luc\ProjetsNettoyesCMSGit\ProjetCarteIO\project\MainDemoV1.c
               __CRC116:0   0x0008fb       data     extern C:\Users\LFRAD\Documents\CMS2Luc\ProjetsNettoyesCMSGit\ProjetCarteIO\project\GenericTCPClient.c
               __CRC116:1   0x0008fd       data     extern C:\Users\LFRAD\Documents\CMS2Luc\ProjetsNettoyesCMSGit\ProjetCarteIO\project\GenericTCPClient.c
                __CRC16:0   0x000678       data     extern C:\Users\LFRAD\Documents\CMS2Luc\ProjetsNettoyesCMSGit\ProjetCarteIO\project\MainDemoV1.c
                __CRC16:1   0x00067a       data     extern C:\Users\LFRAD\Documents\CMS2Luc\ProjetsNettoyesCMSGit\ProjetCarteIO\project\MainDemoV1.c
 __CalcIPBufferChecksum:0   0x000a8e       data     extern C:\Users\LFRAD\Documents\CMS2Luc\ProjetsNettoyesCMSGit\ProjetCarteIO\project\ETH97J60.c
       __CalcIPChecksum:0   0x000a20       data     extern C:\Users\LFRAD\Documents\CMS2Luc\ProjetsNettoyesCMSGit\ProjetCarteIO\project\Helpers.c
       __CalcIPChecksum:1   0x000a22       data     extern C:\Users\LFRAD\Documents\CMS2Luc\ProjetsNettoyesCMSGit\ProjetCarteIO\project\Helpers.c
        __DNSIsResolved:0   0x0007e6       data     extern C:\Users\LFRAD\Documents\CMS2Luc\ProjetsNettoyesCMSGit\ProjetCarteIO\project\DNS.c
      __DNSPutROMString:0   0x0007f2       data     static C:\Users\LFRAD\Documents\CMS2Luc\ProjetsNettoyesCMSGit\ProjetCarteIO\project\DNS.c
         __DNSPutString:0   0x0007f0       data     static C:\Users\LFRAD\Documents\CMS2Luc\ProjetsNettoyesCMSGit\ProjetCarteIO\project\DNS.c
           __DNSResolve:0   0x0007df       data     extern C:\Users\LFRAD\Documents\CMS2Luc\ProjetsNettoyesCMSGit\ProjetCarteIO\project\DNS.c
           __DNSResolve:1   0x0007e1       data     extern C:\Users\LFRAD\Documents\CMS2Luc\ProjetsNettoyesCMSGit\ProjetCarteIO\project\DNS.c
        __DNSResolveROM:0   0x0007e2       data     extern C:\Users\LFRAD\Documents\CMS2Luc\ProjetsNettoyesCMSGit\ProjetCarteIO\project\DNS.c
        __DNSResolveROM:1   0x0007e5       data     extern C:\Users\LFRAD\Documents\CMS2Luc\ProjetsNettoyesCMSGit\ProjetCarteIO\project\DNS.c
       __DisplayIPValue:0   0x00066f       data     extern C:\Users\LFRAD\Documents\CMS2Luc\ProjetsNettoyesCMSGit\ProjetCarteIO\project\MainDemoV1.c
    __ECRIRE_EEPROMBYTE:0   0x0006a3       data     extern C:\Users\LFRAD\Documents\CMS2Luc\ProjetsNettoyesCMSGit\ProjetCarteIO\project\MainDemoV1.c
    __ECRIRE_EEPROMBYTE:1   0x0006a4       data     extern C:\Users\LFRAD\Documents\CMS2Luc\ProjetsNettoyesCMSGit\ProjetCarteIO\project\MainDemoV1.c
    __ECRIRE_EEPROMBYTE:2   0x0006a6       data     extern C:\Users\LFRAD\Documents\CMS2Luc\ProjetsNettoyesCMSGit\ProjetCarteIO\project\MainDemoV1.c
    __ECRIRE_EEPROMBYTE:3   0x0006a8       data     extern C:\Users\LFRAD\Documents\CMS2Luc\ProjetsNettoyesCMSGit\ProjetCarteIO\project\MainDemoV1.c
       __ECRIRE_HORLOGE:0   0x0006bd       data     extern C:\Users\LFRAD\Documents\CMS2Luc\ProjetsNettoyesCMSGit\ProjetCarteIO\project\MainDemoV1.c
       __ECRIRE_HORLOGE:1   0x0006be       data     extern C:\Users\LFRAD\Documents\CMS2Luc\ProjetsNettoyesCMSGit\ProjetCarteIO\project\MainDemoV1.c
    __ENVOIE_DES_TRAMES:0   0x0006ae       data     extern C:\Users\LFRAD\Documents\CMS2Luc\ProjetsNettoyesCMSGit\ProjetCarteIO\project\MainDemoV1.c
    __ENVOIE_DES_TRAMES:1   0x0006af       data     extern C:\Users\LFRAD\Documents\CMS2Luc\ProjetsNettoyesCMSGit\ProjetCarteIO\project\MainDemoV1.c
    __ENVOIE_DES_TRAMES:2   0x0006b1       data     extern C:\Users\LFRAD\Documents\CMS2Luc\ProjetsNettoyesCMSGit\ProjetCarteIO\project\MainDemoV1.c
                __FPFLAGS   0x000001       data     extern E:\MPASM_MPLINK_PIC18_LT_Branch_3_42\pic18-lt\cxx-framework\src\traditional\math\cmath18.asm
            __FPFLAGSbits   0x000001       data     extern E:\MPASM_MPLINK_PIC18_LT_Branch_3_42\pic18-lt\cxx-framework\src\traditional\math\cmath18.asm
   __FindMatchingSocket:0   0x0007af       data     static C:\Users\LFRAD\Documents\CMS2Luc\ProjetsNettoyesCMSGit\ProjetCarteIO\project\TCP.c
   __FindMatchingSocket:0   0x0004f0       data     static C:\Users\LFRAD\Documents\CMS2Luc\ProjetsNettoyesCMSGit\ProjetCarteIO\project\UDP.c
   __FindMatchingSocket:1   0x0007b1       data     static C:\Users\LFRAD\Documents\CMS2Luc\ProjetsNettoyesCMSGit\ProjetCarteIO\project\TCP.c
   __FindMatchingSocket:1   0x0004f2       data     static C:\Users\LFRAD\Documents\CMS2Luc\ProjetsNettoyesCMSGit\ProjetCarteIO\project\UDP.c
   __FindMatchingSocket:2   0x0004f4       data     static C:\Users\LFRAD\Documents\CMS2Luc\ProjetsNettoyesCMSGit\ProjetCarteIO\project\UDP.c
    __FormatNetBIOSName:0   0x000a2d       data     extern C:\Users\LFRAD\Documents\CMS2Luc\ProjetsNettoyesCMSGit\ProjetCarteIO\project\Helpers.c
    __GROUPE_EN_MEMOIRE:0   0x0006b8       data     extern C:\Users\LFRAD\Documents\CMS2Luc\ProjetsNettoyesCMSGit\ProjetCarteIO\project\MainDemoV1.c
    __GROUPE_EN_MEMOIRE:1   0x0006ba       data     extern C:\Users\LFRAD\Documents\CMS2Luc\ProjetsNettoyesCMSGit\ProjetCarteIO\project\MainDemoV1.c
         __HandleTCPSeg:0   0x0007b5       data     static C:\Users\LFRAD\Documents\CMS2Luc\ProjetsNettoyesCMSGit\ProjetCarteIO\project\TCP.c
         __HandleTCPSeg:1   0x0007b7       data     static C:\Users\LFRAD\Documents\CMS2Luc\ProjetsNettoyesCMSGit\ProjetCarteIO\project\TCP.c
          __ICMPProcess:0   0x0001fc       data     extern C:\Users\LFRAD\Documents\CMS2Luc\ProjetsNettoyesCMSGit\ProjetCarteIO\project\ICMP.c
          __ICMPProcess:1   0x0001fe       data     extern C:\Users\LFRAD\Documents\CMS2Luc\ProjetsNettoyesCMSGit\ProjetCarteIO\project\ICMP.c
          __IPGetHeader:0   0x0005eb       data     extern C:\Users\LFRAD\Documents\CMS2Luc\ProjetsNettoyesCMSGit\ProjetCarteIO\project\IP.c
          __IPGetHeader:1   0x0005ed       data     extern C:\Users\LFRAD\Documents\CMS2Luc\ProjetsNettoyesCMSGit\ProjetCarteIO\project\IP.c
          __IPGetHeader:2   0x0005ef       data     extern C:\Users\LFRAD\Documents\CMS2Luc\ProjetsNettoyesCMSGit\ProjetCarteIO\project\IP.c
          __IPGetHeader:3   0x0005f1       data     extern C:\Users\LFRAD\Documents\CMS2Luc\ProjetsNettoyesCMSGit\ProjetCarteIO\project\IP.c
          __IPPutHeader:0   0x0005f3       data     extern C:\Users\LFRAD\Documents\CMS2Luc\ProjetsNettoyesCMSGit\ProjetCarteIO\project\IP.c
          __IPPutHeader:1   0x0005f5       data     extern C:\Users\LFRAD\Documents\CMS2Luc\ProjetsNettoyesCMSGit\ProjetCarteIO\project\IP.c
          __IPPutHeader:2   0x0005f6       data     extern C:\Users\LFRAD\Documents\CMS2Luc\ProjetsNettoyesCMSGit\ProjetCarteIO\project\IP.c
        __IPSetRxBuffer:0   0x0005f8       data     extern C:\Users\LFRAD\Documents\CMS2Luc\ProjetsNettoyesCMSGit\ProjetCarteIO\project\IP.c
           __IntToChar1:0   0x0008f6       data     extern C:\Users\LFRAD\Documents\CMS2Luc\ProjetsNettoyesCMSGit\ProjetCarteIO\project\GenericTCPClient.c
           __IntToChar1:1   0x0008f8       data     extern C:\Users\LFRAD\Documents\CMS2Luc\ProjetsNettoyesCMSGit\ProjetCarteIO\project\GenericTCPClient.c
           __IntToChar1:2   0x0008fa       data     extern C:\Users\LFRAD\Documents\CMS2Luc\ProjetsNettoyesCMSGit\ProjetCarteIO\project\GenericTCPClient.c
           __IntToChar5:0   0x0006d0       data     extern C:\Users\LFRAD\Documents\CMS2Luc\ProjetsNettoyesCMSGit\ProjetCarteIO\project\MainDemoV1.c
           __IntToChar5:1   0x0006d2       data     extern C:\Users\LFRAD\Documents\CMS2Luc\ProjetsNettoyesCMSGit\ProjetCarteIO\project\MainDemoV1.c
           __IntToChar5:2   0x0006d4       data     extern C:\Users\LFRAD\Documents\CMS2Luc\ProjetsNettoyesCMSGit\ProjetCarteIO\project\MainDemoV1.c
            __IntToChar:0   0x000673       data     extern C:\Users\LFRAD\Documents\CMS2Luc\ProjetsNettoyesCMSGit\ProjetCarteIO\project\MainDemoV1.c
            __IntToChar:1   0x000675       data     extern C:\Users\LFRAD\Documents\CMS2Luc\ProjetsNettoyesCMSGit\ProjetCarteIO\project\MainDemoV1.c
            __IntToChar:2   0x000677       data     extern C:\Users\LFRAD\Documents\CMS2Luc\ProjetsNettoyesCMSGit\ProjetCarteIO\project\MainDemoV1.c
         __LFSRSeedRand:0   0x000a00       data     extern C:\Users\LFRAD\Documents\CMS2Luc\ProjetsNettoyesCMSGit\ProjetCarteIO\project\Helpers.c
          __LIRE_EEPROM:0   0x00067e       data     extern C:\Users\LFRAD\Documents\CMS2Luc\ProjetsNettoyesCMSGit\ProjetCarteIO\project\MainDemoV1.c
          __LIRE_EEPROM:1   0x00067f       data     extern C:\Users\LFRAD\Documents\CMS2Luc\ProjetsNettoyesCMSGit\ProjetCarteIO\project\MainDemoV1.c
          __LIRE_EEPROM:2   0x000681       data     extern C:\Users\LFRAD\Documents\CMS2Luc\ProjetsNettoyesCMSGit\ProjetCarteIO\project\MainDemoV1.c
          __LIRE_EEPROM:3   0x000683       data     extern C:\Users\LFRAD\Documents\CMS2Luc\ProjetsNettoyesCMSGit\ProjetCarteIO\project\MainDemoV1.c
         __LIRE_HORLOGE:0   0x0006b3       data     extern C:\Users\LFRAD\Documents\CMS2Luc\ProjetsNettoyesCMSGit\ProjetCarteIO\project\MainDemoV1.c
    __MACCalcRxChecksum:0   0x000a8a       data     extern C:\Users\LFRAD\Documents\CMS2Luc\ProjetsNettoyesCMSGit\ProjetCarteIO\project\ETH97J60.c
    __MACCalcRxChecksum:1   0x000a8c       data     extern C:\Users\LFRAD\Documents\CMS2Luc\ProjetsNettoyesCMSGit\ProjetCarteIO\project\ETH97J60.c
          __MACGetArray:0   0x000a96       data     extern C:\Users\LFRAD\Documents\CMS2Luc\ProjetsNettoyesCMSGit\ProjetCarteIO\project\ETH97J60.c
          __MACGetArray:1   0x000a98       data     extern C:\Users\LFRAD\Documents\CMS2Luc\ProjetsNettoyesCMSGit\ProjetCarteIO\project\ETH97J60.c
         __MACGetHeader:0   0x000a7b       data     extern C:\Users\LFRAD\Documents\CMS2Luc\ProjetsNettoyesCMSGit\ProjetCarteIO\project\ETH97J60.c
         __MACGetHeader:1   0x000a7d       data     extern C:\Users\LFRAD\Documents\CMS2Luc\ProjetsNettoyesCMSGit\ProjetCarteIO\project\ETH97J60.c
      __MACMemCopyAsync:0   0x000a90       data     extern C:\Users\LFRAD\Documents\CMS2Luc\ProjetsNettoyesCMSGit\ProjetCarteIO\project\ETH97J60.c
      __MACMemCopyAsync:1   0x000a92       data     extern C:\Users\LFRAD\Documents\CMS2Luc\ProjetsNettoyesCMSGit\ProjetCarteIO\project\ETH97J60.c
      __MACMemCopyAsync:2   0x000a94       data     extern C:\Users\LFRAD\Documents\CMS2Luc\ProjetsNettoyesCMSGit\ProjetCarteIO\project\ETH97J60.c
               __MACPut:0   0x000a9a       data     extern C:\Users\LFRAD\Documents\CMS2Luc\ProjetsNettoyesCMSGit\ProjetCarteIO\project\ETH97J60.c
          __MACPutArray:0   0x000a9b       data     extern C:\Users\LFRAD\Documents\CMS2Luc\ProjetsNettoyesCMSGit\ProjetCarteIO\project\ETH97J60.c
          __MACPutArray:1   0x000a9d       data     extern C:\Users\LFRAD\Documents\CMS2Luc\ProjetsNettoyesCMSGit\ProjetCarteIO\project\ETH97J60.c
         __MACPutHeader:0   0x000a7f       data     extern C:\Users\LFRAD\Documents\CMS2Luc\ProjetsNettoyesCMSGit\ProjetCarteIO\project\ETH97J60.c
         __MACPutHeader:1   0x000a81       data     extern C:\Users\LFRAD\Documents\CMS2Luc\ProjetsNettoyesCMSGit\ProjetCarteIO\project\ETH97J60.c
         __MACPutHeader:2   0x000a82       data     extern C:\Users\LFRAD\Documents\CMS2Luc\ProjetsNettoyesCMSGit\ProjetCarteIO\project\ETH97J60.c
       __MACPutROMArray:0   0x000a9f       data     extern C:\Users\LFRAD\Documents\CMS2Luc\ProjetsNettoyesCMSGit\ProjetCarteIO\project\ETH97J60.c
       __MACPutROMArray:1   0x000aa2       data     extern C:\Users\LFRAD\Documents\CMS2Luc\ProjetsNettoyesCMSGit\ProjetCarteIO\project\ETH97J60.c
        __MACSetReadPtr:0   0x000a88       data     extern C:\Users\LFRAD\Documents\CMS2Luc\ProjetsNettoyesCMSGit\ProjetCarteIO\project\ETH97J60.c
    __MACSetReadPtrInRx:0   0x000a84       data     extern C:\Users\LFRAD\Documents\CMS2Luc\ProjetsNettoyesCMSGit\ProjetCarteIO\project\ETH97J60.c
       __MACSetWritePtr:0   0x000a86       data     extern C:\Users\LFRAD\Documents\CMS2Luc\ProjetsNettoyesCMSGit\ProjetCarteIO\project\ETH97J60.c
__MODIFICATION_TABLE_DEXISTENCE:0   0x0006a9       data     extern C:\Users\LFRAD\Documents\CMS2Luc\ProjetsNettoyesCMSGit\ProjetCarteIO\project\MainDemoV1.c
__MODIFICATION_TABLE_DEXISTENCE:1   0x0006ab       data     extern C:\Users\LFRAD\Documents\CMS2Luc\ProjetsNettoyesCMSGit\ProjetCarteIO\project\MainDemoV1.c
__MODIFICATION_TABLE_DEXISTENCE:2   0x0006ac       data     extern C:\Users\LFRAD\Documents\CMS2Luc\ProjetsNettoyesCMSGit\ProjetCarteIO\project\MainDemoV1.c
             __MOUCHARD:0   0x000692       data     extern C:\Users\LFRAD\Documents\CMS2Luc\ProjetsNettoyesCMSGit\ProjetCarteIO\project\MainDemoV1.c
       __RECEVOIR_RS485:0   0x0006b4       data     extern C:\Users\LFRAD\Documents\CMS2Luc\ProjetsNettoyesCMSGit\ProjetCarteIO\project\MainDemoV1.c
                  __REMB0   0x000005       data     extern E:\MPASM_MPLINK_PIC18_LT_Branch_3_42\pic18-lt\cxx-framework\src\traditional\math\aarg.asm
                  __REMB1   0x000004       data     extern E:\MPASM_MPLINK_PIC18_LT_Branch_3_42\pic18-lt\cxx-framework\src\traditional\math\aarg.asm
                  __REMB2   0x000003       data     extern E:\MPASM_MPLINK_PIC18_LT_Branch_3_42\pic18-lt\cxx-framework\src\traditional\math\aarg.asm
                  __REMB3   0x000002       data     extern E:\MPASM_MPLINK_PIC18_LT_Branch_3_42\pic18-lt\cxx-framework\src\traditional\math\aarg.asm
 __ROMStringToIPAddress:0   0x000a08       data     extern C:\Users\LFRAD\Documents\CMS2Luc\ProjetsNettoyesCMSGit\ProjetCarteIO\project\Helpers.c
 __ROMStringToIPAddress:1   0x000a0b       data     extern C:\Users\LFRAD\Documents\CMS2Luc\ProjetsNettoyesCMSGit\ProjetCarteIO\project\Helpers.c
                __RS485:0   0x0006bf       data     extern C:\Users\LFRAD\Documents\CMS2Luc\ProjetsNettoyesCMSGit\ProjetCarteIO\project\MainDemoV1.c
           __ReadPHYReg:0   0x000aa4       data     extern C:\Users\LFRAD\Documents\CMS2Luc\ProjetsNettoyesCMSGit\ProjetCarteIO\project\ETH97J60.c
       __SAV_CHG_ALARME:0   0x0006c5       data     extern C:\Users\LFRAD\Documents\CMS2Luc\ProjetsNettoyesCMSGit\ProjetCarteIO\project\MainDemoV1.c
        __SAV_EXISTENCE:0   0x0006b6       data     extern C:\Users\LFRAD\Documents\CMS2Luc\ProjetsNettoyesCMSGit\ProjetCarteIO\project\MainDemoV1.c
              __SendTCP:0   0x0007ad       data     static C:\Users\LFRAD\Documents\CMS2Luc\ProjetsNettoyesCMSGit\ProjetCarteIO\project\TCP.c
              __SendTCP:1   0x0007ae       data     static C:\Users\LFRAD\Documents\CMS2Luc\ProjetsNettoyesCMSGit\ProjetCarteIO\project\TCP.c
    __StringToIPAddress:0   0x000a04       data     extern C:\Users\LFRAD\Documents\CMS2Luc\ProjetsNettoyesCMSGit\ProjetCarteIO\project\Helpers.c
    __StringToIPAddress:1   0x000a06       data     extern C:\Users\LFRAD\Documents\CMS2Luc\ProjetsNettoyesCMSGit\ProjetCarteIO\project\Helpers.c
        __SwapARPPacket:0   0x0006fa       data     extern C:\Users\LFRAD\Documents\CMS2Luc\ProjetsNettoyesCMSGit\ProjetCarteIO\project\ARP.c
         __SwapIPHeader:0   0x0005fa       data     static C:\Users\LFRAD\Documents\CMS2Luc\ProjetsNettoyesCMSGit\ProjetCarteIO\project\IP.c
        __SwapTCPHeader:0   0x0007b3       data     static C:\Users\LFRAD\Documents\CMS2Luc\ProjetsNettoyesCMSGit\ProjetCarteIO\project\TCP.c
          __SyncTCBStub:0   0x000745       data     static C:\Users\LFRAD\Documents\CMS2Luc\ProjetsNettoyesCMSGit\ProjetCarteIO\project\TCP.c
    __TCPAdjustFIFOSize:0   0x0007b9       data     extern C:\Users\LFRAD\Documents\CMS2Luc\ProjetsNettoyesCMSGit\ProjetCarteIO\project\TCP.c
    __TCPAdjustFIFOSize:1   0x0007ba       data     extern C:\Users\LFRAD\Documents\CMS2Luc\ProjetsNettoyesCMSGit\ProjetCarteIO\project\TCP.c
    __TCPAdjustFIFOSize:2   0x0007bc       data     extern C:\Users\LFRAD\Documents\CMS2Luc\ProjetsNettoyesCMSGit\ProjetCarteIO\project\TCP.c
    __TCPAdjustFIFOSize:3   0x0007be       data     extern C:\Users\LFRAD\Documents\CMS2Luc\ProjetsNettoyesCMSGit\ProjetCarteIO\project\TCP.c
             __TCPClose:0   0x000751       data     extern C:\Users\LFRAD\Documents\CMS2Luc\ProjetsNettoyesCMSGit\ProjetCarteIO\project\TCP.c
           __TCPDiscard:0   0x000776       data     extern C:\Users\LFRAD\Documents\CMS2Luc\ProjetsNettoyesCMSGit\ProjetCarteIO\project\TCP.c
        __TCPDisconnect:0   0x000750       data     extern C:\Users\LFRAD\Documents\CMS2Luc\ProjetsNettoyesCMSGit\ProjetCarteIO\project\TCP.c
       __TCPFindArrayEx:0   0x00078b       data     extern C:\Users\LFRAD\Documents\CMS2Luc\ProjetsNettoyesCMSGit\ProjetCarteIO\project\TCP.c
       __TCPFindArrayEx:1   0x00078c       data     extern C:\Users\LFRAD\Documents\CMS2Luc\ProjetsNettoyesCMSGit\ProjetCarteIO\project\TCP.c
       __TCPFindArrayEx:2   0x00078e       data     extern C:\Users\LFRAD\Documents\CMS2Luc\ProjetsNettoyesCMSGit\ProjetCarteIO\project\TCP.c
       __TCPFindArrayEx:3   0x000790       data     extern C:\Users\LFRAD\Documents\CMS2Luc\ProjetsNettoyesCMSGit\ProjetCarteIO\project\TCP.c
       __TCPFindArrayEx:4   0x000792       data     extern C:\Users\LFRAD\Documents\CMS2Luc\ProjetsNettoyesCMSGit\ProjetCarteIO\project\TCP.c
       __TCPFindArrayEx:5   0x000794       data     extern C:\Users\LFRAD\Documents\CMS2Luc\ProjetsNettoyesCMSGit\ProjetCarteIO\project\TCP.c
            __TCPFindEx:0   0x0007a0       data     extern C:\Users\LFRAD\Documents\CMS2Luc\ProjetsNettoyesCMSGit\ProjetCarteIO\project\TCP.c
            __TCPFindEx:1   0x0007a1       data     extern C:\Users\LFRAD\Documents\CMS2Luc\ProjetsNettoyesCMSGit\ProjetCarteIO\project\TCP.c
            __TCPFindEx:2   0x0007a2       data     extern C:\Users\LFRAD\Documents\CMS2Luc\ProjetsNettoyesCMSGit\ProjetCarteIO\project\TCP.c
            __TCPFindEx:3   0x0007a4       data     extern C:\Users\LFRAD\Documents\CMS2Luc\ProjetsNettoyesCMSGit\ProjetCarteIO\project\TCP.c
            __TCPFindEx:4   0x0007a6       data     extern C:\Users\LFRAD\Documents\CMS2Luc\ProjetsNettoyesCMSGit\ProjetCarteIO\project\TCP.c
    __TCPFindROMArrayEx:0   0x000795       data     extern C:\Users\LFRAD\Documents\CMS2Luc\ProjetsNettoyesCMSGit\ProjetCarteIO\project\TCP.c
    __TCPFindROMArrayEx:1   0x000796       data     extern C:\Users\LFRAD\Documents\CMS2Luc\ProjetsNettoyesCMSGit\ProjetCarteIO\project\TCP.c
    __TCPFindROMArrayEx:2   0x000799       data     extern C:\Users\LFRAD\Documents\CMS2Luc\ProjetsNettoyesCMSGit\ProjetCarteIO\project\TCP.c
    __TCPFindROMArrayEx:3   0x00079b       data     extern C:\Users\LFRAD\Documents\CMS2Luc\ProjetsNettoyesCMSGit\ProjetCarteIO\project\TCP.c
    __TCPFindROMArrayEx:4   0x00079d       data     extern C:\Users\LFRAD\Documents\CMS2Luc\ProjetsNettoyesCMSGit\ProjetCarteIO\project\TCP.c
    __TCPFindROMArrayEx:5   0x00079f       data     extern C:\Users\LFRAD\Documents\CMS2Luc\ProjetsNettoyesCMSGit\ProjetCarteIO\project\TCP.c
             __TCPFlush:0   0x00075f       data     extern C:\Users\LFRAD\Documents\CMS2Luc\ProjetsNettoyesCMSGit\ProjetCarteIO\project\TCP.c
               __TCPGet:0   0x000778       data     extern C:\Users\LFRAD\Documents\CMS2Luc\ProjetsNettoyesCMSGit\ProjetCarteIO\project\TCP.c
               __TCPGet:1   0x000779       data     extern C:\Users\LFRAD\Documents\CMS2Luc\ProjetsNettoyesCMSGit\ProjetCarteIO\project\TCP.c
          __TCPGetArray:0   0x00077b       data     extern C:\Users\LFRAD\Documents\CMS2Luc\ProjetsNettoyesCMSGit\ProjetCarteIO\project\TCP.c
          __TCPGetArray:1   0x00077c       data     extern C:\Users\LFRAD\Documents\CMS2Luc\ProjetsNettoyesCMSGit\ProjetCarteIO\project\TCP.c
          __TCPGetArray:2   0x00077e       data     extern C:\Users\LFRAD\Documents\CMS2Luc\ProjetsNettoyesCMSGit\ProjetCarteIO\project\TCP.c
     __TCPGetRemoteInfo:0   0x000752       data     extern C:\Users\LFRAD\Documents\CMS2Luc\ProjetsNettoyesCMSGit\ProjetCarteIO\project\TCP.c
     __TCPGetRxFIFOFree:0   0x000780       data     extern C:\Users\LFRAD\Documents\CMS2Luc\ProjetsNettoyesCMSGit\ProjetCarteIO\project\TCP.c
     __TCPGetTxFIFOFull:0   0x000775       data     extern C:\Users\LFRAD\Documents\CMS2Luc\ProjetsNettoyesCMSGit\ProjetCarteIO\project\TCP.c
       __TCPIsConnected:0   0x00074f       data     extern C:\Users\LFRAD\Documents\CMS2Luc\ProjetsNettoyesCMSGit\ProjetCarteIO\project\TCP.c
        __TCPIsGetReady:0   0x000777       data     extern C:\Users\LFRAD\Documents\CMS2Luc\ProjetsNettoyesCMSGit\ProjetCarteIO\project\TCP.c
        __TCPIsPutReady:0   0x000760       data     extern C:\Users\LFRAD\Documents\CMS2Luc\ProjetsNettoyesCMSGit\ProjetCarteIO\project\TCP.c
              __TCPOpen:0   0x000746       data     extern C:\Users\LFRAD\Documents\CMS2Luc\ProjetsNettoyesCMSGit\ProjetCarteIO\project\TCP.c
              __TCPOpen:1   0x00074a       data     extern C:\Users\LFRAD\Documents\CMS2Luc\ProjetsNettoyesCMSGit\ProjetCarteIO\project\TCP.c
              __TCPOpen:2   0x00074b       data     extern C:\Users\LFRAD\Documents\CMS2Luc\ProjetsNettoyesCMSGit\ProjetCarteIO\project\TCP.c
              __TCPOpen:3   0x00074d       data     extern C:\Users\LFRAD\Documents\CMS2Luc\ProjetsNettoyesCMSGit\ProjetCarteIO\project\TCP.c
              __TCPPeek:0   0x000788       data     extern C:\Users\LFRAD\Documents\CMS2Luc\ProjetsNettoyesCMSGit\ProjetCarteIO\project\TCP.c
              __TCPPeek:1   0x000789       data     extern C:\Users\LFRAD\Documents\CMS2Luc\ProjetsNettoyesCMSGit\ProjetCarteIO\project\TCP.c
         __TCPPeekArray:0   0x000781       data     extern C:\Users\LFRAD\Documents\CMS2Luc\ProjetsNettoyesCMSGit\ProjetCarteIO\project\TCP.c
         __TCPPeekArray:1   0x000782       data     extern C:\Users\LFRAD\Documents\CMS2Luc\ProjetsNettoyesCMSGit\ProjetCarteIO\project\TCP.c
         __TCPPeekArray:2   0x000784       data     extern C:\Users\LFRAD\Documents\CMS2Luc\ProjetsNettoyesCMSGit\ProjetCarteIO\project\TCP.c
         __TCPPeekArray:3   0x000786       data     extern C:\Users\LFRAD\Documents\CMS2Luc\ProjetsNettoyesCMSGit\ProjetCarteIO\project\TCP.c
           __TCPProcess:0   0x0007a7       data     extern C:\Users\LFRAD\Documents\CMS2Luc\ProjetsNettoyesCMSGit\ProjetCarteIO\project\TCP.c
